 phoneutilityG

 Timestamp is 54004943 (Fri Aug 29 17:34:59 2014)

 Preferred load address is 00010000

 Start         Length     Name                   Class
 0001:00000000 00019d08H .text                   CODE
 0001:00019d08 00003180H .text$yc                CODE
 0002:00000000 0000f88cH .rdata                  DATA
 0002:0000f88c 00000230H .xdata                  DATA
 0002:0000fabc 00000050H .idata$2                DATA
 0002:0000fb0c 00000014H .idata$3                DATA
 0002:0000fb20 00000340H .idata$4                DATA
 0002:0000fe60 0000059cH .idata$6                DATA
 0002:000103fc 00000000H .edata                  DATA
 0003:00000000 00000340H .idata$5                DATA
 0003:00000340 00000004H .CRT$XCA                DATA
 0003:00000344 00000004H .CRT$XCAA               DATA
 0003:00000348 00000630H .CRT$XCU                DATA
 0003:00000978 00000004H .CRT$XCZ                DATA
 0003:0000097c 00000004H .CRT$XIA                DATA
 0003:00000980 00000004H .CRT$XIZ                DATA
 0003:00000984 00000004H .CRT$XPA                DATA
 0003:00000988 00000004H .CRT$XPZ                DATA
 0003:0000098c 00000004H .CRT$XTA                DATA
 0003:00000990 00000004H .CRT$XTZ                DATA
 0003:00000998 000004e0H .data                   DATA
 0003:00000e78 000061a5H .bss                    DATA
 0004:00000000 00001488H .pdata                  DATA
 0005:00000000 000000a0H .rsrc$01                DATA
 0005:000000a0 000003dcH .rsrc$02                DATA

  Address         Publics by Value              Rva+Base       Lib:Object

 0000:00000000       ___safe_se_handler_count   00000000     <absolute>
 0000:00000000       ___safe_se_handler_table   00000000     <absolute>
 0001:00000000       ?SaveDDTM@@YAHXZ           00011000 f   advanceddlg.obj
 0001:00000104       ?InitializeAdvanceDlg@@YAHPAUHWND__@@@Z 00011104 f   advanceddlg.obj
 0001:000004ec       ?InitAdvanceDlg@@YAHPAUHWND__@@@Z 000114ec f   advanceddlg.obj
 0001:000006a8       ?WndProcAdvance@@YAHPAUHWND__@@IIJ@Z 000116a8 f   advanceddlg.obj
 0001:000007b0       ?CreateAdvanceDlg@@YAHPAUHWND__@@@Z 000117b0 f   advanceddlg.obj
 0001:000009a0       ?UpdateMenu@@YAXH@Z        000119a0 f   authkey.obj
 0001:00000a38       ?OnMenuPopup@@YAHPAUHWND__@@I@Z 00011a38 f   authkey.obj
 0001:00000b20       ?UpdateCancelMenu@@YAXH@Z  00011b20 f   authkey.obj
 0001:00000b68       ?RenderAllUIControls@@YAXPAUHWND__@@H@Z 00011b68 f   authkey.obj
 0001:00000d3c       ?InitializeAuthKey@@YAHPAUHWND__@@@Z 00011d3c f   authkey.obj
 0001:00000ea0       ?OnSaveAkey@@YAHPAUHWND__@@@Z 00011ea0 f   authkey.obj
 0001:00001094       ?OnSaveMNAuthenticator@@YAHPAUHWND__@@@Z 00012094 f   authkey.obj
 0001:00001364       ?OnChangeMnAuthr@@YAXPAUHWND__@@@Z 00012364 f   authkey.obj
 0001:000013e0       ?OnChangeAkey@@YAXPAUHWND__@@@Z 000123e0 f   authkey.obj
 0001:00001450       ?InitAuthKeyDlg@@YAHPAUHWND__@@@Z 00012450 f   authkey.obj
 0001:0000166c       ?ProcessAuthKeyCtlChange@@YAHIJ@Z 0001266c f   authkey.obj
 0001:000016d0       ?WndProcAuthKey@@YAHPAUHWND__@@IIJ@Z 000126d0 f   authkey.obj
 0001:0000188c       ?CreateAuthKeyDlg@@YAHPAUHWND__@@@Z 0001288c f   authkey.obj
 0001:00001aa8       ?InitBrowserDlg@@YAHPAUHWND__@@@Z 00012aa8 f   browserdlg.obj
 0001:00001c2c       ?WndProcBrowserDlg@@YAHPAUHWND__@@IIJ@Z 00012c2c f   browserdlg.obj
 0001:00001cfc       ?CreateBrowserDlg@@YAHPAUHWND__@@@Z 00012cfc f   browserdlg.obj
 0001:00001ee4       ?ResetCounts@@YAXXZ        00012ee4 f   bwmeterdlg.obj
 0001:00002038       ?UpdateMeters@@YAXXZ       00013038 f   bwmeterdlg.obj
 0001:00002550       ?InitializeBWMeterDlgClass@@YAHPAUHWND__@@@Z 00013550 f   bwmeterdlg.obj
 0001:0000277c       ?PollingThreadProc@@YAKPAX@Z 0001377c f   bwmeterdlg.obj
 0001:00002b4c       ?KillPollingThread@@YAXXZ  00013b4c f   bwmeterdlg.obj
 0001:00002ba8       ?OnSetActive@@YAHPAUHWND__@@@Z 00013ba8 f   bwmeterdlg.obj
 0001:00002cd4       ?OnTimer@@YAXPAUHWND__@@I@Z 00013cd4 f   bwmeterdlg.obj
 0001:00002d74       ?OnRxMaxSelect@@YAHPAUHWND__@@H@Z 00013d74 f   bwmeterdlg.obj
 0001:00002e7c       ?OnTxMaxSelect@@YAHPAUHWND__@@H@Z 00013e7c f   bwmeterdlg.obj
 0001:00002f8c       ?InitBWMeterDlgClass@@YAHPAUHWND__@@@Z 00013f8c f   bwmeterdlg.obj
 0001:00003148       ?CloseBWDialog@@YAXPAUHWND__@@@Z 00014148 f   bwmeterdlg.obj
 0001:00003180       ?WndProcBWMeter@@YAHPAUHWND__@@IIJ@Z 00014180 f   bwmeterdlg.obj
 0001:00003354       ?CreateBandWidthMeterDlg@@YAHPAUHWND__@@@Z 00014354 f   bwmeterdlg.obj
 0001:00003460       ?InitializeConfigDlg@@YAHPAUHWND__@@@Z 00014460 f   configdlg.obj
 0001:000038c8       ?InitConfigDlg@@YAHPAUHWND__@@@Z 000148c8 f   configdlg.obj
 0001:00003a6c       ?WndProcConfig@@YAHPAUHWND__@@IIJ@Z 00014a6c f   configdlg.obj
 0001:00003b3c       ?CreateConfigDlg@@YAHPAUHWND__@@@Z 00014b3c f   configdlg.obj
 0001:00003d54       ?InitializeEVDODlg@@YAHPAUHWND__@@@Z 00014d54 f   evdo.obj
 0001:00003f8c       ?UpdateTechHdrInfo@@YAHXZ  00014f8c f   evdo.obj
 0001:0000467c       ?InitEVDODlg@@YAHPAUHWND__@@@Z 0001567c f   evdo.obj
 0001:00004858       ?WndProcEVDODlg@@YAHPAUHWND__@@IIJ@Z 00015858 f   evdo.obj
 0001:00004a50       ?CreateEVDODlg@@YAHPAUHWND__@@@Z 00015a50 f   evdo.obj
 0001:00004c4c       ?UpdateFingerInfo@@YAXXZ   00015c4c f   finger.obj
 0001:00004f90       ?InitializeFingerDlg@@YAHPAUHWND__@@@Z 00015f90 f   finger.obj
 0001:00005300       ?InitFinger@@YAHPAUHWND__@@@Z 00016300 f   finger.obj
 0001:000054cc       ?WndProcFinger@@YAHPAUHWND__@@IIJ@Z 000164cc f   finger.obj
 0001:00005664       ?CreateFingerDlg@@YAHPAUHWND__@@@Z 00016664 f   finger.obj
 0001:00005850       ?FormatLatLon@@YAXHPAG@Z   00016850 f   gpsdatadlg.obj
 0001:000059d8       ?TimeFromSecs@@YAXKPAGI@Z  000169d8 f   gpsdatadlg.obj
 0001:00005a44       ?OnLBSMenuPopup@@YAHPAUHWND__@@I@Z 00016a44 f   gpsdatadlg.obj
 0001:00005aa4       ?updateLbsData@@YAHXZ      00016aa4 f   gpsdatadlg.obj
 0001:00005c28       ?ReaddataFromCtrl@@YAHXZ   00016c28 f   gpsdatadlg.obj
 0001:00005d28       ?ReadGpsPDdata@@YAHXZ      00016d28 f   gpsdatadlg.obj
 0001:00005e10       ?PopulateLBSDataCtrls@@YAHXZ 00016e10 f   gpsdatadlg.obj
 0001:00005f4c       ?EnableControls@@YAHH@Z    00016f4c f   gpsdatadlg.obj
 0001:00005fa0       ?InitializeGPSDataDlgClass@@YAHPAUHWND__@@@Z 00016fa0 f   gpsdatadlg.obj
 0001:00006094       ?OnStopTrack@@YAHPAUHWND__@@@Z 00017094 f   gpsdatadlg.obj
 0001:00006180       ?OnStartTrack@@YAHPAUHWND__@@@Z 00017180 f   gpsdatadlg.obj
 0001:000062c8       ?InitGpsDataDlgClass@@YAHPAUHWND__@@@Z 000172c8 f   gpsdatadlg.obj
 0001:000064b8       ?WndProcGPSData@@YAHPAUHWND__@@IIJ@Z 000174b8 f   gpsdatadlg.obj
 0001:00006774       ?CreateGpsDataDlg@@YAHPAUHWND__@@@Z 00017774 f   gpsdatadlg.obj
 0001:00006964       ?IsValidPortID@@YAHPAG@Z   00017964 f   gpssettingsdlg.obj
 0001:00006a28       ?IsValidIP@@YAHPAG@Z       00017a28 f   gpssettingsdlg.obj
 0001:00006b0c       ?updateLBSSetsData@@YAHXZ  00017b0c f   gpssettingsdlg.obj
 0001:00006c3c       ?PopulateLBSSetsCtrls@@YAHXZ 00017c3c f   gpssettingsdlg.obj
 0001:00006e8c       ?GetdataFromCtrls@@YAHXZ   00017e8c f   gpssettingsdlg.obj
 0001:000071e8       ?ReadGpsSettings@@YAHXZ    000181e8 f   gpssettingsdlg.obj
 0001:000072ac       ?SaveGpsSettings@@YAHXZ    000182ac f   gpssettingsdlg.obj
 0001:000073c0       ?InitializeGpsSettingsDlgClass@@YAHPAUHWND__@@@Z 000183c0 f   gpssettingsdlg.obj
 0001:00007520       ?InitGpsSettingsDlgClass@@YAHPAUHWND__@@@Z 00018520 f   gpssettingsdlg.obj
 0001:000076e0       ?WndProcGPSSettings@@YAHPAUHWND__@@IIJ@Z 000186e0 f   gpssettingsdlg.obj
 0001:00007864       ?CreateGpsSettingsDlg@@YAHPAUHWND__@@@Z 00018864 f   gpssettingsdlg.obj
 0001:00007a50       ?UpdateGSM2GInfo@@YAHPAUHWND__@@@Z 00018a50 f   gsm2G.obj
 0001:00007ad0       ?InitializeGSM2G@@YAHPAUHWND__@@@Z 00018ad0 f   gsm2G.obj
 0001:00007b98       ?InitGSM2G@@YAHPAUHWND__@@@Z 00018b98 f   gsm2G.obj
 0001:00007d50       ?WndProcGSM2G@@YAHPAUHWND__@@IIJ@Z 00018d50 f   gsm2G.obj
 0001:00007ec4       ?CreateGSM2GDlg@@YAHPAUHWND__@@@Z 00018ec4 f   gsm2G.obj
 0001:0000804c       ?DeallocateListView@@YAXPAUHWND__@@@Z 0001904c f   gsm3G.obj
 0001:000080ec       ?ParseAndBuildDynamicList@@YAXPAUHWND__@@PAG@Z 000190ec f   gsm3G.obj
 0001:00008278       ?UpdateGSM3GItemnizeInfo@@YAHPAUHWND__@@J@Z 00019278 f   gsm3G.obj
 0001:0000831c       ?InitializeGSM3G@@YAHPAUHWND__@@@Z 0001931c f   gsm3G.obj
 0001:000083a4       ?InitGSM3G@@YAHPAUHWND__@@@Z 000193a4 f   gsm3G.obj
 0001:0000854c       ?InitializeGSM3GItemnize@@YAHPAUHWND__@@J@Z 0001954c f   gsm3G.obj
 0001:00008644       ?InitGSM3GItemnize@@YAHPAUHWND__@@J@Z 00019644 f   gsm3G.obj
 0001:00008808       ?WndProcGSM3GItemnize@@YAHPAUHWND__@@IIJ@Z 00019808 f   gsm3G.obj
 0001:00008988       ?CreateGSM3GDlgItemnize@@YAHPAUHWND__@@@Z 00019988 f   gsm3G.obj
 0001:00008b14       ?WndProcGSM3G@@YAHPAUHWND__@@IIJ@Z 00019b14 f   gsm3G.obj
 0001:00008d18       ?CreateGSM3GDlg@@YAHPAUHWND__@@@Z 00019d18 f   gsm3G.obj
 0001:00008ea4       ?DeallocateGSMBandListView@@YAXPAUHWND__@@@Z 00019ea4 f   gsmband.obj
 0001:00008f3c       ?ParseAndBuildDynamicList@@YAXPAUHWND__@@KPAUtagRILBANDINFO@@@Z 00019f3c f   gsmband.obj
 0001:00009070       ?GetGSMBandInfo@@YAHPAUHWND__@@@Z 0001a070 f   gsmband.obj
 0001:000090e8       ?InitializeGSMBand@@YAHPAUHWND__@@@Z 0001a0e8 f   gsmband.obj
 0001:00009164       ?InitGSMBand@@YAHPAUHWND__@@@Z 0001a164 f   gsmband.obj
 0001:000092f4       ?WndProcGSMBand@@YAHPAUHWND__@@IIJ@Z 0001a2f4 f   gsmband.obj
 0001:0000953c       ?CreateGSMBandDlg@@YAHPAUHWND__@@@Z 0001a53c f   gsmband.obj
 0001:000096d0       ?InitIOTADlg@@YAHPAUHWND__@@@Z 0001a6d0 f   iota.obj
 0001:00009858       ?WndProcIOTA@@YAHPAUHWND__@@IIJ@Z 0001a858 f   iota.obj
 0001:00009928       ?CreateIOTADlg@@YAHPAUHWND__@@@Z 0001a928 f   iota.obj
 0001:00009b10       ?CreateListView@@YAPAUHWND__@@PAU1@@Z 0001ab10 f   listview.obj
 0001:00009c04       ?CleanupListView@@YAXPAUHWND__@@@Z 0001ac04 f   listview.obj
 0001:00009c20       ?InitializeList@@YAXPAUHWND__@@0@Z 0001ac20 f   listview.obj
 0001:0000a0a0       ?OnListViewNotify@@YAJPAUHWND__@@J@Z 0001b0a0 f   listview.obj
 0001:0000a1e0       ?FillServiceOption@@YAXPAUHWND__@@@Z 0001b1e0 f   loopbackdlg.obj
 0001:0000a294       ?onCallHangup@@YAHPAUHWND__@@@Z 0001b294 f   loopbackdlg.obj
 0001:0000a320       ?onCallEstablish@@YAHPAUHWND__@@@Z 0001b320 f   loopbackdlg.obj
 0001:0000a47c       ?InitializeLoopBackDlg@@YAHPAUHWND__@@@Z 0001b47c f   loopbackdlg.obj
 0001:0000a560       ?CheckForCallStatus@@YAXXZ 0001b560 f   loopbackdlg.obj
 0001:0000a7c8       ?InitLoopBackDlg@@YAHPAUHWND__@@@Z 0001b7c8 f   loopbackdlg.obj
 0001:0000aa6c       ?OnChangeNumber@@YAHPAUHWND__@@0@Z 0001ba6c f   loopbackdlg.obj
 0001:0000abf8       ?ProcessLoopbackCtlChange@@YAHPAUHWND__@@IJ@Z 0001bbf8 f   loopbackdlg.obj
 0001:0000ac48       ?WndProcLoopBackDlg@@YAHPAUHWND__@@IIJ@Z 0001bc48 f   loopbackdlg.obj
 0001:0000ad80       ?CreateLoopBackDlg@@YAHPAUHWND__@@@Z 0001bd80 f   loopbackdlg.obj
 0001:0000af6c       ?CreateMainMenu@@YAHPAUHWND__@@@Z 0001bf6c f   mainfrm.obj
 0001:0000b020       ?InitializeTabFromIndex@@YAHPAUHWND__@@KHH@Z 0001c020 f   mainfrm.obj
 0001:0000b830       ?PrepareResourceDlg@@YAHPAUHWND__@@@Z 0001c830 f   mainfrm.obj
 0001:0000bef8       ?OnCreateMainWnd@@YAHPAUHWND__@@@Z 0001cef8 f   mainfrm.obj
 0001:0000bfa4       ?MainWndProc@@YAJPAUHWND__@@IIJ@Z 0001cfa4 f   mainfrm.obj
 0001:0000c354       ?RegisterMainWnd@@YAHXZ    0001d354 f   mainfrm.obj
 0001:0000c428       ?CreateMainWnd@@YAHH@Z     0001d428 f   mainfrm.obj
 0001:0000c504       ?SaveMSL@@YAXPAUHWND__@@@Z 0001d504 f   msldlg.obj
 0001:0000c8ac       ?FillAccolc@@YAXPAUHWND__@@G@Z 0001d8ac f   msldlg.obj
 0001:0000c978       ?FillSlotCycle@@YAXPAUHWND__@@G@Z 0001d978 f   msldlg.obj
 0001:0000ca44       ?InitializeMslDlg@@YAHPAUHWND__@@@Z 0001da44 f   msldlg.obj
 0001:0000cf34       ?EnablesaveMenu@@YAXXZ     0001df34 f   msldlg.obj
 0001:0000cfc0       ?OnChangeNumberMsid@@YAXPAUHWND__@@@Z 0001dfc0 f   msldlg.obj
 0001:0000cffc       ?OnChangeEditSid@@YAXPAUHWND__@@@Z 0001dffc f   msldlg.obj
 0001:0000d094       ?OnChangeEditNid@@YAXPAUHWND__@@@Z 0001e094 f   msldlg.obj
 0001:0000d12c       ?OnChangeEditMcc@@YAXPAUHWND__@@@Z 0001e12c f   msldlg.obj
 0001:0000d1c4       ?OnChangeEditMnc@@YAXPAUHWND__@@@Z 0001e1c4 f   msldlg.obj
 0001:0000d24c       ?ProcessMSLDlgCtlChange@@YAHIJ@Z 0001e24c f   msldlg.obj
 0001:0000d370       ?InitMslDlg@@YAHPAUHWND__@@@Z 0001e370 f   msldlg.obj
 0001:0000d5d0       ?WndProcMsl@@YAHPAUHWND__@@IIJ@Z 0001e5d0 f   msldlg.obj
 0001:0000d740       ?CreateMslDlg@@YAHPAUHWND__@@@Z 0001e740 f   msldlg.obj
 0001:0000d958       ?UpdatePwrStatus@@YAHXZ    0001e958 f   network.obj
 0001:0000dd4c       ?InitializeNetworkDlg@@YAHPAUHWND__@@@Z 0001ed4c f   network.obj
 0001:0000df80       ?InitNetwork@@YAHPAUHWND__@@@Z 0001ef80 f   network.obj
 0001:0000e154       ?UpdateNetworkInfo@@YAHXZ  0001f154 f   network.obj
 0001:0000e6f4       ?WndProcNetwork@@YAHPAUHWND__@@IIJ@Z 0001f6f4 f   network.obj
 0001:0000e8a0       ?CreateNetworkDlg@@YAHPAUHWND__@@@Z 0001f8a0 f   network.obj
 0001:0000ea30       ?SaveOTKSL@@YAXPAUHWND__@@@Z 0001fa30 f   otksldlg.obj
 0001:0000ebe4       ?EnableSaveMenu@@YAXXZ     0001fbe4 f   otksldlg.obj
 0001:0000ec2c       ?OnChangeNumberMsidotksl@@YAXPAUHWND__@@@Z 0001fc2c f   otksldlg.obj
 0001:0000ec60       ?ProcessOTKSLCtlChange@@YAHIJ@Z 0001fc60 f   otksldlg.obj
 0001:0000ecf4       ?InitializeOtkslDlg@@YAHPAUHWND__@@@Z 0001fcf4 f   otksldlg.obj
 0001:0000ee7c       ?InitOtkslDlg@@YAHPAUHWND__@@@Z 0001fe7c f   otksldlg.obj
 0001:0000f08c       ?WndProcOtksl@@YAHPAUHWND__@@IIJ@Z 0002008c f   otksldlg.obj
 0001:0000f1ec       ?CreateOtkslDlg@@YAHPAUHWND__@@@Z 000201ec f   otksldlg.obj
 0001:0000f3d8       ?InitializePassThruDlg@@YAHPAUHWND__@@@Z 000203d8 f   passthrudlg.obj
 0001:0000f584       ?InitPassThruDlg@@YAHPAUHWND__@@@Z 00020584 f   passthrudlg.obj
 0001:0000f7a0       ?OnPasstruMenuPopup@@YAHPAUHWND__@@I@Z 000207a0 f   passthrudlg.obj
 0001:0000f7f8       ?WndProcPassThru@@YAHPAUHWND__@@IIJ@Z 000207f8 f   passthrudlg.obj
 0001:0000fbac       ?CreatePassThruDlg@@YAHPAUHWND__@@@Z 00020bac f   passthrudlg.obj
 0001:0000fdc0       ?GetInstanceHandle@@YAPAUHINSTANCE__@@XZ 00020dc0 f   phoneutility.obj
 0001:0000fdd0       ?GetResourceHandle@@YAPAUHINSTANCE__@@XZ 00020dd0 f   phoneutility.obj
 0001:0000fde0       ?GetCarrier@@YAKXZ         00020de0 f   phoneutility.obj
 0001:0000fdf0       ?GetActiveTab@@YAKXZ       00020df0 f   phoneutility.obj
 0001:0000fe00       ?SetWindowTopMost@@YAJPAUHWND__@@@Z 00020e00 f   phoneutility.obj
 0001:0000fe08       ?InitializeGlobalVars@@YAXXZ 00020e08 f   phoneutility.obj
 0001:0000ff0c       ?ParseParam@@YAKXZ         00020f0c f   phoneutility.obj
 0001:00010074       ?CheckPhoneUtilityCanrun@@YAHXZ 00021074 f   phoneutility.obj
 0001:00010120       ?ProcessSwapMenuBar@@YAHPAUHWND__@@0H@Z 00021120 f   phoneutility.obj
 0001:0001015c       ?GetStatus@@YAHXZ          0002115c f   phoneutility.obj
 0001:00010184       ?SpcValidation@@YAHPAUHWND__@@@Z 00021184 f   phoneutility.obj
 0001:0001025c       ?ValidateSpecialPassword@@YAHXZ 0002125c f   phoneutility.obj
 0001:00010264       ?DebugModeStart@@YAHXZ     00021264 f   phoneutility.obj
 0001:000102b4       ?DebugModeStop@@YAHXZ      000212b4 f   phoneutility.obj
 0001:00010304       ?EnableTechHdr@@YAHH@Z     00021304 f   phoneutility.obj
 0001:0001032c       ?GetTechHdrInfo@@YAHXZ     0002132c f   phoneutility.obj
 0001:000107f4       ?CheckDebugStatus@@YAHXZ   000217f4 f   phoneutility.obj
 0001:00010858       ?GetDebugInfo@@YAHXZ       00021858 f   phoneutility.obj
 0001:00010c24       ?GeoSecToDegMinSec@@YAXJAAJAAH1@Z 00021c24 f   phoneutility.obj
 0001:00010cb0       WinMain                    00021cb0 f   phoneutility.obj
 0001:00011094       ?InitializeRTNDlg@@YAHPAUHWND__@@@Z 00022094 f   rtndlg.obj
 0001:000111dc       ?OnInitRTNDialog@@YAHPAUHWND__@@@Z 000221dc f   rtndlg.obj
 0001:0001138c       ?WndProcRTN@@YAHPAUHWND__@@IIJ@Z 0002238c f   rtndlg.obj
 0001:000116a0       ?CreateRTNDlg@@YAHPAUHWND__@@@Z 000226a0 f   rtndlg.obj
 0001:000118b4       ?ReadQcMIP@@YAHXZ          000228b4 f   simpleipdlg.obj
 0001:00011964       ?InitializeSimpleIPDlg@@YAHPAUHWND__@@@Z 00022964 f   simpleipdlg.obj
 0001:00011c0c       ?SaveSimpleIPData@@YAHPAUHWND__@@@Z 00022c0c f   simpleipdlg.obj
 0001:00012034       ?InitSimpleIPDlg@@YAHPAUHWND__@@@Z 00023034 f   simpleipdlg.obj
 0001:000121f0       ?WndProcSimpleIP@@YAHPAUHWND__@@IIJ@Z 000231f0 f   simpleipdlg.obj
 0001:000122e0       ?CreateSimpleIPDlg@@YAHPAUHWND__@@@Z 000232e0 f   simpleipdlg.obj
 0001:000124d4       ?InitSipDlg@@YAHPAUHWND__@@@Z 000234d4 f   sipdlg.obj
 0001:00012664       ?WndProcSipDlg@@YAHPAUHWND__@@IIJ@Z 00023664 f   sipdlg.obj
 0001:00012734       ?CreateSipDlg@@YAHPAUHWND__@@@Z 00023734 f   sipdlg.obj
 0001:00012924       ?InitSPCValidation@@YAHPAUHWND__@@@Z 00023924 f   spcvalidation.obj
 0001:00012b14       ?WndProcSPCValidation@@YAHPAUHWND__@@IIJ@Z 00023b14 f   spcvalidation.obj
 0001:00012d34       ?CreateSPCValidation@@YAHPAUHWND__@@@Z 00023d34 f   spcvalidation.obj
 0001:00012f50       ?FillComboCtrls@@YAXPAUHWND__@@@Z 00023f50 f   systemdlg.obj
 0001:000132b8       ?GetoModemValues@@YAHPAUHWND__@@@Z 000242b8 f   systemdlg.obj
 0001:00013368       ?InitializeSystemDlg@@YAHPAUHWND__@@@Z 00024368 f   systemdlg.obj
 0001:000133e4       ?SaveSelectiontoModem@@YAHPAUHWND__@@@Z 000243e4 f   systemdlg.obj
 0001:00013668       ?InitSystemDlg@@YAHPAUHWND__@@@Z 00024668 f   systemdlg.obj
 0001:000137f8       ?WndProcSystemDlg@@YAHPAUHWND__@@IIJ@Z 000247f8 f   systemdlg.obj
 0001:000139ac       ?CreateSystemDlg@@YAHPAUHWND__@@@Z 000249ac f   systemdlg.obj
 0001:00013b98       ?PopulatePDPListcombo@@YAHPAUHWND__@@@Z 00024b98 f   usernamedlg.obj
 0001:00013c60       ?GetPDPList@@YAHPAUHWND__@@@Z 00024c60 f   usernamedlg.obj
 0001:00013d00       ?PopulateTheProfile@@YAXPAUHWND__@@@Z 00024d00 f   usernamedlg.obj
 0001:00013eb4       ?GetMipGenProfile@@YAHPAUHWND__@@H@Z 00024eb4 f   usernamedlg.obj
 0001:00013f6c       ?InitializeUsernameDlg@@YAHPAUHWND__@@@Z 00024f6c f   usernamedlg.obj
 0001:000140e4       ?UpdatePDPProfile@@YAHPAUHWND__@@@Z 000250e4 f   usernamedlg.obj
 0001:00014574       ?InitUsernameDlg@@YAHPAUHWND__@@@Z 00025574 f   usernamedlg.obj
 0001:00014708       ?WndProcUsername@@YAHPAUHWND__@@IIJ@Z 00025708 f   usernamedlg.obj
 0001:00014870       ?CreateUsernameDlg@@YAHPAUHWND__@@@Z 00025870 f   usernamedlg.obj
 0001:00014a68       ?InitializeVersionInfoDlg@@YAHPAUHWND__@@AAUtagRILVERNOINFO@@@Z 00025a68 f   versioninfo.obj
 0001:0001519c       ?InitVersionInfoDlg@@YAHPAUHWND__@@@Z 0002619c f   versioninfo.obj
 0001:00015380       ?WndProcVersionInfoDlg@@YAHPAUHWND__@@IIJ@Z 00026380 f   versioninfo.obj
 0001:000154d0       ?CreateVersionInfoDlg@@YAHPAUHWND__@@@Z 000264d0 f   versioninfo.obj
 0001:000156bc       ?ReadVOCODER@@YAHXZ        000266bc f   vocoderdlg.obj
 0001:000157b4       ?UpdatedListItem@@YAXPAUHWND__@@G@Z 000267b4 f   vocoderdlg.obj
 0001:00015888       ?InitializeVocoderDlg@@YAHPAUHWND__@@@Z 00026888 f   vocoderdlg.obj
 0001:00015b2c       ?InitVocoderDlg@@YAHPAUHWND__@@@Z 00026b2c f   vocoderdlg.obj
 0001:00015cfc       ?SaveVocoder@@YAHPAUHWND__@@@Z 00026cfc f   vocoderdlg.obj
 0001:00015fd0       ?WndProcVocoderDlg@@YAHPAUHWND__@@IIJ@Z 00026fd0 f   vocoderdlg.obj
 0001:00016100       ?CreateVocoderDlg@@YAHPAUHWND__@@@Z 00027100 f   vocoderdlg.obj
 0001:00016314       SendMessageW               00027314 f   coredll:COREDLL.dll
 0001:00016324       ??3@YAXPAX@Z               00027324 f   coredll:COREDLL.dll
 0001:00016334       _wcsicmp                   00027334 f   coredll:COREDLL.dll
 0001:00016344       LoadStringW                00027344 f   coredll:COREDLL.dll
 0001:00016354       GetWindowTextW             00027354 f   coredll:COREDLL.dll
 0001:00016364       wcsncpy                    00027364 f   coredll:COREDLL.dll
 0001:00016374       wcscpy                     00027374 f   coredll:COREDLL.dll
 0001:00016384       Sleep                      00027384 f   coredll:COREDLL.dll
 0001:00016394       swprintf                   00027394 f   coredll:COREDLL.dll
 0001:000163a4       SetWindowTextW             000273a4 f   coredll:COREDLL.dll
 0001:000163b4       GetDlgItem                 000273b4 f   coredll:COREDLL.dll
 0001:000163c4       SetDlgItemInt              000273c4 f   coredll:COREDLL.dll
 0001:000163d4       SetDlgItemTextW            000273d4 f   coredll:COREDLL.dll
 0001:000163e4       memset                     000273e4 f   coredll:COREDLL.dll
 0001:000163f4       EndDialog                  000273f4 f   coredll:COREDLL.dll
 0001:00016404       MessageBoxW                00027404 f   coredll:COREDLL.dll
 0001:00016414       SetFocus                   00027414 f   coredll:COREDLL.dll
 0001:00016424       DialogBoxIndirectParamW    00027424 f   coredll:COREDLL.dll
 0001:00016434       LoadResource               00027434 f   coredll:COREDLL.dll
 0001:00016444       FindResourceW              00027444 f   coredll:COREDLL.dll
 0001:00016454       GetLastError               00027454 f   coredll:COREDLL.dll
 0001:00016464       RegisterClassW             00027464 f   coredll:COREDLL.dll
 0001:00016474       GetStockObject             00027474 f   coredll:COREDLL.dll
 0001:00016484       RegisterWindowMessageW     00027484 f   coredll:COREDLL.dll
 0001:00016494       EnableMenuItem             00027494 f   coredll:COREDLL.dll
 0001:000164a4       wcslen                     000274a4 f   coredll:COREDLL.dll
 0001:000164b4       EnableWindow               000274b4 f   coredll:COREDLL.dll
 0001:000164c4       ShowWindow                 000274c4 f   coredll:COREDLL.dll
 0001:000164d4       _wtol                      000274d4 f   coredll:COREDLL.dll
 0001:000164e4       PostMessageW               000274e4 f   coredll:COREDLL.dll
 0001:000164f4       PostQuitMessage            000274f4 f   coredll:COREDLL.dll
 0001:00016504       TerminateThread            00027504 f   coredll:COREDLL.dll
 0001:00016514       WaitForSingleObject        00027514 f   coredll:COREDLL.dll
 0001:00016524       CreateThread               00027524 f   coredll:COREDLL.dll
 0001:00016534       KillTimer                  00027534 f   coredll:COREDLL.dll
 0001:00016544       SetTimer                   00027544 f   coredll:COREDLL.dll
 0001:00016554       MultiByteToWideChar        00027554 f   coredll:COREDLL.dll
 0001:00016564       SetWindowPos               00027564 f   coredll:COREDLL.dll
 0001:00016574       GetClientRect              00027574 f   coredll:COREDLL.dll
 0001:00016584       LeaveCriticalSection       00027584 f   coredll:COREDLL.dll
 0001:00016594       EnterCriticalSection       00027594 f   coredll:COREDLL.dll
 0001:000165a4       DeleteCriticalSection      000275a4 f   coredll:COREDLL.dll
 0001:000165b4       InitializeCriticalSection  000275b4 f   coredll:COREDLL.dll
 0001:000165c4       free                       000275c4 f   coredll:COREDLL.dll
 0001:000165d4       wcstombs                   000275d4 f   coredll:COREDLL.dll
 0001:000165e4       malloc                     000275e4 f   coredll:COREDLL.dll
 0001:000165f4       strlen                     000275f4 f   coredll:COREDLL.dll
 0001:00016604       sscanf                     00027604 f   coredll:COREDLL.dll
 0001:00016614       wcscmp                     00027614 f   coredll:COREDLL.dll
 0001:00016624       memcpy                     00027624 f   coredll:COREDLL.dll
 0001:00016634       HideCaret                  00027634 f   coredll:COREDLL.dll
 0001:00016644       GetWindowLongW             00027644 f   coredll:COREDLL.dll
 0001:00016654       ??2@YAPAXI@Z               00027654 f   coredll:COREDLL.dll
 0001:00016664       SetWindowLongW             00027664 f   coredll:COREDLL.dll
 0001:00016674       GetParent                  00027674 f   coredll:COREDLL.dll
 0001:00016684       CreateWindowExW            00027684 f   coredll:COREDLL.dll
 0001:00016694       DestroyWindow              00027694 f   coredll:COREDLL.dll
 0001:000166a4       IsWindow                   000276a4 f   coredll:COREDLL.dll
 0001:000166b4       wcscat                     000276b4 f   coredll:COREDLL.dll
 0001:000166c4       MessageBeep                000276c4 f   coredll:COREDLL.dll
 0001:000166d4       iswctype                   000276d4 f   coredll:COREDLL.dll
 0001:000166e4       OutputDebugStringW         000276e4 f   coredll:COREDLL.dll
 0001:000166f4       DefWindowProcW             000276f4 f   coredll:COREDLL.dll
 0001:00016704       UpdateWindow               00027704 f   coredll:COREDLL.dll
 0001:00016714       GetWindowTextLengthW       00027714 f   coredll:COREDLL.dll
 0001:00016724       LoadBitmapW                00027724 f   coredll:COREDLL.dll
 0001:00016734       _wcsupr                    00027734 f   coredll:COREDLL.dll
 0001:00016744       CloseHandle                00027744 f   coredll:COREDLL.dll
 0001:00016754       SetForegroundWindow        00027754 f   coredll:COREDLL.dll
 0001:00016764       FindWindowW                00027764 f   coredll:COREDLL.dll
 0001:00016774       GetMessageW                00027774 f   coredll:COREDLL.dll
 0001:00016784       DispatchMessageW           00027784 f   coredll:COREDLL.dll
 0001:00016794       TranslateMessage           00027794 f   coredll:COREDLL.dll
 0001:000167a4       CreateMutexW               000277a4 f   coredll:COREDLL.dll
 0001:000167b4       LoadLibraryW               000277b4 f   coredll:COREDLL.dll
 0001:000167c4       _isctype                   000277c4 f   coredll:COREDLL.dll
 0001:000167d4       SendDlgItemMessageW        000277d4 f   coredll:COREDLL.dll
 0001:000167e4       _wtoll                     000277e4 f   coredll:COREDLL.dll
 0001:000167f4       wsprintfW                  000277f4 f   coredll:COREDLL.dll
 0001:00016804       SetActiveWindow            00027804 f   coredll:COREDLL.dll
 0001:00016814       SHInitDialog               00027814 f   aygshell:AYGSHELL.dll
 0001:00016824       SHCreateMenuBar            00027824 f   aygshell:AYGSHELL.dll
 0001:0001683c       WinMainCRTStartup          0002783c f   corelibc:pegwmain.obj
 0001:000168b0       __security_check_cookie    000278b0     corelibc:armsecgs.obj
 0001:000168c4       __gsfailure                000278c4     corelibc:armsecgs.obj
 0001:00016908       _cinit                     00027908 f   corelibc:crt0dat.obj
 0001:00016a78       exit                       00027a78 f   corelibc:crt0dat.obj
 0001:00016a90       _exit                      00027a90 f   corelibc:crt0dat.obj
 0001:00016aa8       __security_init_cookie     00027aa8 f   corelibc:seccinit.obj
 0001:00016af8       __GSHandlerCheckCommon     00027af8 f   LIBCMT:gshandler.obj
 0001:00016b40       __GSHandlerCheck           00027b40 f   LIBCMT:gshandler.obj
 0001:00016d58       wcsftime                   00027d58 f   LIBCMT:wcsftime.obj
 0001:00016d74       _localtime64_s             00027d74 f   LIBCMT:loctim64.obj
 0001:00018718       _Strftime_l                00029718 f   LIBCMT:strftime.obj
 0001:00018950       _invalid_parameter         00029950 f   LIBCMT:invarginternal.obj
 0001:0001897c       _invoke_watson             0002997c f   LIBCMT:invarg.obj
 0001:000192bc       __tzset                    0002a2bc f   LIBCMT:tzset.obj
 0001:00019350       _isindst                   0002a350 f   LIBCMT:tzset.obj
 0001:000193bc       _gmtime64_s                0002a3bc f   LIBCMT:gmtime64.obj
 0001:000197a8       _get_daylight              0002a7a8 f   LIBCMT:timeset.obj
 0001:00019804       _get_dstbias               0002a804 f   LIBCMT:timeset.obj
 0001:00019860       _get_timezone              0002a860 f   LIBCMT:timeset.obj
 0001:000198bc       __daylight                 0002a8bc f   LIBCMT:timeset.obj
 0001:000198c8       __dstbias                  0002a8c8 f   LIBCMT:timeset.obj
 0001:000198d4       __timezone                 0002a8d4 f   LIBCMT:timeset.obj
 0001:000198e0       __tzname                   0002a8e0 f   LIBCMT:timeset.obj
 0001:000198ec       _mtinitlocks               0002a8ec f   LIBCMT:mlock.obj
 0001:0001996c       _unlock                    0002a96c f   LIBCMT:mlock.obj
 0001:0001999c       _mtinitlocknum             0002a99c f   LIBCMT:mlock.obj
 0001:00019a98       _lock                      0002aa98 f   LIBCMT:mlock.obj
 0001:00019b64       __crtInitCritSecAndSpinCount 0002ab64 f   LIBCMT:initcrit.obj
 0001:00019be0       _amsg_exit                 0002abe0 f   LIBCMT:crt0dat.obj
 0001:00019c04       __crtExitProcess           0002ac04 f   LIBCMT:crt0dat.obj
 0001:00019c28       _XcptFilter                0002ac28 f   coredll:COREDLL.dll
 0001:00019c38       __C_specific_handler       0002ac38 f   coredll:COREDLL.dll
 0001:00019c48       __report_gsfailure         0002ac48 f   coredll:COREDLL.dll
 0001:00019c58       LocalFree                  0002ac58 f   coredll:COREDLL.dll
 0001:00019c68       __security_gen_cookie      0002ac68 f   coredll:COREDLL.dll
 0001:00019c78       mbstowcs                   0002ac78 f   coredll:COREDLL.dll
 0001:00019c88       _stricmp                   0002ac88 f   coredll:COREDLL.dll
 0001:00019c98       GetTimeFormatW             0002ac98 f   coredll:COREDLL.dll
 0001:00019ca8       GetDateFormatW             0002aca8 f   coredll:COREDLL.dll
 0001:00019cb8       RaiseException             0002acb8 f   coredll:COREDLL.dll
 0001:00019cc8       WideCharToMultiByte        0002acc8 f   coredll:COREDLL.dll
 0001:00019cd8       GetTimeZoneInformation     0002acd8 f   coredll:COREDLL.dll
 0001:00019ce8       SetLastError               0002ace8 f   coredll:COREDLL.dll
 0001:00019cf8       TerminateProcess           0002acf8 f   coredll:COREDLL.dll
 0002:00000000       ??_C@_1CA@OEPBIHCL@?$AAA?$AAd?$AAv?$AAa?$AAn?$AAc?$AAe?$AAD?$AAl?$AAg?$AAC?$AAl?$AAa?$AAs?$AAs?$AA?$AA@ 0002e000     advanceddlg.obj
 0002:0000004c       ??_C@_1CE@OFHJHMBJ@?$AA?4?$AA?2?$AAa?$AAd?$AAv?$AAa?$AAn?$AAc?$AAe?$AAd?$AAd?$AAl?$AAg?$AA?4?$AAc?$AAp?$AAp?$AA?$AA@ 0002e04c     advanceddlg.obj
 0002:00000070       ??_C@_1GC@CBPJOIIC@?$AAN?$AAV?$AA_?$AAI?$AA_?$AAN?$AAV?$AA_?$AAP?$AAR?$AAE?$AAF?$AA_?$AAV?$AAO?$AAI?$AAC?$AAE?$AA_?$AAS?$AAO?$AA?5?$AAn?$AAv?$AA?5?$AAW?$AAr?$AAi?$AAt?$AAe?$AA?5?$AAf@ 0002e070     advanceddlg.obj
 0002:000000d4       ??_C@_11LOCGONAA@?$AA?$AA@ 0002e0d4     advanceddlg.obj
 0002:000000d8       ??_C@_15KNBIKKIN@?$AA?$CF?$AAd?$AA?$AA@ 0002e0d8     advanceddlg.obj
 0002:000000e0       ??_C@_1O@KPKDPEHK@?$AAU?$AAn?$AAk?$AAn?$AAo?$AAw?$AA?$AA@ 0002e0e0     advanceddlg.obj
 0002:000000f0       ??_C@_15MLPIMJOL@?$AAO?$AAN?$AA?$AA@ 0002e0f0     advanceddlg.obj
 0002:000000f8       ??_C@_17NBOBOEH@?$AAO?$AAF?$AAF?$AA?$AA@ 0002e0f8     advanceddlg.obj
 0002:00000100       ??_C@_1DG@BALLNLHK@?$AAG?$AAe?$AAt?$AAA?$AAd?$AAv?$AAa?$AAn?$AAc?$AAe?$AAd?$AAM?$AAe?$AAn?$AAu?$AAI?$AAn?$AAf?$AAo?$AA?5?$AAf?$AAa?$AAi?$AAl?$AAe?$AAd?$AA?$AA@ 0002e100     advanceddlg.obj
 0002:00000138       ??_C@_1EI@CPKPAKBP@?$AAI?$AAn?$AAi?$AAt?$AAA?$AAd?$AAv?$AAa?$AAn?$AAc?$AAe?$AAD?$AAl?$AAg?$AA?3?$AA?3?$AAS?$AAH?$AAI?$AAn?$AAi?$AAt?$AAD?$AAi?$AAa?$AAl?$AAo?$AAg?$AA?5?$AAF?$AAa?$AAl@ 0002e138     advanceddlg.obj
 0002:00000180       ??_C@_1EG@KJOFOGNB@?$AAI?$AAn?$AAi?$AAt?$AAA?$AAd?$AAv?$AAa?$AAn?$AAc?$AAe?$AAD?$AAl?$AAg?$AA?3?$AAS?$AAH?$AAI?$AAn?$AAi?$AAt?$AAD?$AAi?$AAa?$AAl?$AAo?$AAg?$AA?5?$AAF?$AAa?$AAi?$AAl@ 0002e180     advanceddlg.obj
 0002:000001c8       ??_C@_1EO@BLJDIFCE@?$AAI?$AAn?$AAi?$AAt?$AAA?$AAd?$AAv?$AAa?$AAn?$AAc?$AAe?$AAD?$AAl?$AAg?$AA?3?$AA?3?$AAS?$AAH?$AAC?$AAr?$AAe?$AAa?$AAt?$AAe?$AAM?$AAe?$AAn?$AAu?$AAB?$AAa?$AAr?$AA?5@ 0002e1c8     advanceddlg.obj
 0002:00000218       ??_C@_1EM@JMHHHJAO@?$AAI?$AAn?$AAi?$AAt?$AAA?$AAd?$AAv?$AAa?$AAn?$AAc?$AAe?$AAD?$AAl?$AAg?$AA?3?$AAS?$AAH?$AAC?$AAr?$AAe?$AAa?$AAt?$AAe?$AAM?$AAe?$AAn?$AAu?$AAB?$AAa?$AAr?$AA?5?$AAF@ 0002e218     advanceddlg.obj
 0002:00000264       ??_C@_1CM@PIPCPPPO@?$AAI?$AAn?$AAi?$AAt?$AAA?$AAd?$AAv?$AAa?$AAn?$AAc?$AAe?$AAD?$AAl?$AAg?$AA?5?$AAF?$AAa?$AAi?$AAl?$AAe?$AAd?$AA?$AA@ 0002e264     advanceddlg.obj
 0002:00000290       ??_C@_1FM@FLCBKLCK@?$AAC?$AAr?$AAe?$AAa?$AAt?$AAe?$AAA?$AAd?$AAv?$AAa?$AAn?$AAc?$AAe?$AAD?$AAl?$AAg?$AA?3?$AA?3?$AAF?$AAa?$AAl?$AAi?$AAe?$AAd?$AA?5?$AAt?$AAo?$AA?5?$AAC?$AAr?$AAe?$AAa@ 0002e290     advanceddlg.obj
 0002:000002f0       ??_C@_1FM@NFOLCLOA@?$AAC?$AAr?$AAe?$AAa?$AAt?$AAe?$AAA?$AAd?$AAv?$AAa?$AAn?$AAc?$AAe?$AAD?$AAl?$AAg?$AA?3?$AA?3?$AAF?$AAa?$AAl?$AAi?$AAe?$AAd?$AA?5?$AAt?$AAo?$AA?5?$AAR?$AAe?$AAg?$AAi@ 0002e2f0     advanceddlg.obj
 0002:0000034c       ??_C@_1CG@POBHOMMK@?$AAR?$AAI?$AAL?$AA_?$AAS?$AAT?$AAA?$AAT?$AAU?$AAS?$AA_?$AAC?$AAH?$AAA?$AAN?$AAG?$AAE?$AAD?$AA?$AA@ 0002e34c     advanceddlg.obj
 0002:00000374       ??_C@_1BK@BNOOAAEF@?$AAA?$AAu?$AAt?$AAh?$AAK?$AAe?$AAy?$AAC?$AAl?$AAa?$AAs?$AAs?$AA?$AA@ 0002e374     authkey.obj
 0002:00000390       ??_C@_1BM@GFMJDEAE@?$AA?4?$AA?2?$AAa?$AAu?$AAt?$AAh?$AAk?$AAe?$AAy?$AA?4?$AAc?$AAp?$AAp?$AA?$AA@ 0002e390     authkey.obj
 0002:000003ac       ??_C@_1DA@JAOFIDMD@?$AAP?$AAo?$AAw?$AAe?$AAr?$AA?5?$AAi?$AAs?$AA?5?$AAn?$AAo?$AAt?$AA?5?$AAo?$AAf?$AAf?$AAl?$AAi?$AAn?$AAe?$AA?5?$AA?$CF?$AAd?$AA?$AA@ 0002e3ac     authkey.obj
 0002:000003e0       ??_C@_1EI@NIIOLEGA@?$AAI?$AAn?$AAi?$AAt?$AAA?$AAu?$AAt?$AAh?$AAK?$AAe?$AAy?$AAD?$AAl?$AAg?$AA?3?$AA?3?$AAS?$AAH?$AAI?$AAn?$AAi?$AAt?$AAD?$AAi?$AAa?$AAl?$AAo?$AAg?$AA?5?$AAF?$AAa?$AAl@ 0002e3e0     authkey.obj
 0002:00000428       ??_C@_1EG@CJCOBILJ@?$AAI?$AAn?$AAi?$AAt?$AAA?$AAu?$AAt?$AAh?$AAK?$AAe?$AAy?$AAD?$AAl?$AAg?$AA?3?$AAS?$AAH?$AAI?$AAn?$AAi?$AAt?$AAD?$AAi?$AAa?$AAl?$AAo?$AAg?$AA?5?$AAF?$AAa?$AAi?$AAl@ 0002e428     authkey.obj
 0002:00000470       ??_C@_1EO@OGBFCBEL@?$AAI?$AAn?$AAi?$AAt?$AAA?$AAu?$AAt?$AAh?$AAK?$AAe?$AAy?$AAD?$AAl?$AAg?$AA?3?$AA?3?$AAS?$AAH?$AAC?$AAr?$AAe?$AAa?$AAt?$AAe?$AAM?$AAe?$AAn?$AAu?$AAB?$AAa?$AAr?$AA?5@ 0002e470     authkey.obj
 0002:000004c0       ??_C@_1EM@MPKNGIIC@?$AAI?$AAn?$AAi?$AAt?$AAA?$AAu?$AAt?$AAh?$AAK?$AAe?$AAy?$AAD?$AAl?$AAg?$AA?3?$AAS?$AAH?$AAC?$AAr?$AAe?$AAa?$AAt?$AAe?$AAM?$AAe?$AAn?$AAu?$AAB?$AAa?$AAr?$AA?5?$AAF@ 0002e4c0     authkey.obj
 0002:0000050c       ??_C@_1CM@PHGONND@?$AAI?$AAn?$AAi?$AAt?$AAA?$AAu?$AAt?$AAh?$AAK?$AAe?$AAy?$AAD?$AAl?$AAg?$AA?5?$AAF?$AAa?$AAi?$AAl?$AAe?$AAd?$AA?$AA@ 0002e50c     authkey.obj
 0002:00000538       ??_C@_1FM@FCHIPAHD@?$AAC?$AAr?$AAe?$AAa?$AAt?$AAe?$AAA?$AAu?$AAt?$AAh?$AAK?$AAe?$AAy?$AAD?$AAl?$AAg?$AA?3?$AA?3?$AAF?$AAa?$AAl?$AAi?$AAe?$AAd?$AA?5?$AAt?$AAo?$AA?5?$AAC?$AAr?$AAe?$AAa@ 0002e538     authkey.obj
 0002:00000598       ??_C@_1FM@NMLCHALJ@?$AAC?$AAr?$AAe?$AAa?$AAt?$AAe?$AAA?$AAu?$AAt?$AAh?$AAK?$AAe?$AAy?$AAD?$AAl?$AAg?$AA?3?$AA?3?$AAF?$AAa?$AAl?$AAi?$AAe?$AAd?$AA?5?$AAt?$AAo?$AA?5?$AAR?$AAe?$AAg?$AAi@ 0002e598     authkey.obj
 0002:000005f4       ??_C@_1BO@MBMFFGCA@?$AAP?$AAH?$AAO?$AAN?$AAE?$AAU?$AAT?$AAI?$AAL?$AAS?$AA_?$AAE?$AAN?$AAD?$AA?$AA@ 0002e5f4     authkey.obj
 0002:00000614       ??_C@_1CA@GALPFEIH@?$AAB?$AAr?$AAo?$AAw?$AAs?$AAe?$AAr?$AAD?$AAl?$AAg?$AAC?$AAl?$AAa?$AAs?$AAs?$AA?$AA@ 0002e614     browserdlg.obj
 0002:00000638       ??_C@_1EI@JCMPMONJ@?$AAI?$AAn?$AAi?$AAt?$AAB?$AAr?$AAo?$AAw?$AAs?$AAe?$AAr?$AAD?$AAl?$AAg?$AA?3?$AA?3?$AAS?$AAH?$AAI?$AAn?$AAi?$AAt?$AAD?$AAi?$AAa?$AAl?$AAo?$AAg?$AA?5?$AAF?$AAa?$AAl@ 0002e638     browserdlg.obj
 0002:00000680       ??_C@_1EG@JCEDNPLO@?$AAI?$AAn?$AAi?$AAt?$AAB?$AAr?$AAo?$AAw?$AAs?$AAe?$AAr?$AAD?$AAl?$AAg?$AA?3?$AAS?$AAH?$AAI?$AAn?$AAi?$AAt?$AAD?$AAi?$AAa?$AAl?$AAo?$AAg?$AA?5?$AAF?$AAa?$AAi?$AAl@ 0002e680     browserdlg.obj
 0002:000006c8       ??_C@_1EO@DGBHKMNG@?$AAI?$AAn?$AAi?$AAt?$AAB?$AAr?$AAo?$AAw?$AAs?$AAe?$AAr?$AAD?$AAl?$AAg?$AA?3?$AA?3?$AAS?$AAH?$AAC?$AAr?$AAe?$AAa?$AAt?$AAe?$AAM?$AAe?$AAn?$AAu?$AAB?$AAa?$AAr?$AA?5@ 0002e6c8     browserdlg.obj
 0002:00000718       ??_C@_1CC@NLINJCBG@?$AA?4?$AA?2?$AAb?$AAr?$AAo?$AAw?$AAs?$AAe?$AAr?$AAd?$AAl?$AAg?$AA?4?$AAc?$AAp?$AAp?$AA?$AA@ 0002e718     browserdlg.obj
 0002:00000740       ??_C@_1EM@IJNKFCNO@?$AAI?$AAn?$AAi?$AAt?$AAB?$AAr?$AAo?$AAw?$AAs?$AAe?$AAr?$AAD?$AAl?$AAg?$AA?3?$AAS?$AAH?$AAC?$AAr?$AAe?$AAa?$AAt?$AAe?$AAM?$AAe?$AAn?$AAu?$AAB?$AAa?$AAr?$AA?5?$AAF@ 0002e740     browserdlg.obj
 0002:0000078c       ??_C@_1CM@PEKPPHJI@?$AAI?$AAn?$AAi?$AAt?$AAB?$AAr?$AAo?$AAw?$AAs?$AAe?$AAr?$AAD?$AAl?$AAg?$AA?5?$AAF?$AAa?$AAi?$AAl?$AAe?$AAd?$AA?$AA@ 0002e78c     browserdlg.obj
 0002:000007b8       ??_C@_1FM@BINBBAAK@?$AAC?$AAr?$AAe?$AAa?$AAt?$AAe?$AAB?$AAr?$AAo?$AAw?$AAs?$AAe?$AAr?$AAD?$AAl?$AAg?$AA?3?$AA?3?$AAF?$AAa?$AAl?$AAi?$AAe?$AAd?$AA?5?$AAt?$AAo?$AA?5?$AAC?$AAr?$AAe?$AAa@ 0002e7b8     browserdlg.obj
 0002:00000818       ??_C@_1FM@JGBLJAMA@?$AAC?$AAr?$AAe?$AAa?$AAt?$AAe?$AAB?$AAr?$AAo?$AAw?$AAs?$AAe?$AAr?$AAD?$AAl?$AAg?$AA?3?$AA?3?$AAF?$AAa?$AAl?$AAi?$AAe?$AAd?$AA?5?$AAt?$AAo?$AA?5?$AAR?$AAe?$AAg?$AAi@ 0002e818     browserdlg.obj
 0002:00000874       ??_C@_1M@HNLFDEOA@?$AA3?$AA?4?$AA1?$AAM?$AAB?$AA?$AA@ 0002e874     bwmeterdlg.obj
 0002:00000880       ??_C@_1M@KOPAHGOL@?$AA2?$AA?4?$AA4?$AAM?$AAB?$AA?$AA@ 0002e880     bwmeterdlg.obj
 0002:0000088c       ??_C@_1M@IOMBLBFE@?$AA1?$AA?4?$AA8?$AAM?$AAB?$AA?$AA@ 0002e88c     bwmeterdlg.obj
 0002:00000898       ??_C@_1M@MJLMCIDG@?$AA3?$AA8?$AA4?$AAK?$AAB?$AA?$AA@ 0002e898     bwmeterdlg.obj
 0002:000008a4       ??_C@_1M@NKLMDEAA@?$AA1?$AA5?$AA3?$AAK?$AAB?$AA?$AA@ 0002e8a4     bwmeterdlg.obj
 0002:000008b0       ??_C@_1CA@PHFADNFB@?$AAB?$AAW?$AAM?$AAe?$AAt?$AAe?$AAr?$AAD?$AAl?$AAg?$AAC?$AAl?$AAa?$AAs?$AAs?$AA?$AA@ 0002e8b0     bwmeterdlg.obj
 0002:000008d0       ??_C@_13COJANIEC@?$AA0?$AA?$AA@ 0002e8d0     bwmeterdlg.obj
 0002:000008d4       ??_C@_17PEDLNONE@?$AA?$CF?$AAd?$AAK?$AA?$AA@ 0002e8d4     bwmeterdlg.obj
 0002:000008dc       ??_C@_1CC@KCMFNGC@?$AA?4?$AA?2?$AAb?$AAw?$AAm?$AAe?$AAt?$AAe?$AAr?$AAd?$AAl?$AAg?$AA?4?$AAc?$AAp?$AAp?$AA?$AA@ 0002e8dc     bwmeterdlg.obj
 0002:00000900       ??_C@_1DE@LAFIAKEF@?$AAO?$AAn?$AAT?$AAi?$AAm?$AAe?$AAr?$AA?$CI?$AAC?$AAA?$AAL?$AAL?$AA_?$AAC?$AAH?$AAE?$AAC?$AAK?$AA_?$AAT?$AAI?$AAM?$AAE?$AAR?$AA?$CJ?$AA?$AA@ 0002e900     bwmeterdlg.obj
 0002:00000934       ??_C@_1BK@DLBMHDEB@?$AAI?$AAn?$AAf?$AAo?$AAr?$AAm?$AAa?$AAt?$AAi?$AAo?$AAn?$AA?$CB?$AA?$AA@ 0002e934     bwmeterdlg.obj
 0002:00000950       ??_C@_1DA@JACAAPAO@?$AAP?$AAl?$AAe?$AAa?$AAs?$AAe?$AA?5?$AAs?$AAe?$AAl?$AAe?$AAc?$AAt?$AA?5?$AAM?$AAa?$AAx?$AA?5?$AAS?$AAp?$AAe?$AAe?$AAd?$AA?$AA@ 0002e950     bwmeterdlg.obj
 0002:00000980       ??_C@_1FC@CKJKLCGN@?$AAI?$AAn?$AAi?$AAt?$AAB?$AAW?$AAM?$AAe?$AAt?$AAe?$AAr?$AAD?$AAl?$AAg?$AAC?$AAl?$AAa?$AAs?$AAs?$AA?3?$AA?3?$AAS?$AAH?$AAI?$AAn?$AAi?$AAt?$AAD?$AAi?$AAa?$AAl?$AAo@ 0002e980     bwmeterdlg.obj
 0002:000009d8       ??_C@_1FA@PDCMNLPJ@?$AAI?$AAn?$AAi?$AAt?$AAB?$AAW?$AAM?$AAe?$AAt?$AAe?$AAr?$AAD?$AAl?$AAg?$AAC?$AAl?$AAa?$AAs?$AAs?$AA?3?$AAS?$AAH?$AAI?$AAn?$AAi?$AAt?$AAD?$AAi?$AAa?$AAl?$AAo?$AAg@ 0002e9d8     bwmeterdlg.obj
 0002:00000a28       ??_C@_1FI@LMPAKAED@?$AAI?$AAn?$AAi?$AAt?$AAB?$AAW?$AAM?$AAe?$AAt?$AAe?$AAr?$AAD?$AAl?$AAg?$AAC?$AAl?$AAa?$AAs?$AAs?$AA?3?$AA?3?$AAS?$AAH?$AAC?$AAr?$AAe?$AAa?$AAt?$AAe?$AAM?$AAe?$AAn@ 0002ea28     bwmeterdlg.obj
 0002:00000a80       ??_C@_1FG@EEFHIIII@?$AAI?$AAn?$AAi?$AAt?$AAB?$AAW?$AAM?$AAe?$AAt?$AAe?$AAr?$AAD?$AAl?$AAg?$AAC?$AAl?$AAa?$AAs?$AAs?$AA?3?$AAS?$AAH?$AAC?$AAr?$AAe?$AAa?$AAt?$AAe?$AAM?$AAe?$AAn?$AAu@ 0002ea80     bwmeterdlg.obj
 0002:00000ad8       ??_C@_1DG@HCOAFOFC@?$AAI?$AAn?$AAi?$AAt?$AAB?$AAW?$AAM?$AAe?$AAt?$AAe?$AAr?$AAD?$AAl?$AAg?$AAC?$AAl?$AAa?$AAs?$AAs?$AA?5?$AAF?$AAa?$AAi?$AAl?$AAe?$AAd?$AA?$AA@ 0002ead8     bwmeterdlg.obj
 0002:00000b10       ??_C@_1FO@NIKICLPN@?$AAC?$AAr?$AAe?$AAa?$AAt?$AAe?$AAS?$AAi?$AAm?$AAp?$AAl?$AAe?$AAI?$AAP?$AAD?$AAl?$AAg?$AA?3?$AA?3?$AAF?$AAa?$AAl?$AAi?$AAe?$AAd?$AA?5?$AAt?$AAo?$AA?5?$AAC?$AAr?$AAe@ 0002eb10     bwmeterdlg.obj
 0002:00000b70       ??_C@_1BO@DIMFLEAM@?$AAC?$AAo?$AAn?$AAf?$AAi?$AAg?$AAD?$AAl?$AAg?$AAC?$AAl?$AAa?$AAs?$AAs?$AA?$AA@ 0002eb70     configdlg.obj
 0002:00000b90       ??_C@_1BI@LCELGAKO@?$AAT?$AAe?$AAc?$AAh?$AAn?$AAo?$AAl?$AAo?$AAg?$AAy?$AA?3?$AA?$AA@ 0002eb90     configdlg.obj
 0002:00000ba8       ??_C@_1M@IHPKHBBM@?$AAQ?$AAL?$AAI?$AAC?$AA?3?$AA?$AA@ 0002eba8     configdlg.obj
 0002:00000bb4       ??_C@_1BK@IDIJPNBP@?$AAP?$AAR?$AAL?$AA?5?$AAV?$AAe?$AAr?$AAs?$AAi?$AAo?$AAn?$AA?3?$AA?$AA@ 0002ebb4     configdlg.obj
 0002:00000bd0       ??_C@_1BC@OCMLJLD@?$AAC?$AAh?$AAi?$AAp?$AAs?$AAe?$AAt?$AA?3?$AA?$AA@ 0002ebd0     configdlg.obj
 0002:00000be4       ??_C@_1BM@GGFPPDC@?$AAA?$AAM?$AAS?$AAS?$AA?5?$AAV?$AAe?$AAr?$AAs?$AAi?$AAo?$AAn?$AA?3?$AA?$AA@ 0002ebe4     configdlg.obj
 0002:00000c00       ??_C@_1CA@PBIGDJJE@?$AAD?$AAe?$AAv?$AAi?$AAc?$AAe?$AA?5?$AAV?$AAe?$AAr?$AAs?$AAi?$AAo?$AAn?$AA?3?$AA?$AA@ 0002ec00     configdlg.obj
 0002:00000c20       ??_C@_1CE@MAFNGDHL@?$AAH?$AAa?$AAr?$AAd?$AAw?$AAa?$AAr?$AAe?$AA?5?$AAV?$AAe?$AAr?$AAs?$AAi?$AAo?$AAn?$AA?3?$AA?$AA@ 0002ec20     configdlg.obj
 0002:00000c44       ??_C@_15GANGMFKL@?$AA?$CF?$AAs?$AA?$AA@ 0002ec44     configdlg.obj
 0002:00000c50       ??_C@_1EG@PJBMJF@?$AAI?$AAn?$AAi?$AAt?$AAC?$AAo?$AAn?$AAf?$AAi?$AAg?$AAD?$AAl?$AAg?$AA?3?$AA?3?$AAS?$AAH?$AAI?$AAn?$AAi?$AAt?$AAD?$AAi?$AAa?$AAl?$AAo?$AAg?$AA?5?$AAF?$AAa?$AAl?$AAi@ 0002ec50     configdlg.obj
 0002:00000c98       ??_C@_1EE@MAFLBIDC@?$AAI?$AAn?$AAi?$AAt?$AAC?$AAo?$AAn?$AAf?$AAi?$AAg?$AAD?$AAl?$AAg?$AA?3?$AAS?$AAH?$AAI?$AAn?$AAi?$AAt?$AAD?$AAi?$AAa?$AAl?$AAo?$AAg?$AA?5?$AAF?$AAa?$AAi?$AAl?$AAe@ 0002ec98     configdlg.obj
 0002:00000ce0       ??_C@_1EM@JGGPIBBL@?$AAI?$AAn?$AAi?$AAt?$AAC?$AAo?$AAn?$AAf?$AAi?$AAg?$AAD?$AAl?$AAg?$AA?3?$AA?3?$AAS?$AAH?$AAC?$AAr?$AAe?$AAa?$AAt?$AAe?$AAM?$AAe?$AAn?$AAu?$AAB?$AAa?$AAr?$AA?5?$AAF@ 0002ece0     configdlg.obj
 0002:00000d2c       ??_C@_1CA@GLAHFDND@?$AA?4?$AA?2?$AAc?$AAo?$AAn?$AAf?$AAi?$AAg?$AAd?$AAl?$AAg?$AA?4?$AAc?$AAp?$AAp?$AA?$AA@ 0002ed2c     configdlg.obj
 0002:00000d50       ??_C@_1EK@EBAIDHBI@?$AAI?$AAn?$AAi?$AAt?$AAC?$AAo?$AAn?$AAf?$AAi?$AAg?$AAD?$AAl?$AAg?$AA?3?$AAS?$AAH?$AAC?$AAr?$AAe?$AAa?$AAt?$AAe?$AAM?$AAe?$AAn?$AAu?$AAB?$AAa?$AAr?$AA?5?$AAF?$AAa@ 0002ed50     configdlg.obj
 0002:00000d9c       ??_C@_1CK@JLLAMLIM@?$AAI?$AAn?$AAi?$AAt?$AAC?$AAo?$AAn?$AAf?$AAi?$AAg?$AAD?$AAl?$AAg?$AA?5?$AAF?$AAa?$AAi?$AAl?$AAe?$AAd?$AA?$AA@ 0002ed9c     configdlg.obj
 0002:00000dc8       ??_C@_1FK@IJODJBBM@?$AAC?$AAr?$AAe?$AAa?$AAt?$AAe?$AAC?$AAo?$AAn?$AAf?$AAi?$AAg?$AAD?$AAl?$AAg?$AA?3?$AA?3?$AAF?$AAa?$AAl?$AAi?$AAe?$AAd?$AA?5?$AAt?$AAo?$AA?5?$AAC?$AAr?$AAe?$AAa?$AAt@ 0002edc8     configdlg.obj
 0002:00000e28       ??_C@_1FK@HCJBBNG@?$AAC?$AAr?$AAe?$AAa?$AAt?$AAe?$AAC?$AAo?$AAn?$AAf?$AAi?$AAg?$AAD?$AAl?$AAg?$AA?3?$AA?3?$AAF?$AAa?$AAl?$AAi?$AAe?$AAd?$AA?5?$AAt?$AAo?$AA?5?$AAR?$AAe?$AAg?$AAi?$AAs@ 0002ee28     configdlg.obj
 0002:00000e84       ??_C@_1BC@PCHKAMBP@?$AAP?$AAO?$AAW?$AAE?$AAR?$AA_?$AAO?$AAN?$AA?$AA@ 0002ee84     configdlg.obj
 0002:00000e98       ??_C@_1BE@JGMADFED@?$AAP?$AAO?$AAW?$AAE?$AAR?$AA_?$AAO?$AAF?$AAF?$AA?$AA@ 0002ee98     configdlg.obj
 0002:00000eac       ??_C@_1BG@MAJEEGIE@?$AAI?$AAO?$AAT?$AAA?$AA_?$AAB?$AAE?$AAG?$AAI?$AAN?$AA?$AA@ 0002eeac     configdlg.obj
 0002:00000ec4       ??_C@_1BC@OHNJMDNM@?$AAI?$AAO?$AAT?$AAA?$AA_?$AAE?$AAN?$AAD?$AA?$AA@ 0002eec4     configdlg.obj
 0002:00000ed8       ??_C@_1BO@OOLLGKIG@?$AAI?$AAT?$AAO?$AAA?$AA_?$AAB?$AAE?$AAG?$AAI?$AAN?$AA_?$AAA?$AAC?$AAK?$AA?$AA@ 0002eed8     configdlg.obj
 0002:00000ef8       ??_C@_1CA@NDNGFIJB@?$AAI?$AAT?$AAO?$AAA?$AA_?$AAB?$AAE?$AAG?$AAI?$AAN?$AA_?$AAN?$AAA?$AAC?$AAK?$AA?$AA@ 0002eef8     configdlg.obj
 0002:00000f18       ??_C@_1BK@LHMHCDIP@?$AAI?$AAT?$AAO?$AAA?$AA_?$AAE?$AAN?$AAD?$AA_?$AAA?$AAC?$AAK?$AA?$AA@ 0002ef18     configdlg.obj
 0002:00000f34       ??_C@_1BE@CENHHBC@?$AAI?$AAT?$AAO?$AAA?$AA_?$AAE?$AAX?$AAI?$AAT?$AA?$AA@ 0002ef34     configdlg.obj
 0002:00000f48       ??_C@_1CG@NGJLINHO@?$AAI?$AAO?$AAT?$AAA?$AA_?$AAA?$AAL?$AAI?$AAV?$AAE?$AA_?$AAM?$AAE?$AAS?$AAS?$AAA?$AAG?$AAE?$AA?$AA@ 0002ef48     configdlg.obj
 0002:00000f70       ??_C@_1CE@JLPOCCBE@?$AAI?$AAO?$AAT?$AAA?$AA_?$AAP?$AAI?$AAN?$AAG?$AA_?$AAM?$AAE?$AAS?$AAS?$AAA?$AAG?$AAE?$AA?$AA@ 0002ef70     configdlg.obj
 0002:00000f94       ??_C@_1BM@NCKPFMMC@?$AAI?$AAO?$AAT?$AAA?$AA_?$AAP?$AAI?$AAN?$AAG?$AA_?$AAA?$AAC?$AAK?$AA?$AA@ 0002ef94     configdlg.obj
 0002:00000fb0       ??_C@_1CI@HGBOCMNH@?$AAI?$AAO?$AAT?$AAA?$AA_?$AAC?$AAR?$AAI?$AAT?$AAI?$AAC?$AAA?$AAL?$AA_?$AAE?$AAR?$AAR?$AAO?$AAR?$AA?$AA@ 0002efb0     configdlg.obj
 0002:00000fd8       ??_C@_1DA@BHPKMPLG@?$AAI?$AAO?$AAT?$AAA?$AA_?$AAN?$AAO?$AAN?$AA_?$AAC?$AAR?$AAI?$AAT?$AAI?$AAC?$AAA?$AAL?$AA_?$AAE?$AAR?$AAR?$AAO?$AAR?$AA?$AA@ 0002efd8     configdlg.obj
 0002:00001008       ??_C@_1CC@MLMAKKOO@?$AAK?$AAI?$AAL?$AAL?$AA_?$AAI?$AAO?$AAT?$AAA?$AA_?$AAP?$AAL?$AAE?$AAA?$AAS?$AAE?$AA?$AA@ 0002f008     configdlg.obj
 0002:0000102c       ??_C@_1CG@PGHILCBC@?$AAI?$AAO?$AAT?$AAA?$AA_?$AAU?$AAP?$AAD?$AAA?$AAT?$AAE?$AA_?$AAS?$AAT?$AAA?$AAT?$AAU?$AAS?$AA?$AA@ 0002f02c     configdlg.obj
 0002:00001054       ??_C@_1CK@LDMADEEM@?$AAI?$AAO?$AAT?$AAA?$AA_?$AAD?$AAa?$AAt?$AAa?$AA_?$AAP?$AAo?$AAr?$AAt?$AA_?$AAI?$AAn?$AAU?$AAs?$AAe?$AA?$AA@ 0002f054     configdlg.obj
 0002:00001080       ??_C@_1CO@GLHJIBOI@?$AAI?$AAO?$AAT?$AAA?$AA_?$AAP?$AAR?$AAO?$AAV?$AAI?$AAS?$AAI?$AAO?$AAN?$AAI?$AAN?$AAG?$AA_?$AAD?$AAO?$AAN?$AAE?$AA?$AA@ 0002f080     configdlg.obj
 0002:000010b0       ??_C@_1BE@ELOIOKNB@?$AAI?$AAO?$AAT?$AAA?$AA_?$AAD?$AAI?$AAA?$AAL?$AA?$AA@ 0002f0b0     configdlg.obj
 0002:000010c4       ??_C@_1BM@LJOIKJDC@?$AAI?$AAO?$AAT?$AAA?$AA_?$AA1?$AA0?$AA1?$AA2?$AA_?$AAE?$AAR?$AAR?$AA?$AA@ 0002f0c4     configdlg.obj
 0002:000010e0       ??_C@_1CC@MDIGENCA@?$AAP?$AAH?$AAO?$AAN?$AAE?$AAU?$AAT?$AAI?$AAL?$AAS?$AA_?$AAB?$AAE?$AAG?$AAI?$AAN?$AA?$AA@ 0002f0e0     configdlg.obj
 0002:00001104       ??_C@_1CK@NCAHKLGJ@?$AAP?$AAH?$AAO?$AAN?$AAE?$AAU?$AAT?$AAI?$AAL?$AAS?$AA_?$AAB?$AAE?$AAG?$AAI?$AAN?$AA_?$AAA?$AAC?$AAK?$AA?$AA@ 0002f104     configdlg.obj
 0002:00001130       ??_C@_1CM@OGFDHJCI@?$AAP?$AAH?$AAO?$AAN?$AAE?$AAU?$AAT?$AAI?$AAL?$AAS?$AA_?$AAB?$AAE?$AAG?$AAI?$AAN?$AA_?$AAN?$AAA?$AAC?$AAK?$AA?$AA@ 0002f130     configdlg.obj
 0002:0000115c       ??_C@_1CI@PIELHBKD@?$AAP?$AAH?$AAO?$AAN?$AAE?$AAU?$AAT?$AAI?$AAL?$AAS?$AA_?$AAE?$AAN?$AAD?$AA_?$AAN?$AAA?$AAC?$AAK?$AA?$AA@ 0002f15c     configdlg.obj
 0002:00001184       ??_C@_1CA@FFKJKCCB@?$AAP?$AAH?$AAO?$AAN?$AAE?$AAU?$AAT?$AAI?$AAL?$AAS?$AA_?$AAE?$AAX?$AAI?$AAT?$AA?$AA@ 0002f184     configdlg.obj
 0002:000011a4       ??_C@_1DC@KNIKGFIB@?$AAP?$AAH?$AAO?$AAN?$AAE?$AAU?$AAT?$AAI?$AAL?$AAS?$AA_?$AAA?$AAL?$AAI?$AAV?$AAE?$AA_?$AAM?$AAE?$AAS?$AAS?$AAA?$AAG?$AAE?$AA?$AA@ 0002f1a4     configdlg.obj
 0002:000011d8       ??_C@_1DA@FCENJAPE@?$AAP?$AAH?$AAO?$AAN?$AAE?$AAU?$AAT?$AAI?$AAL?$AAS?$AA_?$AAP?$AAI?$AAN?$AAG?$AA_?$AAM?$AAE?$AAS?$AAS?$AAA?$AAG?$AAE?$AA?$AA@ 0002f1d8     configdlg.obj
 0002:00001208       ??_C@_1CI@NPKEBPGG@?$AAP?$AAH?$AAO?$AAN?$AAE?$AAU?$AAT?$AAI?$AAL?$AAS?$AA_?$AAP?$AAI?$AAN?$AAG?$AA_?$AAA?$AAC?$AAK?$AA?$AA@ 0002f208     configdlg.obj
 0002:00001230       ??_C@_1BC@FNALODJM@?$AAA?$AAW?$AA_?$AAB?$AAE?$AAG?$AAI?$AAN?$AA?$AA@ 0002f230     configdlg.obj
 0002:00001244       ??_C@_1O@LCFHJGAG@?$AAA?$AAW?$AA_?$AAE?$AAN?$AAD?$AA?$AA@ 0002f244     configdlg.obj
 0002:00001254       ??_C@_1BK@IINCFOMF@?$AAA?$AAW?$AA_?$AAB?$AAE?$AAG?$AAI?$AAN?$AA_?$AAA?$AAC?$AAK?$AA?$AA@ 0002f254     configdlg.obj
 0002:00001270       ??_C@_1BM@CJDGNGIL@?$AAA?$AAW?$AA_?$AAB?$AAE?$AAG?$AAI?$AAN?$AA_?$AAN?$AAA?$AAC?$AAK?$AA?$AA@ 0002f270     configdlg.obj
 0002:0000128c       ??_C@_1BG@FJAKJBPC@?$AAA?$AAW?$AA_?$AAE?$AAN?$AAD?$AA_?$AAA?$AAC?$AAK?$AA?$AA@ 0002f28c     configdlg.obj
 0002:000012a4       ??_C@_1BA@NBDJACH@?$AAA?$AAW?$AA_?$AAE?$AAX?$AAI?$AAT?$AA?$AA@ 0002f2a4     configdlg.obj
 0002:000012b4       ??_C@_1CC@FGHONIMK@?$AAA?$AAW?$AA_?$AAA?$AAL?$AAI?$AAV?$AAE?$AA_?$AAM?$AAE?$AAS?$AAS?$AAA?$AAG?$AAE?$AA?$AA@ 0002f2b4     configdlg.obj
 0002:000012d8       ??_C@_1CA@MMOGHMIB@?$AAA?$AAW?$AA_?$AAP?$AAI?$AAN?$AAG?$AA_?$AAM?$AAE?$AAS?$AAS?$AAA?$AAG?$AAE?$AA?$AA@ 0002f2d8     configdlg.obj
 0002:000012f8       ??_C@_1BI@JFAFBGID@?$AAA?$AAW?$AA_?$AAP?$AAI?$AAN?$AAG?$AA_?$AAA?$AAC?$AAK?$AA?$AA@ 0002f2f8     configdlg.obj
 0002:00001310       ??_C@_1BM@NNDEDBAN@?$AAU?$AAP?$AAD?$AAA?$AAT?$AAE?$AAR?$AA_?$AAB?$AAE?$AAG?$AAI?$AAN?$AA?$AA@ 0002f310     configdlg.obj
 0002:0000132c       ??_C@_1BI@KBKNMDLB@?$AAU?$AAP?$AAD?$AAA?$AAT?$AAE?$AAR?$AA_?$AAE?$AAN?$AAD?$AA?$AA@ 0002f32c     configdlg.obj
 0002:00001344       ??_C@_1CE@BDGOPNCM@?$AAU?$AAP?$AAD?$AAA?$AAT?$AAE?$AAR?$AA_?$AAB?$AAE?$AAG?$AAI?$AAN?$AA_?$AAA?$AAC?$AAK?$AA?$AA@ 0002f344     configdlg.obj
 0002:00001368       ??_C@_1CG@OJFFPHMA@?$AAU?$AAP?$AAD?$AAA?$AAT?$AAE?$AAR?$AA_?$AAB?$AAE?$AAG?$AAI?$AAN?$AA_?$AAN?$AAA?$AAC?$AAK?$AA?$AA@ 0002f368     configdlg.obj
 0002:00001390       ??_C@_1CA@GHJNFPHB@?$AAU?$AAP?$AAD?$AAA?$AAT?$AAE?$AAR?$AA_?$AAE?$AAN?$AAD?$AA_?$AAA?$AAC?$AAK?$AA?$AA@ 0002f390     configdlg.obj
 0002:000013b0       ??_C@_1CC@NOJIGCOO@?$AAU?$AAP?$AAD?$AAA?$AAT?$AAE?$AAR?$AA_?$AAE?$AAN?$AAD?$AA_?$AAN?$AAA?$AAC?$AAK?$AA?$AA@ 0002f3b0     configdlg.obj
 0002:000013d4       ??_C@_1BO@NKICKCPO@?$AAR?$AAI?$AAL?$AA_?$AAD?$AAB?$AAG?$AA_?$AAN?$AAO?$AAT?$AAI?$AAF?$AAY?$AA?$AA@ 0002f3d4     configdlg.obj
 0002:000013f4       ??_C@_1CG@HIPGCNFB@?$AAR?$AAI?$AAL?$AA_?$AAT?$AAE?$AAC?$AAH?$AAH?$AAD?$AAR?$AA_?$AAN?$AAO?$AAT?$AAI?$AAF?$AAY?$AA?$AA@ 0002f3f4     configdlg.obj
 0002:0000141c       ??_C@_1DA@MPHILDIE@?$AAR?$AAI?$AAL?$AA_?$AAI?$AAO?$AAT?$AAA?$AA_?$AAS?$AAT?$AAA?$AAT?$AAU?$AAS?$AA_?$AAC?$AAH?$AAA?$AAN?$AAG?$AAE?$AAD?$AA?$AA@ 0002f41c     configdlg.obj
 0002:0000144c       ??_C@_1CC@BEOCDLIL@?$AAR?$AAI?$AAL?$AA_?$AAI?$AAO?$AAT?$AAA?$AA_?$AAW?$AAA?$AAP?$AA_?$AAU?$AAR?$AAI?$AA?$AA@ 0002f44c     configdlg.obj
 0002:00001470       ??_C@_1CC@POEPKLA@?$AAR?$AAI?$AAL?$AA_?$AAP?$AAD?$AAS?$AAM?$AA_?$AAP?$AAD?$AA_?$AAD?$AAA?$AAT?$AAA?$AA?$AA@ 0002f470     configdlg.obj
 0002:00001494       ??_C@_1CC@DHEBFOCI@?$AAR?$AAI?$AAL?$AA_?$AAP?$AAD?$AAS?$AAM?$AA_?$AAP?$AAD?$AA_?$AAD?$AAO?$AAN?$AAE?$AA?$AA@ 0002f494     configdlg.obj
 0002:000014b8       ??_C@_1CA@IJMMNJBM@?$AAR?$AAI?$AAL?$AA_?$AAP?$AAD?$AAS?$AAM?$AA_?$AAP?$AAD?$AA_?$AAE?$AAN?$AAD?$AA?$AA@ 0002f4b8     configdlg.obj
 0002:000014d8       ??_C@_1CE@DKNHCEGP@?$AAR?$AAI?$AAL?$AA_?$AAP?$AAD?$AAS?$AAM?$AA_?$AAP?$AAD?$AA_?$AAB?$AAE?$AAG?$AAI?$AAN?$AA?$AA@ 0002f4d8     configdlg.obj
 0002:000014fc       ??_C@_1DG@ENNLKGLF@?$AAR?$AAI?$AAL?$AA_?$AAP?$AAD?$AAS?$AAM?$AA_?$AAP?$AAD?$AA_?$AAU?$AAP?$AAD?$AAA?$AAT?$AAE?$AA_?$AAF?$AAA?$AAI?$AAL?$AAU?$AAR?$AAE?$AA?$AA@ 0002f4fc     configdlg.obj
 0002:00001534       ??_C@_1CK@FFHNCNLC@?$AAR?$AAI?$AAL?$AA_?$AAP?$AAD?$AAS?$AAM?$AA_?$AAP?$AAD?$AA_?$AAD?$AAL?$AAD?$AA_?$AAD?$AAA?$AAT?$AAA?$AA?$AA@ 0002f534     configdlg.obj
 0002:00001560       ??_C@_1CK@GNNIIJCK@?$AAR?$AAI?$AAL?$AA_?$AAP?$AAD?$AAS?$AAM?$AA_?$AAP?$AAD?$AA_?$AAD?$AAL?$AAD?$AA_?$AAD?$AAO?$AAN?$AAE?$AA?$AA@ 0002f560     configdlg.obj
 0002:0000158c       ??_C@_1CI@IINDIONI@?$AAR?$AAI?$AAL?$AA_?$AAP?$AAD?$AAS?$AAM?$AA_?$AAP?$AAD?$AA_?$AAD?$AAL?$AAD?$AA_?$AAE?$AAN?$AAD?$AA?$AA@ 0002f58c     configdlg.obj
 0002:000015b4       ??_C@_1CM@BAFGFLAD@?$AAR?$AAI?$AAL?$AA_?$AAP?$AAD?$AAS?$AAM?$AA_?$AAP?$AAD?$AA_?$AAD?$AAL?$AAD?$AA_?$AAB?$AAE?$AAG?$AAI?$AAN?$AA?$AA@ 0002f5b4     configdlg.obj
 0002:000015e0       ??_C@_1CE@GDPLDIKM@?$AAR?$AAI?$AAL?$AA_?$AAP?$AAD?$AAS?$AAM?$AA_?$AAP?$AAA?$AA_?$AAP?$AAA?$AAR?$AAA?$AAM?$AA?$AA@ 0002f5e0     configdlg.obj
 0002:00001604       ??_C@_1CE@ILHCKNGC@?$AAR?$AAI?$AAL?$AA_?$AAC?$AAA?$AAL?$AAL?$AA_?$AAB?$AAY?$AAT?$AAE?$AA_?$AAC?$AAT?$AAR?$AA?$AA@ 0002f604     configdlg.obj
 0002:00001628       ??_C@_1CK@HOBLCGKE@?$AAR?$AAI?$AAL?$AA_?$AAC?$AAR?$AAE?$AAA?$AAT?$AAE?$AA_?$AAM?$AAA?$AAI?$AAN?$AA_?$AAL?$AAI?$AAS?$AAT?$AA?$AA@ 0002f628     configdlg.obj
 0002:00001654       ??_C@_1BK@MNEPCMIJ@?$AAE?$AAV?$AAD?$AAO?$AAD?$AAl?$AAg?$AAC?$AAl?$AAa?$AAs?$AAs?$AA?$AA@ 0002f654     evdo.obj
 0002:000016cc       ??_C@_1BA@HAKGIOGJ@?$AA?$CF?$AA?4?$AA1?$AAf?$AA?5?$AAd?$AAB?$AA?$AA@ 0002f6cc     evdo.obj
 0002:000016dc       ??_C@_1BO@IJPGNJJP@?$AA0?$AAx?$AA?$CF?$AAX?$AA?0?$AA0?$AAx?$AA?$CF?$AAX?$AA?0?$AA0?$AAx?$AA?$CF?$AAX?$AA?$AA@ 0002f6dc     evdo.obj
 0002:00001700       ??_C@_1GA@CNCGJEKP@?$AA?$CF?$AAd?$AA?0?$AA?$CF?$AAd?$AA?0?$AA?$CF?$AAd?$AA?0?$AA?$CF?$AAd?$AA?0?$AA?$CF?$AAd?$AA?0?$AA?$CF?$AAd?$AA?0?$AA?$CF?$AAd?$AA?0?$AA?$CF?$AAd?$AA?0?$AA?$CF?$AAd?$AA?0?$AA?$CF?$AAd?$AA?0?$AA?$CF?$AAd@ 0002f700     evdo.obj
 0002:00001760       ??_C@_15EFLNJKHH@?$AA?$CF?$AAu?$AA?$AA@ 0002f760     evdo.obj
 0002:00001768       ??_C@_1BG@EEGEGLGC@?$AAP?$AAI?$AAL?$AAO?$AAT?$AA?5?$AAO?$AAN?$AAL?$AAY?$AA?$AA@ 0002f768     evdo.obj
 0002:00001780       ??_C@_1M@HCOAAOHB@?$AA9?$AAK?$AAB?$AAp?$AAs?$AA?$AA@ 0002f780     evdo.obj
 0002:0000178c       ??_C@_1O@OOFHBEBL@?$AA1?$AA9?$AAK?$AAB?$AAp?$AAs?$AA?$AA@ 0002f78c     evdo.obj
 0002:0000179c       ??_C@_1O@JEJMJMNJ@?$AA3?$AA8?$AAK?$AAB?$AAp?$AAs?$AA?$AA@ 0002f79c     evdo.obj
 0002:000017ac       ??_C@_1O@GEABMANM@?$AA7?$AA6?$AAK?$AAB?$AAp?$AAs?$AA?$AA@ 0002f7ac     evdo.obj
 0002:000017bc       ??_C@_1BA@HPLMJFIB@?$AA1?$AA5?$AA3?$AAK?$AAB?$AAp?$AAs?$AA?$AA@ 0002f7bc     evdo.obj
 0002:000017cc       ??_C@_1CM@FOIEHNEO@?$AAA?$AAU?$AAT?$AAH?$AAE?$AAN?$AAT?$AAI?$AAC?$AAA?$AAT?$AAI?$AAO?$AAN?$AA_?$AAF?$AAA?$AAI?$AAL?$AAE?$AAD?$AA?$AA@ 0002f7cc     evdo.obj
 0002:000017f8       ??_C@_1BM@BBKHBOOM@?$AAA?$AAU?$AAT?$AAH?$AAE?$AAN?$AAT?$AAI?$AAC?$AAA?$AAT?$AAE?$AAD?$AA?$AA@ 0002f7f8     evdo.obj
 0002:00001814       ??_C@_1DE@FNIBCMHL@?$AAN?$AAO?$AA?5?$AAA?$AAU?$AAT?$AAH?$AAE?$AAN?$AAT?$AAI?$AAC?$AAA?$AAT?$AAI?$AAO?$AAN?$AA?5?$AAR?$AAE?$AAQ?$AAU?$AAE?$AAS?$AAT?$AA?$AA@ 0002f814     evdo.obj
 0002:00001848       ??_C@_1M@JBDMLJKJ@?$AAC?$AAL?$AAO?$AAS?$AAE?$AA?$AA@ 0002f848     evdo.obj
 0002:00001854       ??_C@_1DC@MEKEEKKH@?$AAA?$AAD?$AAD?$AAR?$AA_?$AAM?$AAG?$AAM?$AAT?$AA_?$AAP?$AAR?$AAO?$AAT?$AAO?$AAC?$AAO?$AAL?$AA_?$AAS?$AAE?$AAT?$AAU?$AAP?$AA?$AA@ 0002f854     evdo.obj
 0002:00001888       ??_C@_1BK@BJDNDBLH@?$AAA?$AAT?$AA_?$AAI?$AAN?$AAI?$AAT?$AAI?$AAA?$AAT?$AAE?$AAD?$AA?$AA@ 0002f888     evdo.obj
 0002:000018a4       ??_C@_1BK@GNGALODL@?$AAA?$AAN?$AA_?$AAI?$AAN?$AAI?$AAT?$AAI?$AAA?$AAT?$AAE?$AAD?$AA?$AA@ 0002f8a4     evdo.obj
 0002:000018c0       ??_C@_19CLMIMLD@?$AAO?$AAP?$AAE?$AAN?$AA?$AA@ 0002f8c0     evdo.obj
 0002:000018cc       ??_C@_1BC@LPONJHPI@?$AAI?$AAN?$AAA?$AAC?$AAT?$AAI?$AAV?$AAE?$AA?$AA@ 0002f8cc     evdo.obj
 0002:000018e0       ??_C@_1BI@MODBKKGA@?$AAA?$AAC?$AAQ?$AAU?$AAI?$AAS?$AAI?$AAT?$AAI?$AAO?$AAN?$AA?$AA@ 0002f8e0     evdo.obj
 0002:000018f8       ??_C@_19LIMMNOOA@?$AAS?$AAY?$AAN?$AAC?$AA?$AA@ 0002f8f8     evdo.obj
 0002:00001904       ??_C@_19HFNBFOM@?$AAI?$AAD?$AAL?$AAE?$AA?$AA@ 0002f904     evdo.obj
 0002:00001910       ??_C@_1O@PCFNFPIA@?$AAA?$AAC?$AAC?$AAE?$AAS?$AAS?$AA?$AA@ 0002f910     evdo.obj
 0002:00001920       ??_C@_1BE@OFJFCKEM@?$AAC?$AAO?$AAN?$AAN?$AAE?$AAC?$AAT?$AAE?$AAD?$AA?$AA@ 0002f920     evdo.obj
 0002:00001934       ??_C@_1BA@HABJOAEE@?$AAU?$AAN?$AAK?$AAN?$AAO?$AAW?$AAN?$AA?$AA@ 0002f934     evdo.obj
 0002:00001944       ??_C@_1BC@FFOLHNKK@?$AA?9?$AA?$CF?$AA?4?$AA1?$AAf?$AA?5?$AAd?$AAB?$AA?$AA@ 0002f944     evdo.obj
 0002:00001958       ??_C@_15FPHCHCFA@?$AA?$CF?$AAi?$AA?$AA@ 0002f958     evdo.obj
 0002:00001960       ??_C@_1BA@GBCNOEIK@?$AA?9?$AA?$CF?$AAi?$AA?5?$AAd?$AAB?$AAm?$AA?$AA@ 0002f960     evdo.obj
 0002:00001970       ??_C@_1CK@HLMAGLLN@?$AAE?$AAn?$AAa?$AAb?$AAl?$AAe?$AAT?$AAe?$AAc?$AAh?$AAH?$AAd?$AAr?$AA?5?$AAf?$AAa?$AAi?$AAl?$AAe?$AAd?$AA?$AA@ 0002f970     evdo.obj
 0002:000019a0       ??_C@_1EC@DFHGBIJK@?$AAI?$AAn?$AAi?$AAt?$AAE?$AAV?$AAD?$AAO?$AAD?$AAl?$AAg?$AA?3?$AA?3?$AAS?$AAH?$AAI?$AAn?$AAi?$AAt?$AAD?$AAi?$AAa?$AAl?$AAo?$AAg?$AA?5?$AAF?$AAa?$AAl?$AAi?$AAe?$AAd@ 0002f9a0     evdo.obj
 0002:000019e8       ??_C@_1EA@NJPPPOFD@?$AAI?$AAn?$AAi?$AAt?$AAE?$AAV?$AAD?$AAO?$AAD?$AAl?$AAg?$AA?3?$AAS?$AAH?$AAI?$AAn?$AAi?$AAt?$AAD?$AAi?$AAa?$AAl?$AAo?$AAg?$AA?5?$AAF?$AAa?$AAi?$AAl?$AAe?$AAd?$AA?$AA@ 0002f9e8     evdo.obj
 0002:00001a28       ??_C@_1EI@FCDBEBI@?$AAI?$AAn?$AAi?$AAt?$AAE?$AAV?$AAD?$AAO?$AAD?$AAl?$AAg?$AA?3?$AA?3?$AAS?$AAH?$AAC?$AAr?$AAe?$AAa?$AAt?$AAe?$AAM?$AAe?$AAn?$AAu?$AAB?$AAa?$AAr?$AA?5?$AAF?$AAa?$AAl@ 0002fa28     evdo.obj
 0002:00001a70       ??_C@_1BG@DNGPCPOD@?$AA?4?$AA?2?$AAe?$AAv?$AAd?$AAo?$AA?4?$AAc?$AAp?$AAp?$AA?$AA@ 0002fa70     evdo.obj
 0002:00001a88       ??_C@_1EG@PEMKMPDF@?$AAI?$AAn?$AAi?$AAt?$AAE?$AAV?$AAD?$AAO?$AAD?$AAl?$AAg?$AA?3?$AAS?$AAH?$AAC?$AAr?$AAe?$AAa?$AAt?$AAe?$AAM?$AAe?$AAn?$AAu?$AAB?$AAa?$AAr?$AA?5?$AAF?$AAa?$AAi?$AAl@ 0002fa88     evdo.obj
 0002:00001ad0       ??_C@_1CG@OKOLABLL@?$AAI?$AAn?$AAi?$AAt?$AAE?$AAV?$AAD?$AAO?$AAD?$AAl?$AAg?$AA?5?$AAF?$AAa?$AAi?$AAl?$AAe?$AAd?$AA?$AA@ 0002fad0     evdo.obj
 0002:00001af8       ??_C@_1FG@NHDDBKNE@?$AAC?$AAr?$AAe?$AAa?$AAt?$AAe?$AAE?$AAV?$AAD?$AAO?$AAD?$AAl?$AAg?$AA?3?$AA?3?$AAF?$AAa?$AAl?$AAi?$AAe?$AAd?$AA?5?$AAt?$AAo?$AA?5?$AAC?$AAr?$AAe?$AAa?$AAt?$AAe?$AA?5@ 0002faf8     evdo.obj
 0002:00001b50       ??_C@_1FG@FJPJJKBO@?$AAC?$AAr?$AAe?$AAa?$AAt?$AAe?$AAE?$AAV?$AAD?$AAO?$AAD?$AAl?$AAg?$AA?3?$AA?3?$AAF?$AAa?$AAl?$AAi?$AAe?$AAd?$AA?5?$AAt?$AAo?$AA?5?$AAR?$AAe?$AAg?$AAi?$AAs?$AAt?$AAe@ 0002fb50     evdo.obj
 0002:00001ba8       ??_C@_1BO@FPBBHOHH@?$AAF?$AAi?$AAn?$AAg?$AAe?$AAr?$AAD?$AAl?$AAg?$AAC?$AAl?$AAa?$AAs?$AAs?$AA?$AA@ 0002fba8     finger.obj
 0002:00001bc8       ??_C@_1BC@HHHDCBLB@?$AA?$CF?$AA?4?$AA1?$AAf?$AA?5?$AAd?$AAB?$AAm?$AA?$AA@ 0002fbc8     finger.obj
 0002:00001bdc       ??_C@_1BC@IOLLLBHP@?$AA?$HL?$AA?$CF?$AAu?$AA?0?$AA?5?$AA?$CF?$AAu?$AA?$HN?$AA?$AA@ 0002fbdc     finger.obj
 0002:00001bf0       ??_C@_1O@NMPHOONC@?$AA?$CF?$AAd?$AA?5?$AAd?$AAB?$AAm?$AA?$AA@ 0002fbf0     finger.obj
 0002:00001c00       ??_C@_1CE@MPJNAFJK@?$AAD?$AAe?$AAb?$AAu?$AAg?$AAS?$AAt?$AAa?$AAr?$AAt?$AA?5?$AAf?$AAa?$AAi?$AAl?$AAe?$AAd?$AA?$AA@ 0002fc00     finger.obj
 0002:00001c28       ??_C@_1EA@GFKEIHN@?$AAI?$AAn?$AAi?$AAt?$AAF?$AAi?$AAn?$AAg?$AAe?$AAr?$AA?3?$AA?3?$AAS?$AAH?$AAI?$AAn?$AAi?$AAt?$AAD?$AAi?$AAa?$AAl?$AAo?$AAg?$AA?5?$AAF?$AAa?$AAl?$AAi?$AAe?$AAd?$AA?$AA@ 0002fc28     finger.obj
 0002:00001c68       ??_C@_1DO@PLIBBEGP@?$AAI?$AAn?$AAi?$AAt?$AAF?$AAi?$AAn?$AAg?$AAe?$AAr?$AA?3?$AAS?$AAH?$AAI?$AAn?$AAi?$AAt?$AAD?$AAi?$AAa?$AAl?$AAo?$AAg?$AA?5?$AAF?$AAa?$AAi?$AAl?$AAe?$AAd?$AA?$AA@ 0002fc68     finger.obj
 0002:00001ca8       ??_C@_1EE@GBOCNGME@?$AAI?$AAn?$AAi?$AAt?$AAA?$AAu?$AAt?$AAh?$AAK?$AAe?$AAy?$AAD?$AAl?$AAg?$AA?3?$AA?3?$AAI?$AAn?$AAi?$AAt?$AAF?$AAi?$AAn?$AAg?$AAe?$AAr?$AA?5?$AAF?$AAa?$AAl?$AAi?$AAe@ 0002fca8     finger.obj
 0002:00001cec       ??_C@_1BK@CFKJLIBH@?$AA?4?$AA?2?$AAf?$AAi?$AAn?$AAg?$AAe?$AAr?$AA?4?$AAc?$AAp?$AAp?$AA?$AA@ 0002fcec     finger.obj
 0002:00001d08       ??_C@_1EC@OAHFNCMK@?$AAI?$AAn?$AAi?$AAt?$AAA?$AAu?$AAt?$AAh?$AAK?$AAe?$AAy?$AAD?$AAl?$AAg?$AA?3?$AAI?$AAn?$AAi?$AAt?$AAF?$AAi?$AAn?$AAg?$AAe?$AAr?$AA?5?$AAF?$AAa?$AAi?$AAl?$AAe?$AAd@ 0002fd08     finger.obj
 0002:00001d4c       ??_C@_1CE@ELFELO@?$AAI?$AAn?$AAi?$AAt?$AAF?$AAi?$AAn?$AAg?$AAe?$AAr?$AA?5?$AAF?$AAa?$AAi?$AAl?$AAe?$AAd?$AA?$AA@ 0002fd4c     finger.obj
 0002:00001d70       ??_C@_1CK@BKGGNMEA@?$AAD?$AAe?$AAb?$AAu?$AAg?$AAM?$AAo?$AAd?$AAe?$AAS?$AAt?$AAo?$AAp?$AA?5?$AAf?$AAa?$AAi?$AAl?$AAe?$AAd?$AA?$AA@ 0002fd70     finger.obj
 0002:00001da0       ??_C@_1FK@NONFGHEF@?$AAC?$AAr?$AAe?$AAa?$AAt?$AAe?$AAF?$AAi?$AAn?$AAg?$AAe?$AAr?$AAD?$AAl?$AAg?$AA?3?$AA?3?$AAF?$AAa?$AAl?$AAi?$AAe?$AAd?$AA?5?$AAt?$AAo?$AA?5?$AAC?$AAr?$AAe?$AAa?$AAt@ 0002fda0     finger.obj
 0002:00001e00       ??_C@_1FK@FABPOHIP@?$AAC?$AAr?$AAe?$AAa?$AAt?$AAe?$AAF?$AAi?$AAn?$AAg?$AAe?$AAr?$AAD?$AAl?$AAg?$AA?3?$AA?3?$AAF?$AAa?$AAl?$AAi?$AAe?$AAd?$AA?5?$AAt?$AAo?$AA?5?$AAR?$AAe?$AAg?$AAi?$AAs@ 0002fe00     finger.obj
 0002:00001e5c       ??_C@_1CA@NPFOOGJC@?$AAG?$AAP?$AAS?$AAD?$AAa?$AAt?$AAa?$AAD?$AAl?$AAg?$AAC?$AAl?$AAa?$AAs?$AAs?$AA?$AA@ 0002fe5c     gpsdatadlg.obj
 0002:00001e94       ??_C@_1CG@CNBDFNPN@?$AA?$CF?$AA0?$AA2?$AAd?$AA?$CF?$AAc?$AA?5?$AA?$CF?$AA0?$AA2?$AAd?$AA?$CC?$AA?5?$AA?$CF?$AA0?$AA2?$AAd?$AA?8?$AA?$AA@ 0002fe94     gpsdatadlg.obj
 0002:00001ebc       ??_C@_1CG@KFLCFJJF@?$AA?$CF?$AAB?$AA?5?$AA?$CF?$AAd?$AA?0?$AA?5?$AA?$CF?$AAY?$AA?5?$AA?$CF?$AAH?$AA?3?$AA?$CF?$AAM?$AA?3?$AA?$CF?$AAS?$AA?$AA@ 0002febc     gpsdatadlg.obj
 0002:00001ee4       ??_C@_1CC@CBLMKDND@?$AA?4?$AA?2?$AAg?$AAp?$AAs?$AAd?$AAa?$AAt?$AAa?$AAd?$AAl?$AAg?$AA?4?$AAc?$AAp?$AAp?$AA?$AA@ 0002fee4     gpsdatadlg.obj
 0002:00001f08       ??_C@_1FA@BAJIFONF@?$AAR?$AAe?$AAa?$AAd?$AAP?$AAD?$AAS?$AAM?$AAP?$AAA?$AAD?$AAa?$AAt?$AAa?$AA?5?$AAF?$AAa?$AAi?$AAl?$AAe?$AAd?$AA?5?$AAE?$AAr?$AAr?$AAc?$AAo?$AAd?$AAe?$AA?$DN?$AA?$CF?$AAd@ 0002ff08     gpsdatadlg.obj
 0002:00001f58       ??_C@_1FG@IGLKIBDI@?$AAE?$AAn?$AAd?$AAL?$AAB?$AAT?$AAr?$AAa?$AAc?$AAk?$AAS?$AAe?$AAs?$AAs?$AAi?$AAo?$AAn?$AA?5?$AAF?$AAa?$AAi?$AAl?$AAe?$AAd?$AA?5?$AAE?$AAr?$AAr?$AAc?$AAo?$AAd?$AAe@ 0002ff58     gpsdatadlg.obj
 0002:00001fb0       ??_C@_1FK@LDAIPOM@?$AAS?$AAt?$AAa?$AAr?$AAt?$AAL?$AAB?$AAT?$AAr?$AAa?$AAc?$AAk?$AAS?$AAe?$AAs?$AAs?$AAi?$AAo?$AAn?$AA?5?$AAF?$AAa?$AAi?$AAl?$AAe?$AAd?$AA?5?$AAE?$AAr?$AAr?$AAc?$AAo@ 0002ffb0     gpsdatadlg.obj
 0002:0000200c       ??_C@_1BI@EIJMAPGH@?$AAL?$AAB?$AAS?$AA?5?$AAS?$AAe?$AAs?$AAs?$AAi?$AAo?$AAn?$AA?$AA@ 0003000c     gpsdatadlg.obj
 0002:00002028       ??_C@_1EK@CPPGFHAH@?$AAC?$AAo?$AAu?$AAn?$AAt?$AA?5?$AAn?$AAu?$AAm?$AAb?$AAe?$AAr?$AA?5?$AAm?$AAu?$AAs?$AAt?$AA?5?$AAb?$AAe?$AA?5?$AAg?$AAr?$AAe?$AAa?$AAt?$AAe?$AAr?$AA?5?$AAt?$AAh?$AAa@ 00030028     gpsdatadlg.obj
 0002:00002078       ??_C@_1FC@OEEHBGHI@?$AAI?$AAn?$AAi?$AAt?$AAG?$AAp?$AAs?$AAD?$AAa?$AAt?$AAa?$AAD?$AAl?$AAg?$AAC?$AAl?$AAa?$AAs?$AAs?$AA?3?$AA?3?$AAS?$AAH?$AAI?$AAn?$AAi?$AAt?$AAD?$AAi?$AAa?$AAl?$AAo@ 00030078     gpsdatadlg.obj
 0002:000020d0       ??_C@_1FA@NFCFLGEI@?$AAI?$AAn?$AAi?$AAt?$AAG?$AAp?$AAs?$AAD?$AAa?$AAt?$AAa?$AAD?$AAl?$AAg?$AAC?$AAl?$AAa?$AAs?$AAs?$AA?3?$AAS?$AAH?$AAI?$AAn?$AAi?$AAt?$AAD?$AAi?$AAa?$AAl?$AAo?$AAg@ 000300d0     gpsdatadlg.obj
 0002:00002120       ??_C@_1FI@CFEDNADD@?$AAI?$AAn?$AAi?$AAt?$AAG?$AAp?$AAs?$AAD?$AAa?$AAt?$AAa?$AAD?$AAl?$AAg?$AAC?$AAl?$AAa?$AAs?$AAs?$AA?3?$AA?3?$AAS?$AAH?$AAC?$AAr?$AAe?$AAa?$AAt?$AAe?$AAM?$AAe?$AAn@ 00030120     gpsdatadlg.obj
 0002:00002178       ??_C@_1FG@LFKLIOHM@?$AAI?$AAn?$AAi?$AAt?$AAG?$AAp?$AAs?$AAD?$AAa?$AAt?$AAa?$AAD?$AAl?$AAg?$AAC?$AAl?$AAa?$AAs?$AAs?$AA?3?$AAS?$AAH?$AAC?$AAr?$AAe?$AAa?$AAt?$AAe?$AAM?$AAe?$AAn?$AAu@ 00030178     gpsdatadlg.obj
 0002:000021d0       ??_C@_1DG@DEDALOII@?$AAI?$AAn?$AAi?$AAt?$AAG?$AAp?$AAs?$AAD?$AAa?$AAt?$AAa?$AAD?$AAl?$AAg?$AAC?$AAl?$AAa?$AAs?$AAs?$AA?5?$AAF?$AAa?$AAi?$AAl?$AAe?$AAd?$AA?$AA@ 000301d0     gpsdatadlg.obj
 0002:00002208       ??_C@_1O@EMLLFJNI@?$AAA?$AAc?$AAt?$AAi?$AAv?$AAe?$AA?$AA@ 00030208     gpsdatadlg.obj
 0002:00002218       ??_C@_1BC@GMDCIECL@?$AAI?$AAn?$AAa?$AAc?$AAt?$AAi?$AAv?$AAe?$AA?$AA@ 00030218     gpsdatadlg.obj
 0002:00002230       ??_C@_1FM@BKKNMCDN@?$AAC?$AAr?$AAe?$AAa?$AAt?$AAe?$AAG?$AAp?$AAs?$AAD?$AAa?$AAt?$AAa?$AAD?$AAl?$AAg?$AA?3?$AA?3?$AAF?$AAa?$AAl?$AAi?$AAe?$AAd?$AA?5?$AAt?$AAo?$AA?5?$AAC?$AAr?$AAe?$AAa@ 00030230     gpsdatadlg.obj
 0002:00002290       ??_C@_1FM@JEGHECPH@?$AAC?$AAr?$AAe?$AAa?$AAt?$AAe?$AAG?$AAp?$AAs?$AAD?$AAa?$AAt?$AAa?$AAD?$AAl?$AAg?$AA?3?$AA?3?$AAF?$AAa?$AAl?$AAi?$AAe?$AAd?$AA?5?$AAt?$AAo?$AA?5?$AAR?$AAe?$AAg?$AAi@ 00030290     gpsdatadlg.obj
 0002:000022ec       ??_C@_1CI@LIMCLCKJ@?$AAG?$AAP?$AAS?$AAS?$AAe?$AAt?$AAt?$AAi?$AAn?$AAg?$AAs?$AAD?$AAl?$AAg?$AAC?$AAl?$AAa?$AAs?$AAs?$AA?$AA@ 000302ec     gpssettingsdlg.obj
 0002:00002360       ??_C@_0M@CDHNGIPM@?$CFu?4?$CFu?4?$CFu?4?$CFu?$AA@ 00030360     gpssettingsdlg.obj
 0002:0000236c       ??_C@_1CA@MGANECGC@?$AA?$CK?$AA?$CK?$AA?$CK?$AA?4?$AA?$CK?$AA?$CK?$AA?$CK?$AA?4?$AA?$CK?$AA?$CK?$AA?$CK?$AA?4?$AA?$CK?$AA?$CK?$AA?$CK?$AA?$AA@ 0003036c     gpssettingsdlg.obj
 0002:0000238c       ??_C@_19EFAEBDAE@?$AA?$CK?$AA?$CK?$AA?$CK?$AA?$CK?$AA?$AA@ 0003038c     gpssettingsdlg.obj
 0002:00002398       ??_C@_1DG@PKPFFJGG@?$AAA?$AAb?$AAo?$AAu?$AAt?$AA?5?$AAt?$AAo?$AA?5?$AAs?$AAa?$AAv?$AAe?$AA?5?$AAF?$AAi?$AAx?$AAM?$AAo?$AAd?$AAe?$AA?5?$AA?$DN?$AA?5?$AA?$CF?$AAd?$AA?$AA@ 00030398     gpssettingsdlg.obj
 0002:000023d0       ??_C@_1IG@BMBMBHGO@?$AAG?$AAe?$AAt?$AAd?$AAa?$AAt?$AAa?$AAF?$AAr?$AAo?$AAm?$AAC?$AAt?$AAr?$AAl?$AAs?$AA?3?$AA?3?$AA?5?$AAU?$AAs?$AAe?$AAr?$AA?5?$AAh?$AAa?$AAs?$AA?5?$AAe?$AAn?$AAt?$AAe@ 000303d0     gpssettingsdlg.obj
 0002:00002458       ??_C@_1BCM@LHECELJN@?$AAY?$AAo?$AAu?$AA?5?$AAh?$AAa?$AAv?$AAe?$AA?5?$AAe?$AAn?$AAt?$AAe?$AAr?$AAe?$AAd?$AA?5?$AAa?$AAn?$AA?5?$AAi?$AAn?$AAv?$AAa?$AAl?$AAi?$AAd?$AA?5?$AAI?$AAP?$AA?5?$AAa@ 00030458     gpssettingsdlg.obj
 0002:00002588       ??_C@_1MO@IJIFDFDF@?$AA?5?$AAG?$AAe?$AAt?$AAd?$AAa?$AAt?$AAa?$AAF?$AAr?$AAo?$AAm?$AAC?$AAt?$AAr?$AAl?$AAs?$AA?3?$AA?3?$AA?5?$AAU?$AAs?$AAe?$AAr?$AA?5?$AAh?$AAa?$AAs?$AA?5?$AAN?$AAO?$AAT@ 00030588     gpssettingsdlg.obj
 0002:00002658       ??_C@_1IA@COKOAIOD@?$AAG?$AAe?$AAt?$AAd?$AAa?$AAt?$AAa?$AAF?$AAr?$AAo?$AAm?$AAC?$AAt?$AAr?$AAl?$AAs?$AA?3?$AA?3?$AA?5?$AAU?$AAs?$AAe?$AAr?$AA?5?$AAh?$AAa?$AAs?$AA?5?$AAe?$AAn?$AAt?$AAe@ 00030658     gpssettingsdlg.obj
 0002:000026d8       ??_C@_1BAK@GDBKDPIF@?$AAY?$AAo?$AAu?$AA?5?$AAh?$AAa?$AAv?$AAe?$AA?5?$AAe?$AAn?$AAt?$AAe?$AAr?$AAe?$AAd?$AA?5?$AAa?$AAn?$AA?5?$AAi?$AAn?$AAv?$AAa?$AAl?$AAi?$AAd?$AA?5?$AAP?$AAo?$AAr?$AAt@ 000306d8     gpssettingsdlg.obj
 0002:000027e4       ??_C@_1M@ILHOPKA@?$AAE?$AAr?$AAr?$AAo?$AAr?$AA?$AA@ 000307e4     gpssettingsdlg.obj
 0002:000027f0       ??_C@_1CK@IJMEHDCP@?$AA?4?$AA?2?$AAg?$AAp?$AAs?$AAs?$AAe?$AAt?$AAt?$AAi?$AAn?$AAg?$AAs?$AAd?$AAl?$AAg?$AA?4?$AAc?$AAp?$AAp?$AA?$AA@ 000307f0     gpssettingsdlg.obj
 0002:00002820       ??_C@_1MC@DBBOFFBK@?$AA?5?$AAG?$AAe?$AAt?$AAd?$AAa?$AAt?$AAa?$AAF?$AAr?$AAo?$AAm?$AAC?$AAt?$AAr?$AAl?$AAs?$AA?3?$AA?3?$AA?5?$AAU?$AAs?$AAe?$AAr?$AA?5?$AAh?$AAa?$AAs?$AA?5?$AAN?$AAO?$AAT@ 00030820     gpssettingsdlg.obj
 0002:000028e8       ??_C@_1FC@KEKIGJAN@?$AAR?$AAe?$AAa?$AAd?$AAP?$AAD?$AAS?$AAM?$AAP?$AAA?$AAP?$AAa?$AAr?$AAa?$AAm?$AA?5?$AAF?$AAa?$AAi?$AAl?$AAe?$AAd?$AA?5?$AAE?$AAr?$AAr?$AAc?$AAo?$AAd?$AAe?$AA?$DN?$AA?$CF@ 000308e8     gpssettingsdlg.obj
 0002:00002940       ??_C@_1FK@MPDDKGOM@?$AAS?$AAa?$AAv?$AAe?$AAG?$AAp?$AAs?$AAS?$AAe?$AAt?$AAt?$AAi?$AAn?$AAg?$AAs?$AA?3?$AA?3?$AA?5?$AAG?$AAP?$AAS?$AA?5?$AAs?$AAe?$AAt?$AAt?$AAi?$AAn?$AAg?$AAs?$AA?5?$AAa@ 00030940     gpssettingsdlg.obj
 0002:000029a0       ??_C@_1HE@GLNCAMGC@?$AAS?$AAa?$AAv?$AAe?$AAG?$AAp?$AAs?$AAS?$AAe?$AAt?$AAt?$AAi?$AAn?$AAg?$AAs?$AA?3?$AA?3?$AA?5?$AAS?$AAe?$AAt?$AAP?$AAD?$AAS?$AAM?$AAP?$AAA?$AAP?$AAa?$AAr?$AAa?$AAm@ 000309a0     gpssettingsdlg.obj
 0002:00002a18       ??_C@_1FK@JFCDMCHM@?$AAI?$AAn?$AAi?$AAt?$AAG?$AAp?$AAs?$AAS?$AAe?$AAt?$AAt?$AAi?$AAn?$AAg?$AAs?$AAD?$AAl?$AAg?$AAC?$AAl?$AAa?$AAs?$AAs?$AA?3?$AA?3?$AAS?$AAH?$AAI?$AAn?$AAi?$AAt?$AAD@ 00030a18     gpssettingsdlg.obj
 0002:00002a78       ??_C@_1FI@OEOJBGGK@?$AAI?$AAn?$AAi?$AAt?$AAG?$AAp?$AAs?$AAS?$AAe?$AAt?$AAt?$AAi?$AAn?$AAg?$AAs?$AAD?$AAl?$AAg?$AAC?$AAl?$AAa?$AAs?$AAs?$AA?3?$AAS?$AAH?$AAI?$AAn?$AAi?$AAt?$AAD?$AAi@ 00030a78     gpssettingsdlg.obj
 0002:00002ad0       ??_C@_1GA@CDNACJIP@?$AAI?$AAn?$AAi?$AAt?$AAG?$AAp?$AAs?$AAS?$AAe?$AAt?$AAt?$AAi?$AAn?$AAg?$AAs?$AAD?$AAl?$AAg?$AAC?$AAl?$AAa?$AAs?$AAs?$AA?3?$AA?3?$AAS?$AAH?$AAC?$AAr?$AAe?$AAa?$AAt@ 00030ad0     gpssettingsdlg.obj
 0002:00002b30       ??_C@_1FO@JGNKGLMO@?$AAI?$AAn?$AAi?$AAt?$AAG?$AAp?$AAs?$AAS?$AAe?$AAt?$AAt?$AAi?$AAn?$AAg?$AAs?$AAD?$AAl?$AAg?$AAC?$AAl?$AAa?$AAs?$AAs?$AA?3?$AAS?$AAH?$AAC?$AAr?$AAe?$AAa?$AAt?$AAe@ 00030b30     gpssettingsdlg.obj
 0002:00002b90       ??_C@_1DO@PIKGDJK@?$AAI?$AAn?$AAi?$AAt?$AAG?$AAp?$AAs?$AAS?$AAe?$AAt?$AAt?$AAi?$AAn?$AAg?$AAs?$AAD?$AAl?$AAg?$AAC?$AAl?$AAa?$AAs?$AAs?$AA?5?$AAF?$AAa?$AAi?$AAl?$AAe?$AAd?$AA?$AA@ 00030b90     gpssettingsdlg.obj
 0002:00002bd0       ??_C@_1FE@NIGLGLJH@?$AAP?$AAh?$AAo?$AAn?$AAe?$AAU?$AAt?$AAi?$AAl?$AAi?$AAt?$AAy?$AA?3?$AA?5?$AAF?$AAa?$AAi?$AAl?$AAe?$AAd?$AA?5?$AAt?$AAo?$AA?5?$AAs?$AAa?$AAv?$AAe?$AA?5?$AAG?$AAP?$AAS@ 00030bd0     gpssettingsdlg.obj
 0002:00002c28       ??_C@_1JO@IOOCDDDE@?$AAP?$AAh?$AAo?$AAn?$AAe?$AAU?$AAt?$AAi?$AAl?$AAi?$AAt?$AAy?$AA?3?$AA?5?$AAF?$AAa?$AAi?$AAl?$AAe?$AAd?$AA?5?$AAt?$AAo?$AA?5?$AAr?$AAe?$AAs?$AAe?$AAt?$AA?5?$AAt?$AAh@ 00030c28     gpssettingsdlg.obj
 0002:00002cc8       ??_C@_1GE@PFIGHMK@?$AAC?$AAr?$AAe?$AAa?$AAt?$AAe?$AAG?$AAp?$AAs?$AAS?$AAe?$AAt?$AAt?$AAi?$AAn?$AAg?$AAs?$AAD?$AAl?$AAg?$AA?3?$AA?3?$AAF?$AAa?$AAl?$AAi?$AAe?$AAd?$AA?5?$AAt?$AAo?$AA?5@ 00030cc8     gpssettingsdlg.obj
 0002:00002d30       ??_C@_1GE@IBJCOHAA@?$AAC?$AAr?$AAe?$AAa?$AAt?$AAe?$AAG?$AAp?$AAs?$AAS?$AAe?$AAt?$AAt?$AAi?$AAn?$AAg?$AAs?$AAD?$AAl?$AAg?$AA?3?$AA?3?$AAF?$AAa?$AAl?$AAi?$AAe?$AAd?$AA?5?$AAt?$AAo?$AA?5@ 00030d30     gpssettingsdlg.obj
 0002:00002d94       ??_C@_1BG@PNGHMGJN@?$AAG?$AAS?$AAM?$AA2?$AAG?$AAC?$AAl?$AAa?$AAs?$AAs?$AA?$AA@ 00030d94     gsm2G.obj
 0002:00002dac       ??_C@_1DO@MGMEFCKJ@?$AAI?$AAn?$AAi?$AAt?$AAG?$AAS?$AAM?$AA2?$AAG?$AA?3?$AA?3?$AAS?$AAH?$AAI?$AAn?$AAi?$AAt?$AAD?$AAi?$AAa?$AAl?$AAo?$AAg?$AA?5?$AAF?$AAa?$AAl?$AAi?$AAe?$AAd?$AA?$AA@ 00030dac     gsm2G.obj
 0002:00002dec       ??_C@_1DM@DJFLMNJM@?$AAI?$AAn?$AAi?$AAt?$AAG?$AAS?$AAM?$AA2?$AAG?$AA?3?$AAS?$AAH?$AAI?$AAn?$AAi?$AAt?$AAD?$AAi?$AAa?$AAl?$AAo?$AAg?$AA?5?$AAF?$AAa?$AAi?$AAl?$AAe?$AAd?$AA?$AA@ 00030dec     gsm2G.obj
 0002:00002e28       ??_C@_1EE@JFHHGKGL@?$AAI?$AAn?$AAi?$AAt?$AAG?$AAS?$AAM?$AA2?$AAG?$AA?3?$AA?3?$AAS?$AAH?$AAC?$AAr?$AAe?$AAa?$AAt?$AAe?$AAM?$AAe?$AAn?$AAu?$AAB?$AAa?$AAr?$AA?5?$AAF?$AAa?$AAl?$AAi?$AAe@ 00030e28     gsm2G.obj
 0002:00002e6c       ??_C@_1BI@PKIIEOLH@?$AA?4?$AA?2?$AAg?$AAs?$AAm?$AA2?$AAG?$AA?4?$AAc?$AAp?$AAp?$AA?$AA@ 00030e6c     gsm2G.obj
 0002:00002e88       ??_C@_1EC@JJBOPPPA@?$AAI?$AAn?$AAi?$AAt?$AAG?$AAS?$AAM?$AA2?$AAG?$AA?3?$AAS?$AAH?$AAC?$AAr?$AAe?$AAa?$AAt?$AAe?$AAM?$AAe?$AAn?$AAu?$AAB?$AAa?$AAr?$AA?5?$AAF?$AAa?$AAi?$AAl?$AAe?$AAd@ 00030e88     gsm2G.obj
 0002:00002ecc       ??_C@_1CC@LIGHGKCJ@?$AAI?$AAn?$AAi?$AAt?$AAG?$AAS?$AAM?$AA2?$AAG?$AA?5?$AAF?$AAa?$AAi?$AAl?$AAe?$AAd?$AA?$AA@ 00030ecc     gsm2G.obj
 0002:00002ef0       ??_C@_1FC@HFPMKOHD@?$AAC?$AAr?$AAe?$AAa?$AAt?$AAe?$AAG?$AAS?$AAM?$AA2?$AAG?$AA?3?$AA?3?$AAF?$AAa?$AAl?$AAi?$AAe?$AAd?$AA?5?$AAt?$AAo?$AA?5?$AAR?$AAe?$AAg?$AAi?$AAs?$AAt?$AAe?$AAr?$AAC@ 00030ef0     gsm2G.obj
 0002:00002f44       ??_C@_1CG@KEDNNPKD@?$AAG?$AAS?$AAM?$AA3?$AAG?$AAI?$AAt?$AAe?$AAm?$AAn?$AAi?$AAz?$AAe?$AAC?$AAl?$AAa?$AAs?$AAs?$AA?$AA@ 00030f44     gsm3G.obj
 0002:00002f6c       ??_C@_1BG@FDAPFHAM@?$AAG?$AAS?$AAM?$AA3?$AAG?$AAC?$AAl?$AAa?$AAs?$AAs?$AA?$AA@ 00030f6c     gsm3G.obj
 0002:00002f88       ??_C@_1EO@LMKGBJDP@?$AAI?$AAn?$AAi?$AAt?$AAG?$AAS?$AAM?$AA3?$AAG?$AAI?$AAt?$AAe?$AAm?$AAn?$AAi?$AAz?$AAe?$AA?3?$AA?3?$AAS?$AAH?$AAI?$AAn?$AAi?$AAt?$AAD?$AAi?$AAa?$AAl?$AAo?$AAg?$AA?5@ 00030f88     gsm3G.obj
 0002:00002fd8       ??_C@_1EM@EFFIGLNB@?$AAI?$AAn?$AAi?$AAt?$AAG?$AAS?$AAM?$AA3?$AAG?$AAI?$AAt?$AAe?$AAm?$AAn?$AAi?$AAz?$AAe?$AA?3?$AAS?$AAH?$AAI?$AAn?$AAi?$AAt?$AAD?$AAi?$AAa?$AAl?$AAo?$AAg?$AA?5?$AAF@ 00030fd8     gsm3G.obj
 0002:00003028       ??_C@_1FE@LJCCCEGD@?$AAI?$AAn?$AAi?$AAt?$AAG?$AAS?$AAM?$AA3?$AAG?$AAI?$AAt?$AAe?$AAm?$AAn?$AAi?$AAz?$AAe?$AA?3?$AA?3?$AAS?$AAH?$AAC?$AAr?$AAe?$AAa?$AAt?$AAe?$AAM?$AAe?$AAn?$AAu?$AAB@ 00031028     gsm3G.obj
 0002:0000307c       ??_C@_1BI@GHIHKPMB@?$AA?4?$AA?2?$AAg?$AAs?$AAm?$AA3?$AAG?$AA?4?$AAc?$AAp?$AAp?$AA?$AA@ 0003107c     gsm3G.obj
 0002:00003098       ??_C@_1FC@JKOBLCKO@?$AAI?$AAn?$AAi?$AAt?$AAG?$AAS?$AAM?$AA3?$AAG?$AAI?$AAt?$AAe?$AAm?$AAn?$AAi?$AAz?$AAe?$AA?3?$AAS?$AAH?$AAC?$AAr?$AAe?$AAa?$AAt?$AAe?$AAM?$AAe?$AAn?$AAu?$AAB?$AAa@ 00031098     gsm3G.obj
 0002:000030ec       ??_C@_1DC@GLAEKDBP@?$AAI?$AAn?$AAi?$AAt?$AAG?$AAS?$AAM?$AA3?$AAG?$AAI?$AAt?$AAe?$AAm?$AAn?$AAi?$AAz?$AAe?$AA?5?$AAF?$AAa?$AAi?$AAl?$AAe?$AAd?$AA?$AA@ 000310ec     gsm3G.obj
 0002:00003120       ??_C@_1GC@DFKLCNO@?$AAC?$AAr?$AAe?$AAa?$AAt?$AAe?$AAG?$AAS?$AAM?$AA3?$AAG?$AAI?$AAt?$AAe?$AAm?$AAn?$AAi?$AAz?$AAe?$AA?3?$AA?3?$AAF?$AAa?$AAl?$AAi?$AAe?$AAd?$AA?5?$AAt?$AAo?$AA?5?$AAR@ 00031120     gsm3G.obj
 0002:00003184       ??_C@_1CC@NNAAFBGP@?$AAI?$AAn?$AAi?$AAt?$AAG?$AAS?$AAM?$AA3?$AAG?$AA?5?$AAF?$AAa?$AAi?$AAl?$AAe?$AAd?$AA?$AA@ 00031184     gsm3G.obj
 0002:000031a8       ??_C@_1FC@PKMJIDOG@?$AAC?$AAr?$AAe?$AAa?$AAt?$AAe?$AAG?$AAS?$AAM?$AA3?$AAG?$AA?3?$AA?3?$AAF?$AAa?$AAl?$AAi?$AAe?$AAd?$AA?5?$AAt?$AAo?$AA?5?$AAR?$AAe?$AAg?$AAi?$AAs?$AAt?$AAe?$AAr?$AAC@ 000311a8     gsm3G.obj
 0002:000031fc       ??_C@_1BK@GKGBABJM@?$AAG?$AAS?$AAM?$AAB?$AAa?$AAn?$AAd?$AAC?$AAl?$AAa?$AAs?$AAs?$AA?$AA@ 000311fc     gsmband.obj
 0002:00003218       ??_C@_1FC@PGACGEHL@?$AAI?$AAn?$AAi?$AAt?$AAG?$AAS?$AAM?$AAB?$AAa?$AAn?$AAd?$AAI?$AAt?$AAe?$AAm?$AAn?$AAi?$AAz?$AAe?$AA?3?$AA?3?$AAS?$AAH?$AAI?$AAn?$AAi?$AAt?$AAD?$AAi?$AAa?$AAl?$AAo@ 00031218     gsmband.obj
 0002:00003270       ??_C@_1FA@CMHGKBBL@?$AAI?$AAn?$AAi?$AAt?$AAG?$AAS?$AAM?$AAB?$AAa?$AAn?$AAd?$AAI?$AAt?$AAe?$AAm?$AAn?$AAi?$AAz?$AAe?$AA?3?$AAS?$AAH?$AAI?$AAn?$AAi?$AAt?$AAD?$AAi?$AAa?$AAl?$AAo?$AAg@ 00031270     gsmband.obj
 0002:000032c0       ??_C@_1FI@JDKNMOCD@?$AAI?$AAn?$AAi?$AAt?$AAG?$AAS?$AAM?$AAB?$AAa?$AAn?$AAd?$AAI?$AAt?$AAe?$AAm?$AAn?$AAi?$AAz?$AAe?$AA?3?$AA?3?$AAS?$AAH?$AAC?$AAr?$AAe?$AAa?$AAt?$AAe?$AAM?$AAe?$AAn@ 000312c0     gsmband.obj
 0002:00003318       ??_C@_1BM@IEMGNCFJ@?$AA?4?$AA?2?$AAg?$AAs?$AAm?$AAb?$AAa?$AAn?$AAd?$AA?4?$AAc?$AAp?$AAp?$AA?$AA@ 00031318     gsmband.obj
 0002:00003338       ??_C@_1FG@IONMFHKE@?$AAI?$AAn?$AAi?$AAt?$AAG?$AAS?$AAM?$AAB?$AAa?$AAn?$AAd?$AAI?$AAt?$AAe?$AAm?$AAn?$AAi?$AAz?$AAe?$AA?3?$AAS?$AAH?$AAC?$AAr?$AAe?$AAa?$AAt?$AAe?$AAM?$AAe?$AAn?$AAu@ 00031338     gsmband.obj
 0002:00003390       ??_C@_1CG@POAMEMMC@?$AAI?$AAn?$AAi?$AAt?$AAG?$AAS?$AAM?$AAB?$AAa?$AAn?$AAd?$AA?5?$AAF?$AAa?$AAi?$AAl?$AAe?$AAd?$AA?$AA@ 00031390     gsmband.obj
 0002:000033b8       ??_C@_1EE@PFOHEFLH@?$AAF?$AAa?$AAi?$AAl?$AA?5?$AAt?$AAo?$AA?5?$AAS?$AAe?$AAl?$AAe?$AAc?$AAt?$AAG?$AAS?$AAM?$AAB?$AAa?$AAn?$AAd?$AA?0?$AA?5?$AAe?$AAr?$AAr?$AAo?$AAr?$AA?5?$AA?$DN?$AA?5?$AA?$CF@ 000313b8     gsmband.obj
 0002:00003400       ??_C@_1FG@GLDLBJJN@?$AAC?$AAr?$AAe?$AAa?$AAt?$AAe?$AAG?$AAS?$AAM?$AAB?$AAa?$AAn?$AAd?$AA?3?$AA?3?$AAF?$AAa?$AAi?$AAl?$AAe?$AAd?$AA?5?$AAt?$AAo?$AA?5?$AAR?$AAe?$AAg?$AAi?$AAs?$AAt?$AAe@ 00031400     gsmband.obj
 0002:00003458       ??_C@_1FG@IHNDGHBD@?$AAC?$AAr?$AAe?$AAa?$AAt?$AAe?$AAG?$AAS?$AAM?$AAB?$AAa?$AAn?$AAd?$AA?3?$AA?3?$AAF?$AAa?$AAl?$AAi?$AAe?$AAd?$AA?5?$AAt?$AAo?$AA?5?$AAR?$AAe?$AAg?$AAi?$AAs?$AAt?$AAe@ 00031458     gsmband.obj
 0002:000034b0       ??_C@_1BK@COLOLAGJ@?$AAI?$AAO?$AAT?$AAA?$AAD?$AAl?$AAg?$AAC?$AAl?$AAa?$AAs?$AAs?$AA?$AA@ 000314b0     iota.obj
 0002:000034d0       ??_C@_1EC@EAKJJJHH@?$AAI?$AAn?$AAi?$AAt?$AAI?$AAO?$AAT?$AAA?$AAD?$AAl?$AAg?$AA?3?$AA?3?$AAS?$AAH?$AAI?$AAn?$AAi?$AAt?$AAD?$AAi?$AAa?$AAl?$AAo?$AAg?$AA?5?$AAF?$AAa?$AAl?$AAi?$AAe?$AAd@ 000314d0     iota.obj
 0002:00003518       ??_C@_1EA@CLEBANOO@?$AAI?$AAn?$AAi?$AAt?$AAI?$AAO?$AAT?$AAA?$AAD?$AAl?$AAg?$AA?3?$AAS?$AAH?$AAI?$AAn?$AAi?$AAt?$AAD?$AAi?$AAa?$AAl?$AAo?$AAg?$AA?5?$AAF?$AAa?$AAi?$AAl?$AAe?$AAd?$AA?$AA@ 00031518     iota.obj
 0002:00003558       ??_C@_1EI@PHCIGBC@?$AAI?$AAn?$AAi?$AAt?$AAI?$AAO?$AAT?$AAA?$AAD?$AAl?$AAg?$AA?3?$AA?3?$AAS?$AAH?$AAC?$AAr?$AAe?$AAa?$AAt?$AAe?$AAM?$AAe?$AAn?$AAu?$AAB?$AAa?$AAr?$AA?5?$AAF?$AAa?$AAl@ 00031558     iota.obj
 0002:000035a0       ??_C@_1BG@JFEJIJNL@?$AA?4?$AA?2?$AAi?$AAo?$AAt?$AAa?$AA?4?$AAc?$AAp?$AAp?$AA?$AA@ 000315a0     iota.obj
 0002:000035b8       ??_C@_1EG@BGOHHLAE@?$AAI?$AAn?$AAi?$AAt?$AAI?$AAO?$AAT?$AAA?$AAD?$AAl?$AAg?$AA?3?$AAS?$AAH?$AAC?$AAr?$AAe?$AAa?$AAt?$AAe?$AAM?$AAe?$AAn?$AAu?$AAB?$AAa?$AAr?$AA?5?$AAF?$AAa?$AAi?$AAl@ 000315b8     iota.obj
 0002:00003600       ??_C@_1CG@PMDJGCCJ@?$AAI?$AAn?$AAi?$AAt?$AAI?$AAO?$AAT?$AAA?$AAD?$AAl?$AAg?$AA?5?$AAF?$AAa?$AAi?$AAl?$AAe?$AAd?$AA?$AA@ 00031600     iota.obj
 0002:00003628       ??_C@_1FG@BJIOEMLD@?$AAC?$AAr?$AAe?$AAa?$AAt?$AAe?$AAI?$AAO?$AAT?$AAA?$AAD?$AAl?$AAg?$AA?3?$AA?3?$AAF?$AAa?$AAl?$AAi?$AAe?$AAd?$AA?5?$AAt?$AAo?$AA?5?$AAC?$AAr?$AAe?$AAa?$AAt?$AAe?$AA?5@ 00031628     iota.obj
 0002:00003680       ??_C@_1FG@JHEEMMHJ@?$AAC?$AAr?$AAe?$AAa?$AAt?$AAe?$AAI?$AAO?$AAT?$AAA?$AAD?$AAl?$AAg?$AA?3?$AA?3?$AAF?$AAa?$AAl?$AAi?$AAe?$AAd?$AA?5?$AAt?$AAo?$AA?5?$AAR?$AAe?$AAg?$AAi?$AAs?$AAt?$AAe@ 00031680     iota.obj
 0002:0000b394       ??_C@_1BM@FEGPDFAG@?$AAS?$AAy?$AAs?$AAL?$AAi?$AAs?$AAt?$AAV?$AAi?$AAe?$AAw?$AA3?$AA2?$AA?$AA@ 00039394     listview.obj
 0002:0000b3b0       ??_C@_1BO@CKMBKLHM@?$AA?4?$AA?2?$AAl?$AAi?$AAs?$AAt?$AAv?$AAi?$AAe?$AAw?$AA?4?$AAc?$AAp?$AAp?$AA?$AA@ 000393b0     listview.obj
 0002:0000b3d0       ??_C@_1GA@OPNDGMGH@?$AAC?$AAr?$AAe?$AAa?$AAt?$AAe?$AAE?$AAR?$AAI?$AAW?$AAi?$AAn?$AAd?$AAo?$AAw?$AA?5?$AA?5?$AAF?$AAa?$AAi?$AAl?$AAe?$AAd?$AA?5?$AAt?$AAo?$AA?5?$AAG?$AAe?$AAt?$AA?5?$AAP@ 000393d0     listview.obj
 0002:0000b430       ??_C@_1DC@EBFLAGON@?$AAC?$AAa?$AAn?$AA?5?$AAn?$AAo?$AAt?$AA?5?$AAc?$AAr?$AAe?$AAa?$AAt?$AAe?$AA?5?$AAd?$AAi?$AAa?$AAl?$AAo?$AAg?$AA?5?$AA?$CF?$AAd?$AA?$AA@ 00039430     listview.obj
 0002:0000b464       ??_C@_1M@IDCMGJNH@?$AAC?$AAL?$AAE?$AAA?$AAR?$AA?$AA@ 00039464     listview.obj
 0002:0000b470       ??_C@_1CC@CJNFMFAA@?$AAL?$AAo?$AAo?$AAp?$AAB?$AAa?$AAc?$AAk?$AAD?$AAl?$AAg?$AAC?$AAl?$AAa?$AAs?$AAs?$AA?$AA@ 00039470     loopbackdlg.obj
 0002:0000b590       ??_C@_1CE@EHOHAHMC@?$AA?4?$AA?2?$AAl?$AAo?$AAo?$AAp?$AAb?$AAa?$AAc?$AAk?$AAd?$AAl?$AAg?$AA?4?$AAc?$AAp?$AAp?$AA?$AA@ 00039590     loopbackdlg.obj
 0002:0000b5b4       ??_C@_1CK@BLHDMNPF@?$AAE?$AAr?$AAr?$AA?5?$AA?$DN?$AA?5?$AA?$CF?$AAd?$AA?5?$AA?0?$AAE?$AAr?$AAr?$AAD?$AAe?$AAs?$AAc?$AA?$DN?$AA?$CF?$AAs?$AA?$AA@ 000395b4     loopbackdlg.obj
 0002:0000b5e0       ??_C@_17LGKOMLJ@?$AA?4?$AA?4?$AA?4?$AA?$AA@ 000395e0     loopbackdlg.obj
 0002:0000b5e8       ??_C@_13EBCNDICG@?$AA?3?$AA?$AA@ 000395e8     loopbackdlg.obj
 0002:0000b5f0       ??_C@_1EK@LCALJOEH@?$AAI?$AAn?$AAi?$AAt?$AAL?$AAo?$AAo?$AAp?$AAB?$AAa?$AAc?$AAk?$AAD?$AAl?$AAg?$AA?3?$AA?3?$AAS?$AAH?$AAI?$AAn?$AAi?$AAt?$AAD?$AAi?$AAa?$AAl?$AAo?$AAg?$AA?5?$AAF?$AAa@ 000395f0     loopbackdlg.obj
 0002:0000b640       ??_C@_1EI@JGFDPDJB@?$AAI?$AAn?$AAi?$AAt?$AAL?$AAo?$AAo?$AAp?$AAB?$AAa?$AAc?$AAk?$AAD?$AAl?$AAg?$AA?3?$AAS?$AAH?$AAI?$AAn?$AAi?$AAt?$AAD?$AAi?$AAa?$AAl?$AAo?$AAg?$AA?5?$AAF?$AAa?$AAi@ 00039640     loopbackdlg.obj
 0002:0000b688       ??_C@_1HG@CFNJBJNO@?$AAI?$AAn?$AAi?$AAt?$AAL?$AAo?$AAo?$AAp?$AAB?$AAa?$AAc?$AAk?$AAD?$AAl?$AAg?$AA?3?$AA?3?$AAS?$AAH?$AAC?$AAr?$AAe?$AAa?$AAt?$AAe?$AAM?$AAe?$AAn?$AAu?$AAB?$AAa?$AAr@ 00039688     loopbackdlg.obj
 0002:0000b700       ??_C@_1HE@IEGCMDDI@?$AAI?$AAn?$AAi?$AAt?$AAL?$AAo?$AAo?$AAp?$AAB?$AAa?$AAc?$AAk?$AAD?$AAl?$AAg?$AA?3?$AAS?$AAH?$AAC?$AAr?$AAe?$AAa?$AAt?$AAe?$AAM?$AAe?$AAn?$AAu?$AAB?$AAa?$AAr?$AA?5@ 00039700     loopbackdlg.obj
 0002:0000b778       ??_C@_1HA@CMLBBFFG@?$AAI?$AAn?$AAi?$AAt?$AAL?$AAo?$AAo?$AAp?$AAB?$AAa?$AAc?$AAk?$AAD?$AAl?$AAg?$AA?3?$AA?3?$AAS?$AAH?$AAC?$AAr?$AAe?$AAa?$AAt?$AAe?$AAM?$AAe?$AAn?$AAu?$AAB?$AAa?$AAr@ 00039778     loopbackdlg.obj
 0002:0000b7e8       ??_C@_1GO@DKPPGMJK@?$AAI?$AAn?$AAi?$AAt?$AAL?$AAo?$AAo?$AAp?$AAB?$AAa?$AAc?$AAk?$AAD?$AAl?$AAg?$AA?3?$AAS?$AAH?$AAC?$AAr?$AAe?$AAa?$AAt?$AAe?$AAM?$AAe?$AAn?$AAu?$AAB?$AAa?$AAr?$AA?5@ 000397e8     loopbackdlg.obj
 0002:0000b858       ??_C@_13BBDEGPLJ@?$AA?$CK?$AA?$AA@ 00039858     loopbackdlg.obj
 0002:0000b85c       ??_C@_13GMDMCADD@?$AA?$CD?$AA?$AA@ 0003985c     loopbackdlg.obj
 0002:0000b860       ??_C@_1CO@NDKNAJDN@?$AAI?$AAn?$AAi?$AAt?$AAL?$AAo?$AAo?$AAp?$AAB?$AAa?$AAc?$AAk?$AAD?$AAl?$AAg?$AA?5?$AAF?$AAa?$AAi?$AAl?$AAe?$AAd?$AA?$AA@ 00039860     loopbackdlg.obj
 0002:0000b890       ??_C@_1FO@GABGMGPJ@?$AAC?$AAr?$AAe?$AAa?$AAt?$AAe?$AAL?$AAo?$AAo?$AAp?$AAB?$AAa?$AAc?$AAk?$AAD?$AAl?$AAg?$AA?3?$AA?3?$AAF?$AAa?$AAl?$AAi?$AAe?$AAd?$AA?5?$AAt?$AAo?$AA?5?$AAC?$AAr?$AAe@ 00039890     loopbackdlg.obj
 0002:0000b8f0       ??_C@_1FO@OONMEGDD@?$AAC?$AAr?$AAe?$AAa?$AAt?$AAe?$AAL?$AAo?$AAo?$AAp?$AAB?$AAa?$AAc?$AAk?$AAD?$AAl?$AAg?$AA?3?$AA?3?$AAF?$AAa?$AAl?$AAi?$AAe?$AAd?$AA?5?$AAt?$AAo?$AA?5?$AAR?$AAe?$AAg@ 000398f0     loopbackdlg.obj
 0002:0000b950       ??_C@_1BM@HGFEFMNP@?$AA?4?$AA?2?$AAm?$AAa?$AAi?$AAn?$AAf?$AAr?$AAm?$AA?4?$AAc?$AAp?$AAp?$AA?$AA@ 00039950     mainfrm.obj
 0002:0000b970       ??_C@_1EM@JIKJLGIF@?$AAC?$AAr?$AAe?$AAa?$AAt?$AAe?$AAM?$AAa?$AAi?$AAn?$AAM?$AAe?$AAn?$AAu?$AA?3?$AAS?$AAH?$AAC?$AAr?$AAe?$AAa?$AAt?$AAe?$AAM?$AAe?$AAn?$AAu?$AAB?$AAa?$AAr?$AA?5?$AAF@ 00039970     mainfrm.obj
 0002:0000b9c0       ??_C@_1FK@DLNKLABG@?$AAI?$AAn?$AAi?$AAt?$AAi?$AAa?$AAl?$AAi?$AAz?$AAe?$AAT?$AAa?$AAb?$AAF?$AAr?$AAo?$AAm?$AAI?$AAn?$AAd?$AAe?$AAx?$AA?5?$AA?3?$AA?5?$AAI?$AAn?$AAv?$AAa?$AAl?$AAi?$AAd@ 000399c0     mainfrm.obj
 0002:0000ba1c       ??_C@_1CM@CEIFGLCB@?$AAF?$AAa?$AAl?$AAi?$AAe?$AAd?$AA?5?$AAt?$AAo?$AA?5?$AAI?$AAo?$AAt?$AAa?$AA?5?$AAD?$AAi?$AAa?$AAl?$AAo?$AAg?$AA?$AA@ 00039a1c     mainfrm.obj
 0002:0000ba48       ??_C@_1DE@HNECOEIF@?$AAF?$AAa?$AAl?$AAi?$AAe?$AAd?$AA?5?$AAt?$AAo?$AA?5?$AAS?$AAI?$AAM?$AAP?$AAL?$AAE?$AAI?$AAP?$AA?5?$AAD?$AAi?$AAa?$AAl?$AAo?$AAg?$AA?$AA@ 00039a48     mainfrm.obj
 0002:0000ba7c       ??_C@_1DA@PACMLMPN@?$AAF?$AAa?$AAl?$AAi?$AAe?$AAd?$AA?5?$AAt?$AAo?$AA?5?$AAS?$AAy?$AAs?$AAt?$AAe?$AAm?$AA?5?$AAD?$AAi?$AAa?$AAl?$AAo?$AAg?$AA?$AA@ 00039a7c     mainfrm.obj
 0002:0000baac       ??_C@_1CK@CCGLFEMM@?$AAF?$AAa?$AAl?$AAi?$AAe?$AAd?$AA?5?$AAt?$AAo?$AA?5?$AAS?$AAI?$AAP?$AA?5?$AAD?$AAi?$AAa?$AAl?$AAo?$AAg?$AA?$AA@ 00039aac     mainfrm.obj
 0002:0000bad8       ??_C@_1DC@NKNPBGPN@?$AAF?$AAa?$AAl?$AAi?$AAe?$AAd?$AA?5?$AAt?$AAo?$AA?5?$AAB?$AAr?$AAo?$AAw?$AAs?$AAe?$AAr?$AA?5?$AAD?$AAi?$AAa?$AAl?$AAo?$AAg?$AA?$AA@ 00039ad8     mainfrm.obj
 0002:0000bb0c       ??_C@_1DE@MAJMPKEN@?$AAF?$AAa?$AAl?$AAi?$AAe?$AAd?$AA?5?$AAt?$AAo?$AA?5?$AAA?$AAd?$AAv?$AAa?$AAn?$AAc?$AAe?$AAd?$AA?5?$AAD?$AAi?$AAa?$AAl?$AAo?$AAg?$AA?$AA@ 00039b0c     mainfrm.obj
 0002:0000bb40       ??_C@_1DE@JMNEHPOM@?$AAF?$AAa?$AAl?$AAi?$AAe?$AAd?$AA?5?$AAt?$AAo?$AA?5?$AAL?$AAo?$AAo?$AAp?$AAB?$AAa?$AAc?$AAk?$AA?5?$AAD?$AAi?$AAa?$AAl?$AAo?$AAg?$AA?$AA@ 00039b40     mainfrm.obj
 0002:0000bb74       ??_C@_1DM@DPGIMNLL@?$AAF?$AAa?$AAl?$AAi?$AAe?$AAd?$AA?5?$AAt?$AAo?$AA?5?$AAP?$AAD?$AAP?$AA?1?$AAU?$AAS?$AAE?$AAR?$AAN?$AAA?$AAM?$AAE?$AA?5?$AAD?$AAi?$AAa?$AAl?$AAo?$AAg?$AA?$AA@ 00039b74     mainfrm.obj
 0002:0000bbb0       ??_C@_1DK@BAAFPOBI@?$AAF?$AAa?$AAl?$AAi?$AAe?$AAd?$AA?5?$AAt?$AAo?$AA?5?$AAV?$AAe?$AAr?$AAs?$AAi?$AAo?$AAn?$AAI?$AAn?$AAf?$AAo?$AA?5?$AAD?$AAi?$AAa?$AAl?$AAo?$AAg?$AA?$AA@ 00039bb0     mainfrm.obj
 0002:0000bbec       ??_C@_1CM@JPCPIGJH@?$AAF?$AAa?$AAl?$AAi?$AAe?$AAd?$AA?5?$AAt?$AAo?$AA?5?$AAe?$AAv?$AAd?$AAo?$AA?5?$AAD?$AAi?$AAa?$AAl?$AAo?$AAg?$AA?$AA@ 00039bec     mainfrm.obj
 0002:0000bc18       ??_C@_1GK@GFNCOGAN@?$AAU?$AAn?$AAa?$AAb?$AAl?$AAe?$AA?5?$AAt?$AAo?$AA?5?$AAp?$AAr?$AAo?$AAc?$AAe?$AAs?$AAs?$AA?5?$AAt?$AAh?$AAe?$AA?5?$AA?$CD?$AA?$CD?$AAM?$AAS?$AAL?$AA?5?$AAd?$AAu?$AAe?$AA?5@ 00039c18     mainfrm.obj
 0002:0000bc88       ??_C@_1EE@LOGIOJMG@?$AAF?$AAa?$AAl?$AAi?$AAe?$AAd?$AA?5?$AAt?$AAo?$AA?5?$AAO?$AAT?$AAK?$AAS?$AAL?$AA?1?$AAA?$AAC?$AAT?$AAI?$AAV?$AAA?$AAT?$AAI?$AAO?$AAN?$AA?5?$AAD?$AAi?$AAa?$AAl?$AAo@ 00039c88     mainfrm.obj
 0002:0000bcd0       ??_C@_1EA@KPECMNLE@?$AAF?$AAa?$AAl?$AAi?$AAe?$AAd?$AA?5?$AAt?$AAo?$AA?5?$AAM?$AAS?$AAL?$AA?1?$AAA?$AAC?$AAT?$AAI?$AAV?$AAA?$AAT?$AAI?$AAO?$AAN?$AA?5?$AAD?$AAi?$AAa?$AAl?$AAo?$AAg?$AA?$AA@ 00039cd0     mainfrm.obj
 0002:0000bd10       ??_C@_1DA@HNKOCILK@?$AAF?$AAa?$AAl?$AAi?$AAe?$AAd?$AA?5?$AAt?$AAo?$AA?5?$AAC?$AAo?$AAn?$AAf?$AAi?$AAg?$AA?5?$AAD?$AAi?$AAa?$AAl?$AAo?$AAg?$AA?$AA@ 00039d10     mainfrm.obj
 0002:0000bd40       ??_C@_1DC@FENHBKGO@?$AAF?$AAa?$AAl?$AAi?$AAe?$AAd?$AA?5?$AAt?$AAo?$AA?5?$AAV?$AAo?$AAc?$AAo?$AAd?$AAe?$AAr?$AA?5?$AAD?$AAi?$AAa?$AAl?$AAo?$AAg?$AA?$AA@ 00039d40     mainfrm.obj
 0002:0000bd74       ??_C@_1DE@ENCOLEM@?$AAF?$AAa?$AAl?$AAi?$AAe?$AAd?$AA?5?$AAt?$AAo?$AA?5?$AAP?$AAA?$AAS?$AAS?$AAT?$AAH?$AAR?$AAU?$AA?5?$AAD?$AAi?$AAa?$AAl?$AAo?$AAg?$AA?$AA@ 00039d74     mainfrm.obj
 0002:0000bda8       ??_C@_1CK@FEFKNDBF@?$AAF?$AAa?$AAl?$AAi?$AAe?$AAd?$AA?5?$AAt?$AAo?$AA?5?$AAR?$AAT?$AAN?$AA?5?$AAD?$AAi?$AAa?$AAl?$AAo?$AAg?$AA?$AA@ 00039da8     mainfrm.obj
 0002:0000bdd4       ??_C@_1CM@BGHKKGOI@?$AAF?$AAa?$AAl?$AAi?$AAe?$AAd?$AA?5?$AAt?$AAo?$AA?5?$AAA?$AAk?$AAe?$AAy?$AA?5?$AAD?$AAi?$AAa?$AAl?$AAo?$AAg?$AA?$AA@ 00039dd4     mainfrm.obj
 0002:0000be00       ??_C@_1DA@ELFFJILG@?$AAF?$AAa?$AAl?$AAi?$AAe?$AAd?$AA?5?$AAt?$AAo?$AA?5?$AAF?$AAi?$AAn?$AAg?$AAe?$AAr?$AA?5?$AAD?$AAi?$AAa?$AAl?$AAo?$AAg?$AA?$AA@ 00039e00     mainfrm.obj
 0002:0000be30       ??_C@_1FA@LIOLKHM@?$AAF?$AAa?$AAl?$AAi?$AAe?$AAd?$AA?5?$AAt?$AAo?$AA?5?$AAc?$AAr?$AAe?$AAa?$AAt?$AAe?$AA?5?$AAb?$AAa?$AAn?$AAd?$AAw?$AAi?$AAd?$AAt?$AAh?$AA?5?$AAm?$AAe?$AAt?$AAe?$AAr@ 00039e30     mainfrm.obj
 0002:0000be80       ??_C@_1EC@BMJOKJJN@?$AAF?$AAa?$AAl?$AAi?$AAe?$AAd?$AA?5?$AAt?$AAo?$AA?5?$AAc?$AAr?$AAe?$AAa?$AAt?$AAe?$AA?5?$AAG?$AAP?$AAS?$AA?5?$AAD?$AAa?$AAt?$AAa?$AA?5?$AAD?$AAi?$AAa?$AAl?$AAo?$AAg@ 00039e80     mainfrm.obj
 0002:0000bec8       ??_C@_1EK@LBBIMDJH@?$AAF?$AAa?$AAl?$AAi?$AAe?$AAd?$AA?5?$AAt?$AAo?$AA?5?$AAc?$AAr?$AAe?$AAa?$AAt?$AAe?$AA?5?$AAG?$AAP?$AAS?$AA?5?$AAs?$AAe?$AAt?$AAt?$AAi?$AAn?$AAg?$AAs?$AA?5?$AAD?$AAi@ 00039ec8     mainfrm.obj
 0002:0000bf14       ??_C@_1DC@JKGHILGB@?$AAF?$AAa?$AAl?$AAi?$AAe?$AAd?$AA?5?$AAt?$AAo?$AA?5?$AAN?$AAe?$AAt?$AAw?$AAo?$AAr?$AAk?$AA?5?$AAD?$AAi?$AAa?$AAl?$AAo?$AAg?$AA?$AA@ 00039f14     mainfrm.obj
 0002:0000bf48       ??_C@_1CM@DGANOIML@?$AAF?$AAa?$AAl?$AAi?$AAe?$AAd?$AA?5?$AAt?$AAo?$AA?5?$AAB?$AAa?$AAn?$AAd?$AA?5?$AAD?$AAi?$AAa?$AAl?$AAo?$AAg?$AA?$AA@ 00039f48     mainfrm.obj
 0002:0000bf74       ??_C@_1DA@OAFJLBEN@?$AAF?$AAa?$AAl?$AAi?$AAe?$AAd?$AA?5?$AAt?$AAo?$AA?5?$AAG?$AAS?$AAM?$AA?5?$AA3?$AAG?$AA?5?$AAD?$AAi?$AAa?$AAl?$AAo?$AAg?$AA?$AA@ 00039f74     mainfrm.obj
 0002:0000bfa4       ??_C@_1DA@IFDOIKAL@?$AAF?$AAa?$AAl?$AAi?$AAe?$AAd?$AA?5?$AAt?$AAo?$AA?5?$AAG?$AAS?$AAM?$AA?5?$AA2?$AAG?$AA?5?$AAD?$AAi?$AAa?$AAl?$AAo?$AAg?$AA?$AA@ 00039fa4     mainfrm.obj
 0002:0000bfd8       ??_C@_1EE@CLEKMAEK@?$AA?5?$AA?$CL?$AA?$CL?$AA?5?$AAI?$AAn?$AAi?$AAt?$AAi?$AAa?$AAl?$AAi?$AAz?$AAe?$AAT?$AAa?$AAb?$AAF?$AAr?$AAo?$AAm?$AAI?$AAn?$AAd?$AAe?$AAx?$AA?5?$AA?$DN?$AA?5?$AA?$CF?$AAd?$AA?$AN@ 00039fd8     mainfrm.obj
 0002:0000c01c       ??_C@_1DG@FPECGFEO@?$AAF?$AAa?$AAl?$AAi?$AAe?$AAd?$AA?5?$AAt?$AAo?$AA?5?$AAc?$AAr?$AAe?$AAa?$AAt?$AAe?$AA?5?$AAL?$AAi?$AAs?$AAt?$AA?5?$AAv?$AAi?$AAe?$AAw?$AA?$AA@ 0003a01c     mainfrm.obj
 0002:0000c058       ??_C@_1EA@PCKDKLLN@?$AA?5?$AA?$CL?$AA?$CL?$AA?5?$AAP?$AAr?$AAe?$AAp?$AAa?$AAr?$AAe?$AAR?$AAe?$AAs?$AAo?$AAu?$AAr?$AAc?$AAe?$AAD?$AAi?$AAa?$AAl?$AAg?$AA?5?$AA?$DN?$AA?5?$AA?$CF?$AAd?$AA?$AN?$AA?6?$AA?$AA@ 0003a058     mainfrm.obj
 0002:0000c098       ??_C@_1EE@GLNGELBC@?$AAI?$AAn?$AAi?$AAt?$AAi?$AAa?$AAl?$AAi?$AAz?$AAe?$AAT?$AAa?$AAb?$AAF?$AAr?$AAo?$AAm?$AAI?$AAn?$AAd?$AAe?$AAx?$AA?5?$AAF?$AAa?$AAi?$AAl?$AAe?$AAd?$AA?5?$AAD?$AAl@ 0003a098     mainfrm.obj
 0002:0000c0dc       ??_C@_1DM@DFGDONGN@?$AAI?$AAn?$AAi?$AAt?$AAi?$AAa?$AAl?$AAi?$AAz?$AAe?$AAT?$AAa?$AAb?$AAF?$AAr?$AAo?$AAm?$AAI?$AAn?$AAd?$AAe?$AAx?$AA?5?$AAF?$AAa?$AAl?$AAi?$AAe?$AAd?$AA?$AA@ 0003a0dc     mainfrm.obj
 0002:0000c118       ??_C@_1DM@KBHDPEHP@?$AA?5?$AA?$CL?$AA?$CL?$AA?5?$AAP?$AAr?$AAe?$AAp?$AAa?$AAr?$AAe?$AAR?$AAe?$AAs?$AAo?$AAu?$AAr?$AAc?$AAe?$AAD?$AAl?$AAg?$AA?5?$AA?$DN?$AA?5?$AA?$CF?$AAd?$AA?$AN?$AA?6?$AA?$AA@ 0003a118     mainfrm.obj
 0002:0000c154       ??_C@_1DC@KFKNNIJM@?$AAF?$AAa?$AAi?$AAl?$AAe?$AAd?$AA?5?$AAt?$AAo?$AA?5?$AAC?$AAr?$AAe?$AAa?$AAt?$AAe?$AAM?$AAa?$AAi?$AAn?$AAM?$AAe?$AAn?$AAu?$AA?$AA@ 0003a154     mainfrm.obj
 0002:0000c188       ??_C@_1DE@IPCGKLIO@?$AAF?$AAa?$AAi?$AAl?$AAe?$AAd?$AA?5?$AAt?$AAo?$AA?5?$AAO?$AAn?$AAC?$AAr?$AAe?$AAa?$AAt?$AAe?$AAM?$AAa?$AAi?$AAn?$AAW?$AAn?$AAd?$AA?$AA@ 0003a188     mainfrm.obj
 0002:0000c1c0       ??_C@_1GO@MDLJMJNA@?$AAI?$AAg?$AAn?$AAo?$AAr?$AAe?$AAd?$AA?5?$AAP?$AAH?$AAO?$AAN?$AAE?$AAU?$AAT?$AAI?$AAL?$AAS?$AA_?$AAB?$AAE?$AAG?$AAI?$AAN?$AA_?$AAN?$AAA?$AAC?$AAK?$AA?5?$AAt?$AAo@ 0003a1c0     mainfrm.obj
 0002:0000c230       ??_C@_1DE@MJAMAFPL@?$AAP?$AAr?$AAe?$AAp?$AAa?$AAr?$AAe?$AAR?$AAe?$AAs?$AAo?$AAu?$AAr?$AAc?$AAe?$AAD?$AAl?$AAg?$AA?5?$AAF?$AAa?$AAi?$AAl?$AAe?$AAd?$AA?$AA@ 0003a230     mainfrm.obj
 0002:0000c264       ??_C@_1DI@ILPHEIEJ@?$AAF?$AAa?$AAi?$AAl?$AAe?$AAd?$AA?5?$AAt?$AAo?$AA?5?$AAR?$AAe?$AAg?$AAi?$AAs?$AAt?$AAe?$AAr?$AAC?$AAl?$AAa?$AAs?$AAs?$AA?5?$AA?$CF?$AAd?$AA?0?$AA?$AA@ 0003a264     mainfrm.obj
 0002:0000c2a0       ??_C@_1EE@BABHFJEK@?$AAC?$AAr?$AAe?$AAa?$AAt?$AAe?$AAW?$AAi?$AAn?$AAd?$AAo?$AAw?$AA?5?$AAf?$AAa?$AAi?$AAl?$AAe?$AAd?$AA?5?$AAw?$AAi?$AAt?$AAh?$AA?5?$AAe?$AAr?$AAr?$AAo?$AAr?$AA?5?$AA?$CF@ 0003a2a0     mainfrm.obj
 0002:0000c2e4       ??_C@_1BI@MMKNBOFJ@?$AAM?$AAs?$AAl?$AAD?$AAl?$AAg?$AAC?$AAl?$AAa?$AAs?$AAs?$AA?$AA@ 0003a2e4     msldlg.obj
 0002:0000c2fc       ??_C@_19FCOLCMFM@?$AA0?$AAx?$AA?$CF?$AAX?$AA?$AA@ 0003a2fc     msldlg.obj
 0002:0000c308       ??_C@_1BM@CMGDHIJB@?$AAG?$AAe?$AAt?$AAM?$AAS?$AAL?$AA?5?$AAf?$AAa?$AAi?$AAl?$AAe?$AAd?$AA?$AA@ 0003a308     msldlg.obj
 0002:0000c328       ??_C@_1EA@MBBPAICF@?$AAI?$AAn?$AAi?$AAt?$AAM?$AAs?$AAl?$AAD?$AAl?$AAg?$AA?3?$AA?3?$AAS?$AAH?$AAI?$AAn?$AAi?$AAt?$AAD?$AAi?$AAa?$AAl?$AAo?$AAg?$AA?5?$AAF?$AAa?$AAl?$AAi?$AAe?$AAd?$AA?$AA@ 0003a328     msldlg.obj
 0002:0000c368       ??_C@_1DO@MBODPEKD@?$AAI?$AAn?$AAi?$AAt?$AAM?$AAs?$AAl?$AAD?$AAl?$AAg?$AA?3?$AAS?$AAH?$AAI?$AAn?$AAi?$AAt?$AAD?$AAi?$AAa?$AAl?$AAo?$AAg?$AA?5?$AAF?$AAa?$AAi?$AAl?$AAe?$AAd?$AA?$AA@ 0003a368     msldlg.obj
 0002:0000c3a8       ??_C@_1EG@HKLMEBLP@?$AAI?$AAn?$AAi?$AAt?$AAM?$AAs?$AAl?$AAD?$AAl?$AAg?$AA?3?$AA?3?$AAS?$AAH?$AAC?$AAr?$AAe?$AAa?$AAt?$AAe?$AAM?$AAe?$AAn?$AAu?$AAB?$AAa?$AAr?$AA?5?$AAF?$AAa?$AAl?$AAi@ 0003a3a8     msldlg.obj
 0002:0000c3f0       ??_C@_1BK@ELAICJB@?$AA?4?$AA?2?$AAm?$AAs?$AAl?$AAd?$AAl?$AAg?$AA?4?$AAc?$AAp?$AAp?$AA?$AA@ 0003a3f0     msldlg.obj
 0002:0000c410       ??_C@_1EE@KDBCNEGC@?$AAI?$AAn?$AAi?$AAt?$AAM?$AAs?$AAl?$AAD?$AAl?$AAg?$AA?3?$AAS?$AAH?$AAC?$AAr?$AAe?$AAa?$AAt?$AAe?$AAM?$AAe?$AAn?$AAu?$AAB?$AAa?$AAr?$AA?5?$AAF?$AAa?$AAi?$AAl?$AAe@ 0003a410     msldlg.obj
 0002:0000c454       ??_C@_1CE@LPDCKFFN@?$AAI?$AAn?$AAi?$AAt?$AAM?$AAs?$AAl?$AAD?$AAl?$AAg?$AA?5?$AAF?$AAa?$AAi?$AAl?$AAe?$AAd?$AA?$AA@ 0003a454     msldlg.obj
 0002:0000c478       ??_C@_1FE@CPNCHBHB@?$AAC?$AAr?$AAe?$AAa?$AAt?$AAe?$AAM?$AAs?$AAl?$AAD?$AAl?$AAg?$AA?3?$AA?3?$AAF?$AAa?$AAl?$AAi?$AAe?$AAd?$AA?5?$AAt?$AAo?$AA?5?$AAC?$AAr?$AAe?$AAa?$AAt?$AAe?$AA?5?$AAD@ 0003a478     msldlg.obj
 0002:0000c4d0       ??_C@_1FE@KBBIPBLL@?$AAC?$AAr?$AAe?$AAa?$AAt?$AAe?$AAM?$AAs?$AAl?$AAD?$AAl?$AAg?$AA?3?$AA?3?$AAF?$AAa?$AAl?$AAi?$AAe?$AAd?$AA?5?$AAt?$AAo?$AA?5?$AAR?$AAe?$AAg?$AAi?$AAs?$AAt?$AAe?$AAr@ 0003a4d0     msldlg.obj
 0002:0000c524       ??_C@_1CA@DDPFDONA@?$AAN?$AAe?$AAt?$AAw?$AAo?$AAr?$AAk?$AAD?$AAl?$AAg?$AAC?$AAl?$AAa?$AAs?$AAs?$AA?$AA@ 0003a524     network.obj
 0002:0000c5a4       ??_C@_1BE@JBHONDLM@?$AAR?$AAe?$AAs?$AAe?$AAt?$AAt?$AAi?$AAn?$AAg?$AA?$AA@ 0003a5a4     network.obj
 0002:0000c5b8       ??_C@_1BA@DKNJBOGI@?$AAO?$AAf?$AAf?$AAl?$AAi?$AAn?$AAe?$AA?$AA@ 0003a5b8     network.obj
 0002:0000c5c8       ??_C@_1BA@LEPJIIOK@?$AAU?$AAn?$AAk?$AAn?$AAo?$AAw?$AAn?$AA?$AA@ 0003a5c8     network.obj
 0002:0000c5d8       ??_C@_19FJLFNNLC@?$AAI?$AAd?$AAl?$AAe?$AA?$AA@ 0003a5d8     network.obj
 0002:0000c5e4       ??_C@_1BG@NGOJCIFJ@?$AA?$CF?$AAs?$AA?5?$AA?$CI?$AA0?$AAx?$AA?$CF?$AA4?$AAx?$AA?$CJ?$AA?$AA@ 0003a5e4     network.obj
 0002:0000c600       ??_C@_1EC@BCCEMHHB@?$AAI?$AAn?$AAi?$AAt?$AAN?$AAe?$AAt?$AAw?$AAo?$AAr?$AAk?$AA?3?$AA?3?$AAS?$AAH?$AAI?$AAn?$AAi?$AAt?$AAD?$AAi?$AAa?$AAl?$AAo?$AAg?$AA?5?$AAF?$AAa?$AAl?$AAi?$AAe?$AAd@ 0003a600     network.obj
 0002:0000c648       ??_C@_1EA@ECMPLDCD@?$AAI?$AAn?$AAi?$AAt?$AAN?$AAe?$AAt?$AAw?$AAo?$AAr?$AAk?$AA?3?$AAS?$AAH?$AAI?$AAn?$AAi?$AAt?$AAD?$AAi?$AAa?$AAl?$AAo?$AAg?$AA?5?$AAF?$AAa?$AAi?$AAl?$AAe?$AAd?$AA?$AA@ 0003a648     network.obj
 0002:0000c688       ??_C@_1EI@COADIAJN@?$AAI?$AAn?$AAi?$AAt?$AAN?$AAe?$AAt?$AAw?$AAo?$AAr?$AAk?$AA?3?$AA?3?$AAS?$AAH?$AAC?$AAr?$AAe?$AAa?$AAt?$AAe?$AAM?$AAe?$AAn?$AAu?$AAB?$AAa?$AAr?$AA?5?$AAF?$AAa?$AAl@ 0003a688     network.obj
 0002:0000c6d0       ??_C@_1BM@MAJKCELE@?$AA?4?$AA?2?$AAn?$AAe?$AAt?$AAw?$AAo?$AAr?$AAk?$AA?4?$AAc?$AAp?$AAp?$AA?$AA@ 0003a6d0     network.obj
 0002:0000c6f0       ??_C@_1EG@FOOGPBLM@?$AAI?$AAn?$AAi?$AAt?$AAN?$AAe?$AAt?$AAw?$AAo?$AAr?$AAk?$AA?3?$AAS?$AAH?$AAC?$AAr?$AAe?$AAa?$AAt?$AAe?$AAM?$AAe?$AAn?$AAu?$AAB?$AAa?$AAr?$AA?5?$AAF?$AAa?$AAi?$AAl@ 0003a6f0     network.obj
 0002:0000c738       ??_C@_1BI@JKEPHKPE@?$AAP?$AAr?$AAo?$AAv?$AAi?$AAs?$AAi?$AAo?$AAn?$AAe?$AAd?$AA?$AA@ 0003a738     network.obj
 0002:0000c750       ??_C@_1CA@ECGKDFDH@?$AAN?$AAo?$AAt?$AA?5?$AAP?$AAr?$AAo?$AAv?$AAi?$AAs?$AAi?$AAo?$AAn?$AAe?$AAd?$AA?$AA@ 0003a750     network.obj
 0002:0000c770       ??_C@_19PCNJIDGC@?$AA0?$AAx?$AA?$CF?$AAx?$AA?$AA@ 0003a770     network.obj
 0002:0000c77c       ??_C@_1BA@GEIAOBPM@?$AA0?$AAx?$AA?$CF?$AAx?$AA?3?$AA?$CF?$AAs?$AA?$AA@ 0003a77c     network.obj
 0002:0000c78c       ??_C@_1BI@IONHJEKN@?$AA?$CF?$AAi?$AA?$LA?$AAc?$AA?1?$AA?$CF?$AA?4?$AA1?$AAf?$AA?$LA?$AAf?$AA?$AA@ 0003a78c     network.obj
 0002:0000c7a4       ??_C@_1BC@DKLGNPOA@?$AA?$CF?$AAd?$AA?3?$AA?$CF?$AAu?$AA?3?$AA?$CF?$AAu?$AA?$AA@ 0003a7a4     network.obj
 0002:0000c7b8       ??_C@_1O@MCOKPIKF@?$AA?$CF?$AA?4?$AA2?$AAf?$AA?$CF?$AAs?$AA?$AA@ 0003a7b8     network.obj
 0002:0000c7c8       ??_C@_1BC@LBCAEGK@?$AA?$CF?$AA?4?$AA2?$AAf?$AA?5?$AAd?$AAB?$AAm?$AA?$AA@ 0003a7c8     network.obj
 0002:0000c7dc       ??_C@_17BLILKDMA@?$AA?9?$AA?$CF?$AAd?$AA?$AA@ 0003a7dc     network.obj
 0002:0000c7e4       ??_C@_1BA@PPICOFGE@?$AA?9?$AA?$CF?$AAd?$AA?5?$AAd?$AAB?$AAm?$AA?$AA@ 0003a7e4     network.obj
 0002:0000c7f4       ??_C@_1CG@CCFGJJAO@?$AAI?$AAn?$AAi?$AAt?$AAN?$AAe?$AAt?$AAw?$AAo?$AAr?$AAk?$AA?5?$AAF?$AAa?$AAi?$AAl?$AAe?$AAd?$AA?$AA@ 0003a7f4     network.obj
 0002:0000c820       ??_C@_1FM@LAJIFOAN@?$AAC?$AAr?$AAe?$AAa?$AAt?$AAe?$AAN?$AAe?$AAt?$AAw?$AAo?$AAr?$AAk?$AAD?$AAl?$AAg?$AA?3?$AA?3?$AAF?$AAa?$AAl?$AAi?$AAe?$AAd?$AA?5?$AAt?$AAo?$AA?5?$AAR?$AAe?$AAg?$AAi@ 0003a820     network.obj
 0002:0000c87c       ??_C@_1BM@OOHEJHF@?$AAO?$AAt?$AAk?$AAs?$AAl?$AAD?$AAl?$AAg?$AAC?$AAl?$AAa?$AAs?$AAs?$AA?$AA@ 0003a87c     otksldlg.obj
 0002:0000c898       ??_C@_1EE@IAAFLBAA@?$AAI?$AAn?$AAi?$AAt?$AAO?$AAt?$AAk?$AAs?$AAl?$AAD?$AAl?$AAg?$AA?3?$AA?3?$AAS?$AAH?$AAI?$AAn?$AAi?$AAt?$AAD?$AAi?$AAa?$AAl?$AAo?$AAg?$AA?5?$AAF?$AAa?$AAl?$AAi?$AAe@ 0003a898     otksldlg.obj
 0002:0000c8e0       ??_C@_1EC@DFEDHDB@?$AAI?$AAn?$AAi?$AAt?$AAO?$AAt?$AAk?$AAs?$AAl?$AAD?$AAl?$AAg?$AA?3?$AAS?$AAH?$AAI?$AAn?$AAi?$AAt?$AAD?$AAi?$AAa?$AAl?$AAo?$AAg?$AA?5?$AAF?$AAa?$AAi?$AAl?$AAe?$AAd@ 0003a8e0     otksldlg.obj
 0002:0000c928       ??_C@_1EK@HOPGOPFD@?$AAI?$AAn?$AAi?$AAt?$AAO?$AAt?$AAk?$AAs?$AAl?$AAD?$AAl?$AAg?$AA?3?$AA?3?$AAS?$AAH?$AAC?$AAr?$AAe?$AAa?$AAt?$AAe?$AAM?$AAe?$AAn?$AAu?$AAB?$AAa?$AAr?$AA?5?$AAF?$AAa@ 0003a928     otksldlg.obj
 0002:0000c974       ??_C@_1BO@PLABPNNP@?$AA?4?$AA?2?$AAo?$AAt?$AAk?$AAs?$AAl?$AAd?$AAl?$AAg?$AA?4?$AAc?$AAp?$AAp?$AA?$AA@ 0003a974     otksldlg.obj
 0002:0000c998       ??_C@_1EI@EPIHMFCM@?$AAI?$AAn?$AAi?$AAt?$AAO?$AAt?$AAk?$AAs?$AAl?$AAD?$AAl?$AAg?$AA?3?$AAS?$AAH?$AAC?$AAr?$AAe?$AAa?$AAt?$AAe?$AAM?$AAe?$AAn?$AAu?$AAB?$AAa?$AAr?$AA?5?$AAF?$AAa?$AAi@ 0003a998     otksldlg.obj
 0002:0000c9e0       ??_C@_1CI@GBAAHGIL@?$AAI?$AAn?$AAi?$AAt?$AAO?$AAt?$AAk?$AAs?$AAl?$AAD?$AAl?$AAg?$AA?5?$AAF?$AAa?$AAi?$AAl?$AAe?$AAd?$AA?$AA@ 0003a9e0     otksldlg.obj
 0002:0000ca08       ??_C@_1FI@BGHFLMGB@?$AAC?$AAr?$AAe?$AAa?$AAt?$AAe?$AAO?$AAt?$AAk?$AAs?$AAl?$AAD?$AAl?$AAg?$AA?3?$AA?3?$AAF?$AAa?$AAl?$AAi?$AAe?$AAd?$AA?5?$AAt?$AAo?$AA?5?$AAC?$AAr?$AAe?$AAa?$AAt?$AAe@ 0003aa08     otksldlg.obj
 0002:0000ca60       ??_C@_1FI@JILPDMKL@?$AAC?$AAr?$AAe?$AAa?$AAt?$AAe?$AAO?$AAt?$AAk?$AAs?$AAl?$AAD?$AAl?$AAg?$AA?3?$AA?3?$AAF?$AAa?$AAl?$AAi?$AAe?$AAd?$AA?5?$AAt?$AAo?$AA?5?$AAR?$AAe?$AAg?$AAi?$AAs?$AAt@ 0003aa60     otksldlg.obj
 0002:0000cab8       ??_C@_1CC@PBNAIMHG@?$AAP?$AAa?$AAs?$AAs?$AAT?$AAh?$AAr?$AAu?$AAD?$AAl?$AAg?$AAC?$AAl?$AAa?$AAs?$AAs?$AA?$AA@ 0003aab8     passthrudlg.obj
 0002:0000cae0       ??_C@_1FO@OGJPLGMA@?$AAI?$AAn?$AAi?$AAt?$AAi?$AAa?$AAl?$AAi?$AAz?$AAe?$AAP?$AAa?$AAs?$AAs?$AAT?$AAh?$AAr?$AAu?$AAD?$AAl?$AAg?$AA?3?$AAA?$AAl?$AAr?$AAe?$AAa?$AAd?$AAy?$AA?5?$AAi?$AAn@ 0003aae0     passthrudlg.obj
 0002:0000cb40       ??_C@_1FC@MAEJIIEL@?$AAI?$AAn?$AAi?$AAt?$AAi?$AAa?$AAl?$AAi?$AAz?$AAe?$AAP?$AAa?$AAs?$AAs?$AAT?$AAh?$AAr?$AAu?$AAD?$AAl?$AAg?$AA?3?$AAA?$AAl?$AAr?$AAe?$AAa?$AAd?$AAy?$AA?5?$AAi?$AAn@ 0003ab40     passthrudlg.obj
 0002:0000cb98       ??_C@_1FO@JHMANNHD@?$AAI?$AAn?$AAi?$AAt?$AAi?$AAa?$AAl?$AAi?$AAz?$AAe?$AAP?$AAa?$AAs?$AAs?$AAT?$AAh?$AAr?$AAu?$AAD?$AAl?$AAg?$AA?3?$AAC?$AAa?$AAn?$AAn?$AAo?$AAt?$AA?5?$AAd?$AAe?$AAt@ 0003ab98     passthrudlg.obj
 0002:0000cbf8       ??_C@_1CE@EIHGICIP@?$AA?4?$AA?2?$AAp?$AAa?$AAs?$AAs?$AAt?$AAh?$AAr?$AAu?$AAd?$AAl?$AAg?$AA?4?$AAc?$AAp?$AAp?$AA?$AA@ 0003abf8     passthrudlg.obj
 0002:0000cc20       ??_C@_1FO@GNDCGMEG@?$AAI?$AAn?$AAi?$AAt?$AAi?$AAa?$AAl?$AAi?$AAz?$AAe?$AAP?$AAa?$AAs?$AAs?$AAT?$AAh?$AAr?$AAu?$AAD?$AAl?$AAg?$AA?3?$AAC?$AAa?$AAn?$AAn?$AAo?$AAt?$AA?5?$AAd?$AAe?$AAt@ 0003ac20     passthrudlg.obj
 0002:0000cc80       ??_C@_1EK@KBCOHDIK@?$AAI?$AAn?$AAi?$AAt?$AAP?$AAa?$AAs?$AAs?$AAT?$AAh?$AAr?$AAu?$AAD?$AAl?$AAg?$AA?3?$AA?3?$AAS?$AAH?$AAI?$AAn?$AAi?$AAt?$AAD?$AAi?$AAa?$AAl?$AAo?$AAg?$AA?5?$AAF?$AAa@ 0003ac80     passthrudlg.obj
 0002:0000ccd0       ??_C@_1EI@IKIPKGHH@?$AAI?$AAn?$AAi?$AAt?$AAP?$AAa?$AAs?$AAs?$AAT?$AAh?$AAr?$AAu?$AAD?$AAl?$AAg?$AA?3?$AAS?$AAH?$AAI?$AAn?$AAi?$AAt?$AAD?$AAi?$AAa?$AAl?$AAo?$AAg?$AA?5?$AAF?$AAa?$AAi@ 0003acd0     passthrudlg.obj
 0002:0000cd18       ??_C@_1FA@BMLEGHLO@?$AAI?$AAn?$AAi?$AAt?$AAP?$AAa?$AAs?$AAs?$AAT?$AAh?$AAr?$AAu?$AAD?$AAl?$AAg?$AA?3?$AA?3?$AAS?$AAH?$AAC?$AAr?$AAe?$AAa?$AAt?$AAe?$AAM?$AAe?$AAn?$AAu?$AAB?$AAa?$AAr@ 0003ad18     passthrudlg.obj
 0002:0000cd68       ??_C@_1EO@GFFBDMGK@?$AAI?$AAn?$AAi?$AAt?$AAP?$AAa?$AAs?$AAs?$AAT?$AAh?$AAr?$AAu?$AAD?$AAl?$AAg?$AA?3?$AAS?$AAH?$AAC?$AAr?$AAe?$AAa?$AAt?$AAe?$AAM?$AAe?$AAn?$AAu?$AAB?$AAa?$AAr?$AA?5@ 0003ad68     passthrudlg.obj
 0002:0000cdb8       ??_C@_1CO@BHMNOOJB@?$AAI?$AAn?$AAi?$AAt?$AAP?$AAa?$AAs?$AAs?$AAT?$AAh?$AAr?$AAu?$AAD?$AAl?$AAg?$AA?5?$AAF?$AAa?$AAi?$AAl?$AAe?$AAd?$AA?$AA@ 0003adb8     passthrudlg.obj
 0002:0000cde8       ??_C@_1CG@LFCPILJH@?$AAS?$AAt?$AAa?$AAr?$AAt?$AAP?$AAT?$AAM?$AAo?$AAd?$AAe?$AA?5?$AAF?$AAa?$AAi?$AAl?$AAe?$AAd?$AA?$AA@ 0003ade8     passthrudlg.obj
 0002:0000ce10       ??_C@_1CG@LAMBHOGA@?$AAS?$AAt?$AAa?$AAr?$AAt?$AAD?$AAM?$AAM?$AAo?$AAd?$AAe?$AA?5?$AAF?$AAa?$AAi?$AAl?$AAe?$AAd?$AA?$AA@ 0003ae10     passthrudlg.obj
 0002:0000ce38       ??_C@_1CE@FNICLCEM@?$AAS?$AAt?$AAo?$AAp?$AAP?$AAT?$AAM?$AAo?$AAd?$AAe?$AA?5?$AAF?$AAa?$AAi?$AAl?$AAe?$AAd?$AA?$AA@ 0003ae38     passthrudlg.obj
 0002:0000ce5c       ??_C@_1CE@FIGMEHLL@?$AAS?$AAt?$AAo?$AAp?$AAD?$AAM?$AAM?$AAo?$AAd?$AAe?$AA?5?$AAF?$AAa?$AAi?$AAl?$AAe?$AAd?$AA?$AA@ 0003ae5c     passthrudlg.obj
 0002:0000ce80       ??_C@_1FO@KLGCIEFL@?$AAC?$AAr?$AAe?$AAa?$AAt?$AAe?$AAP?$AAa?$AAs?$AAs?$AAT?$AAh?$AAr?$AAu?$AAD?$AAl?$AAg?$AA?3?$AA?3?$AAF?$AAa?$AAl?$AAi?$AAe?$AAd?$AA?5?$AAt?$AAo?$AA?5?$AAC?$AAr?$AAe@ 0003ae80     passthrudlg.obj
 0002:0000cee0       ??_C@_1FO@CFKIAEJB@?$AAC?$AAr?$AAe?$AAa?$AAt?$AAe?$AAP?$AAa?$AAs?$AAs?$AAT?$AAh?$AAr?$AAu?$AAD?$AAl?$AAg?$AA?3?$AA?3?$AAF?$AAa?$AAl?$AAi?$AAe?$AAd?$AA?5?$AAt?$AAo?$AA?5?$AAR?$AAe?$AAg@ 0003aee0     passthrudlg.obj
 0002:0000cf40       ??_C@_1BA@MFHCPFOB@?$AA?$CD?$AA?$CD?$AA2?$AA5?$AA3?$AA2?$AA7?$AA?$AA@ 0003af40     phoneutility.obj
 0002:0000cf50       ??_C@_1BA@JLLAHGGB@?$AA?$CD?$AA?$CD?$AAC?$AAL?$AAE?$AAA?$AAR?$AA?$AA@ 0003af50     phoneutility.obj
 0002:0000cf60       ??_C@_1M@PNIOPAJC@?$AA?$CD?$AA?$CD?$AA7?$AA8?$AA6?$AA?$AA@ 0003af60     phoneutility.obj
 0002:0000cf6c       ??_C@_1M@LEDIBJBP@?$AA?$CD?$AA?$CD?$AAR?$AAT?$AAN?$AA?$AA@ 0003af6c     phoneutility.obj
 0002:0000cf78       ??_C@_1BE@FKAPHCCO@?$AA?$CD?$AA?$CD?$AA8?$AA6?$AA2?$AA6?$AA3?$AA3?$AA7?$AA?$AA@ 0003af78     phoneutility.obj
 0002:0000cf8c       ??_C@_1BE@MFFAFHKK@?$AA?$CD?$AA?$CD?$AAV?$AAO?$AAC?$AAO?$AAD?$AAE?$AAR?$AA?$AA@ 0003af8c     phoneutility.obj
 0002:0000cfa0       ??_C@_1BA@OOAADCOK@?$AA?$CD?$AA?$CD?$AA7?$AA4?$AA6?$AA6?$AA3?$AA?$AA@ 0003afa0     phoneutility.obj
 0002:0000cfb0       ??_C@_1BA@EEIFCICM@?$AA?$CD?$AA?$CD?$AAP?$AAH?$AAO?$AAN?$AAE?$AA?$AA@ 0003afb0     phoneutility.obj
 0002:0000cfc0       ??_C@_1O@GMJAKOC@?$AA?$CD?$AA?$CD?$AA3?$AA2?$AA8?$AA2?$AA?$AA@ 0003afc0     phoneutility.obj
 0002:0000cfd0       ??_C@_1O@DGDPMCCD@?$AA?$CD?$AA?$CD?$AAD?$AAA?$AAT?$AAA?$AA?$AA@ 0003afd0     phoneutility.obj
 0002:0000cfe0       ??_C@_1BE@KNFFNLGK@?$AA?$CD?$AA?$CD?$AA2?$AA8?$AA8?$AA4?$AA5?$AA3?$AA9?$AA?$AA@ 0003afe0     phoneutility.obj
 0002:0000cff4       ??_C@_1BE@POHGPNBB@?$AA?$CD?$AA?$CD?$AAA?$AAU?$AAT?$AAH?$AAK?$AAE?$AAY?$AA?$AA@ 0003aff4     phoneutility.obj
 0002:0000d008       ??_C@_1BG@FBJKOJDE@?$AA?$CD?$AA?$CD?$AA3?$AA3?$AA2?$AA8?$AA4?$AA8?$AA7?$AA8?$AA?$AA@ 0003b008     phoneutility.obj
 0002:0000d020       ??_C@_1BG@NBBGPNNO@?$AA?$CD?$AA?$CD?$AAD?$AAE?$AAB?$AAU?$AAG?$AAT?$AAS?$AAT?$AA?$AA@ 0003b020     phoneutility.obj
 0002:0000d038       ??_C@_1BA@CMENEFNP@?$AA?$CD?$AA?$CD?$AA3?$AA3?$AA2?$AA8?$AA4?$AA?$AA@ 0003b038     phoneutility.obj
 0002:0000d048       ??_C@_1BA@OGHIFKBN@?$AA?$CD?$AA?$CD?$AAD?$AAE?$AAB?$AAU?$AAG?$AA?$AA@ 0003b048     phoneutility.obj
 0002:0000d058       ??_C@_1BK@OJNJHOHE@?$AAP?$AAh?$AAo?$AAn?$AAe?$AAU?$AAt?$AAi?$AAl?$AAi?$AAt?$AAy?$AA?$AA@ 0003b058     phoneutility.obj
 0002:0000d0d8       ??_C@_1BC@JLHJOJGJ@?$AA?$CD?$AA?$CD?$AA7?$AA2?$AA7?$AA8?$AA6?$AA?$CD?$AA?$AA@ 0003b0d8     phoneutility.obj
 0002:0000d0ec       ??_C@_1CG@IBJEMLEC@?$AA?4?$AA?2?$AAp?$AAh?$AAo?$AAn?$AAe?$AAu?$AAt?$AAi?$AAl?$AAi?$AAt?$AAy?$AA?4?$AAc?$AAp?$AAp?$AA?$AA@ 0003b0ec     phoneutility.obj
 0002:0000d118       ??_C@_1FG@PDOPIELP@?$AAP?$AAo?$AAw?$AAe?$AAr?$AA?5?$AAs?$AAt?$AAa?$AAt?$AAe?$AA?5?$AAi?$AAs?$AA?5?$AA?$CF?$AAd?$AA?5?$AAc?$AAa?$AAn?$AA?5?$AAn?$AAo?$AAt?$AA?5?$AAr?$AAu?$AAn?$AA?5?$AAP?$AAh@ 0003b118     phoneutility.obj
 0002:0000d170       ??_C@_1CM@BJBCLOLP@?$AAS?$AAP?$AAC?$AA?5?$AAv?$AAa?$AAl?$AAi?$AAd?$AAa?$AAt?$AAi?$AAo?$AAn?$AA?5?$AAF?$AAa?$AAi?$AAl?$AAe?$AAd?$AA?$AA@ 0003b170     phoneutility.obj
 0002:0000d1a0       ??_C@_1EA@EIFDBHFG@?$AAU?$AAn?$AAa?$AAb?$AAl?$AAe?$AA?5?$AAt?$AAo?$AA?5?$AAc?$AAr?$AAe?$AAa?$AAt?$AAe?$AA?5?$AAt?$AAh?$AAe?$AA?5?$AAS?$AAP?$AAC?$AA?5?$AAd?$AAi?$AAa?$AAl?$AAo?$AAg?$AA?$AA@ 0003b1a0     phoneutility.obj
 0002:0000d1e0       ??_C@_1DM@NLDGHGHH@?$AAS?$AAw?$AAi?$AAG?$AAe?$AAt?$AAC?$AAd?$AAm?$AAa?$AAD?$AAo?$AAm?$AAi?$AAn?$AAa?$AAn?$AAt?$AAP?$AAn?$AA?5?$AAr?$AAe?$AAt?$AA?5?$AA?$DN?$AA?5?$AA?$CF?$AAd?$AA?$AA@ 0003b1e0     phoneutility.obj
 0002:0000d21c       ??_C@_1CI@PLJPFDGP@?$AAG?$AAe?$AAt?$AAE?$AAr?$AAr?$AAR?$AAa?$AAt?$AAe?$AA?5?$AAr?$AAe?$AAt?$AA?5?$AA?$DN?$AA?5?$AA?$CF?$AAd?$AA?$AA@ 0003b21c     phoneutility.obj
 0002:0000d248       ??_C@_1EE@KCIELDIB@?$AAS?$AAw?$AAi?$AAG?$AAe?$AAt?$AAS?$AAi?$AAg?$AAn?$AAa?$AAl?$AAS?$AAt?$AAr?$AAe?$AAn?$AAg?$AAt?$AAh?$AAI?$AAn?$AAf?$AAo?$AA?5?$AAr?$AAe?$AAt?$AA?5?$AA?$DN?$AA?5?$AA?$CF@ 0003b248     phoneutility.obj
 0002:0000d290       ??_C@_1EM@GANBBOHC@?$AAG?$AAe?$AAt?$AAA?$AAN?$AAA?$AAA?$AAA?$AAA?$AAu?$AAt?$AAh?$AAe?$AAn?$AAt?$AAi?$AAc?$AAa?$AAt?$AAi?$AAo?$AAn?$AAS?$AAt?$AAa?$AAt?$AAu?$AAs?$AA?5?$AAr?$AAe?$AAt@ 0003b290     phoneutility.obj
 0002:0000d2e0       ??_C@_1OO@MPMILFEH@?$AAD?$AAr?$AAc?$AAV?$AAa?$AAl?$AAu?$AAe?$AA?5?$AA?$DN?$AA?5?$AA?$CF?$AAd?$AA?0?$AA?5?$AAD?$AAr?$AAc?$AAC?$AAo?$AAv?$AAe?$AAr?$AA?5?$AA?$DN?$AA?5?$AA?$CF?$AAd?$AA?5?$AAA?$AAr?$AAr@ 0003b2e0     phoneutility.obj
 0002:0000d3d0       ??_C@_1DC@HDIAEHCP@?$AAS?$AAw?$AAi?$AAG?$AAe?$AAt?$AAH?$AAr?$AAp?$AAd?$AAS?$AAt?$AAa?$AAt?$AAs?$AA?5?$AAr?$AAe?$AAt?$AA?5?$AA?$DN?$AA?5?$AA?$CF?$AAd?$AA?$AA@ 0003b3d0     phoneutility.obj
 0002:0000d404       ??_C@_1DC@ICPFEEIA@?$AAG?$AAe?$AAt?$AAH?$AAd?$AAr?$AAC?$AAo?$AAl?$AAo?$AAr?$AAC?$AAo?$AAd?$AAe?$AA?5?$AAr?$AAe?$AAt?$AA?5?$AA?$DN?$AA?5?$AA?$CF?$AAd?$AA?$AA@ 0003b404     phoneutility.obj
 0002:0000d438       ??_C@_1CG@KJFGPEIH@?$AAG?$AAe?$AAt?$AAR?$AAF?$AAI?$AAn?$AAf?$AAo?$AA?5?$AAr?$AAe?$AAt?$AA?5?$AA?$DN?$AA?5?$AA?$CF?$AAd?$AA?$AA@ 0003b438     phoneutility.obj
 0002:0000d460       ??_C@_1CK@DAPDLPDM@?$AAC?$AAr?$AAe?$AAa?$AAt?$AAe?$AAM?$AAa?$AAi?$AAn?$AAW?$AAn?$AAd?$AA?5?$AAf?$AAa?$AAi?$AAl?$AAe?$AAd?$AA?$AA@ 0003b460     phoneutility.obj
 0002:0000d48c       ??_C@_1DO@PLLNPPOH@?$AAC?$AAh?$AAe?$AAc?$AAk?$AAP?$AAh?$AAo?$AAn?$AAe?$AAU?$AAt?$AAi?$AAl?$AAi?$AAt?$AAy?$AAC?$AAa?$AAn?$AAr?$AAu?$AAn?$AA?5?$AAf?$AAa?$AAi?$AAl?$AAe?$AAd?$AA?$AA@ 0003b48c     phoneutility.obj
 0002:0000d4cc       ??_C@_1CI@IKFHBAEG@?$AA_?$AAP?$AAV?$AAI?$AAE?$AAW?$AAC?$AAE?$AA_?$AAE?$AAX?$AAE?$AA_?$AAM?$AAU?$AAT?$AAE?$AAX?$AA_?$AA?$AA@ 0003b4cc     phoneutility.obj
 0002:0000d4f4       ??_C@_1DO@GNDAEGEA@?$AAL?$AAo?$AAa?$AAd?$AAL?$AAi?$AAb?$AAr?$AAa?$AAr?$AAy?$AA?5?$AA?$CF?$AAs?$AA?5?$AAf?$AAa?$AAi?$AAl?$AAe?$AAd?$AA?5?$AAe?$AAr?$AAr?$AAo?$AAr?$AA?5?$AA?$CF?$AAd?$AA?$AA@ 0003b4f4     phoneutility.obj
 0002:0000d534       ??_C@_1CA@MNHLNOBN@?$AAs?$AAw?$AAi?$AA_?$AAr?$AAi?$AAl?$AAr?$AAe?$AAs?$AAG?$AA?4?$AAd?$AAl?$AAl?$AA?$AA@ 0003b534     phoneutility.obj
 0002:0000d558       ??_C@_1EG@BCLEKMNG@?$AAI?$AAn?$AAv?$AAa?$AAl?$AAi?$AAd?$AA?5?$AAc?$AAo?$AAm?$AAm?$AAa?$AAn?$AAd?$AA?5?$AAl?$AAi?$AAn?$AAe?$AA?5?$AAa?$AAr?$AAg?$AAu?$AAm?$AAe?$AAn?$AAt?$AA?5?$AA?$DN?$AA?5@ 0003b558     phoneutility.obj
 0002:0000d5a0       ??_C@_1BI@GNKHOAKJ@?$AAR?$AAT?$AAN?$AAD?$AAl?$AAg?$AAC?$AAl?$AAa?$AAs?$AAs?$AA?$AA@ 0003b5a0     rtndlg.obj
 0002:0000d5b8       ??_C@_15BHOFONJE@?$AA?$CF?$AAX?$AA?$AA@ 0003b5b8     rtndlg.obj
 0002:0000d5c0       ??_C@_1BK@JFENBNIA@?$AA?4?$AA?2?$AAr?$AAt?$AAn?$AAd?$AAl?$AAg?$AA?4?$AAc?$AAp?$AAp?$AA?$AA@ 0003b5c0     rtndlg.obj
 0002:0000d5e0       ??_C@_1EK@OPPOJAOO@?$AAO?$AAn?$AAI?$AAn?$AAi?$AAt?$AAR?$AAT?$AAN?$AAD?$AAi?$AAa?$AAl?$AAo?$AAg?$AA?3?$AA?3?$AAS?$AAH?$AAI?$AAn?$AAi?$AAt?$AAD?$AAi?$AAa?$AAl?$AAo?$AAg?$AA?5?$AAF?$AAa@ 0003b5e0     rtndlg.obj
 0002:0000d630       ??_C@_1EI@FBIPKGBE@?$AAO?$AAn?$AAI?$AAn?$AAi?$AAt?$AAR?$AAT?$AAN?$AAD?$AAi?$AAa?$AAl?$AAo?$AAg?$AA?3?$AAS?$AAH?$AAI?$AAn?$AAi?$AAt?$AAD?$AAi?$AAa?$AAl?$AAo?$AAg?$AA?5?$AAF?$AAa?$AAi@ 0003b630     rtndlg.obj
 0002:0000d678       ??_C@_1FA@LMPFIOKO@?$AAO?$AAn?$AAI?$AAn?$AAi?$AAt?$AAR?$AAT?$AAN?$AAD?$AAi?$AAa?$AAl?$AAo?$AAg?$AA?3?$AA?3?$AAS?$AAH?$AAC?$AAr?$AAe?$AAa?$AAt?$AAe?$AAM?$AAe?$AAn?$AAu?$AAB?$AAa?$AAr@ 0003b678     rtndlg.obj
 0002:0000d6c8       ??_C@_1EO@GKONJLEP@?$AAO?$AAn?$AAI?$AAn?$AAi?$AAt?$AAR?$AAT?$AAN?$AAD?$AAi?$AAa?$AAl?$AAo?$AAg?$AA?3?$AAS?$AAH?$AAC?$AAr?$AAe?$AAa?$AAt?$AAe?$AAM?$AAe?$AAn?$AAu?$AAB?$AAa?$AAr?$AA?5@ 0003b6c8     rtndlg.obj
 0002:0000d718       ??_C@_1DC@PHNCJBJP@?$AAO?$AAn?$AAI?$AAn?$AAi?$AAt?$AAR?$AAT?$AAN?$AAD?$AAi?$AAa?$AAl?$AAo?$AAg?$AA?$CI?$AA?$CJ?$AA?5?$AAF?$AAa?$AAi?$AAl?$AAe?$AAd?$AA?$AA@ 0003b718     rtndlg.obj
 0002:0000d750       ??_C@_1EG@MKOKHJG@?$AAW?$AAn?$AAd?$AAP?$AAr?$AAo?$AAc?$AAR?$AAT?$AAN?$AA?3?$AA?5?$AAR?$AAT?$AAN?$AA?1?$AAC?$AAL?$AAE?$AAA?$AAR?$AA?5?$AAr?$AAe?$AAs?$AAe?$AAt?$AA?5?$AAf?$AAa?$AAi?$AAl@ 0003b750     rtndlg.obj
 0002:0000d798       ??_C@_1CO@JJFFHDEN@?$AAR?$AAT?$AAN?$AA?1?$AAC?$AAL?$AAE?$AAA?$AAR?$AA?5?$AAr?$AAe?$AAs?$AAe?$AAt?$AA?5?$AAf?$AAa?$AAi?$AAl?$AAe?$AAd?$AA?$AA@ 0003b798     rtndlg.obj
 0002:0000d7c8       ??_C@_1BGC@BLHGJIBI@?$AAY?$AAo?$AAu?$AA?5?$AAa?$AAr?$AAe?$AA?5?$AAa?$AAb?$AAo?$AAu?$AAt?$AA?5?$AAt?$AAo?$AA?5?$AAp?$AAe?$AAr?$AAf?$AAo?$AAr?$AAm?$AA?5?$AAa?$AA?5?$AAR?$AAT?$AAN?$AA?5?$AAr@ 0003b7c8     rtndlg.obj
 0002:0000d92c       ??_C@_1DK@NHHIDGPK@?$AAW?$AAn?$AAd?$AAP?$AAr?$AAo?$AAc?$AAR?$AAT?$AAN?$AA?3?$AA?5?$AAR?$AAT?$AAN?$AA?5?$AAr?$AAe?$AAs?$AAe?$AAt?$AA?5?$AAf?$AAa?$AAi?$AAl?$AAe?$AAd?$AA?$AA@ 0003b92c     rtndlg.obj
 0002:0000d968       ??_C@_1CC@IECKHGCE@?$AAR?$AAT?$AAN?$AA?5?$AAr?$AAe?$AAs?$AAe?$AAt?$AA?5?$AAf?$AAa?$AAi?$AAl?$AAe?$AAd?$AA?$AA@ 0003b968     rtndlg.obj
 0002:0000d990       ??_C@_1BFA@JHHFOHBM@?$AAY?$AAo?$AAu?$AA?5?$AAa?$AAr?$AAe?$AA?5?$AAa?$AAb?$AAo?$AAu?$AAt?$AA?5?$AAt?$AAo?$AA?5?$AAp?$AAe?$AAr?$AAf?$AAo?$AAr?$AAm?$AA?5?$AAa?$AA?5?$AAR?$AAT?$AAN?$AA?5?$AAr@ 0003b990     rtndlg.obj
 0002:0000dae0       ??_C@_1BK@CPDHDMLD@?$AAD?$AAo?$AA?5?$AAR?$AAT?$AAN?$AA?5?$AAr?$AAe?$AAs?$AAe?$AAt?$AA?$AA@ 0003bae0     rtndlg.obj
 0002:0000db00       ??_C@_1FE@DKJONJIG@?$AAC?$AAr?$AAe?$AAa?$AAt?$AAe?$AAR?$AAT?$AAN?$AAD?$AAl?$AAg?$AA?3?$AA?3?$AAF?$AAa?$AAl?$AAi?$AAe?$AAd?$AA?5?$AAt?$AAo?$AA?5?$AAC?$AAr?$AAe?$AAa?$AAt?$AAe?$AA?5?$AAD@ 0003bb00     rtndlg.obj
 0002:0000db58       ??_C@_1FE@LEFEFJEM@?$AAC?$AAr?$AAe?$AAa?$AAt?$AAe?$AAR?$AAT?$AAN?$AAD?$AAl?$AAg?$AA?3?$AA?3?$AAF?$AAa?$AAl?$AAi?$AAe?$AAd?$AA?5?$AAt?$AAo?$AA?5?$AAR?$AAe?$AAg?$AAi?$AAs?$AAt?$AAe?$AAr@ 0003bb58     rtndlg.obj
 0002:0000dbac       ??_C@_1BC@JBHBKKDL@?$AAM?$AAI?$AAP?$AA?5?$AAo?$AAn?$AAl?$AAy?$AA?$AA@ 0003bbac     simpleipdlg.obj
 0002:0000dbc0       ??_C@_1BM@MLMHMDIE@?$AAM?$AAI?$AAP?$AA?5?$AAp?$AAr?$AAe?$AAf?$AAe?$AAr?$AAr?$AAe?$AAd?$AA?$AA@ 0003bbc0     simpleipdlg.obj
 0002:0000dbdc       ??_C@_1BC@KGPPOEKK@?$AAS?$AAI?$AAP?$AA?5?$AAo?$AAn?$AAl?$AAy?$AA?$AA@ 0003bbdc     simpleipdlg.obj
 0002:0000dbf0       ??_C@_1CC@GGOBPGAJ@?$AAS?$AAi?$AAm?$AAp?$AAl?$AAe?$AAI?$AAP?$AAD?$AAl?$AAg?$AAC?$AAl?$AAa?$AAs?$AAs?$AA?$AA@ 0003bbf0     simpleipdlg.obj
 0002:0000dc20       ??_C@_1EM@CJJJBGDE@?$AAN?$AAV?$AA_?$AAI?$AA_?$AAQ?$AAC?$AAM?$AAI?$AAP?$AA?5?$AAn?$AAv?$AA?5?$AAW?$AAr?$AAi?$AAt?$AAe?$AA?5?$AAf?$AAa?$AAi?$AAl?$AAe?$AAd?$AA?5?$AAv?$AAa?$AAl?$AAu?$AAe@ 0003bc20     simpleipdlg.obj
 0002:0000dc6c       ??_C@_1DC@NCFBACDC@?$AAS?$AAe?$AAt?$AAS?$AAI?$AAP?$AAN?$AAa?$AAi?$AAP?$AAa?$AAs?$AAs?$AAw?$AAo?$AAr?$AAd?$AA?5?$AAf?$AAa?$AAi?$AAl?$AAe?$AAd?$AA?$AA@ 0003bc6c     simpleipdlg.obj
 0002:0000dca0       ??_C@_1CE@DBOGINEG@?$AA?4?$AA?2?$AAs?$AAi?$AAm?$AAp?$AAl?$AAe?$AAi?$AAp?$AAd?$AAl?$AAg?$AA?4?$AAc?$AAp?$AAp?$AA?$AA@ 0003bca0     simpleipdlg.obj
 0002:0000dcc8       ??_C@_1EK@BAKDDNFF@?$AAI?$AAn?$AAi?$AAt?$AAS?$AAi?$AAm?$AAp?$AAl?$AAe?$AAI?$AAP?$AAD?$AAl?$AAg?$AA?3?$AA?3?$AAS?$AAH?$AAI?$AAn?$AAi?$AAt?$AAD?$AAi?$AAa?$AAl?$AAo?$AAg?$AA?5?$AAF?$AAa@ 0003bcc8     simpleipdlg.obj
 0002:0000dd18       ??_C@_1EI@POKGEJKH@?$AAI?$AAn?$AAi?$AAt?$AAS?$AAi?$AAm?$AAp?$AAl?$AAe?$AAI?$AAP?$AAD?$AAl?$AAg?$AA?3?$AAS?$AAH?$AAI?$AAn?$AAi?$AAt?$AAD?$AAi?$AAa?$AAl?$AAo?$AAg?$AA?5?$AAF?$AAa?$AAi@ 0003bd18     simpleipdlg.obj
 0002:0000dd60       ??_C@_1FA@MDLANFKN@?$AAI?$AAn?$AAi?$AAt?$AAS?$AAi?$AAm?$AAp?$AAl?$AAe?$AAI?$AAP?$AAD?$AAl?$AAg?$AA?3?$AA?3?$AAS?$AAH?$AAC?$AAr?$AAe?$AAa?$AAt?$AAe?$AAM?$AAe?$AAn?$AAu?$AAB?$AAa?$AAr@ 0003bd60     simpleipdlg.obj
 0002:0000ddb0       ??_C@_1EO@FDCJFAHD@?$AAI?$AAn?$AAi?$AAt?$AAS?$AAi?$AAm?$AAp?$AAl?$AAe?$AAI?$AAP?$AAD?$AAl?$AAg?$AA?3?$AAS?$AAH?$AAC?$AAr?$AAe?$AAa?$AAt?$AAe?$AAM?$AAe?$AAn?$AAu?$AAB?$AAa?$AAr?$AA?5@ 0003bdb0     simpleipdlg.obj
 0002:0000de00       ??_C@_1CO@NFMBLCII@?$AAI?$AAn?$AAi?$AAt?$AAS?$AAi?$AAm?$AAp?$AAl?$AAe?$AAI?$AAP?$AAD?$AAl?$AAg?$AA?5?$AAF?$AAa?$AAi?$AAl?$AAe?$AAd?$AA?$AA@ 0003be00     simpleipdlg.obj
 0002:0000de30       ??_C@_1FO@FGGCKLDH@?$AAC?$AAr?$AAe?$AAa?$AAt?$AAe?$AAS?$AAi?$AAm?$AAp?$AAl?$AAe?$AAI?$AAP?$AAD?$AAl?$AAg?$AA?3?$AA?3?$AAF?$AAa?$AAl?$AAi?$AAe?$AAd?$AA?5?$AAt?$AAo?$AA?5?$AAR?$AAe?$AAg@ 0003be30     simpleipdlg.obj
 0002:0000de90       ??_C@_1BI@NMOCDMIF@?$AAS?$AAi?$AAp?$AAD?$AAl?$AAg?$AAC?$AAl?$AAa?$AAs?$AAs?$AA?$AA@ 0003be90     sipdlg.obj
 0002:0000dea8       ??_C@_1EA@NIGIIFOI@?$AAI?$AAn?$AAi?$AAt?$AAS?$AAi?$AAp?$AAD?$AAl?$AAg?$AA?3?$AA?3?$AAS?$AAH?$AAI?$AAn?$AAi?$AAt?$AAD?$AAi?$AAa?$AAl?$AAo?$AAg?$AA?5?$AAF?$AAa?$AAl?$AAi?$AAe?$AAd?$AA?$AA@ 0003bea8     sipdlg.obj
 0002:0000dee8       ??_C@_1DO@HLPKBJPG@?$AAI?$AAn?$AAi?$AAt?$AAS?$AAi?$AAp?$AAD?$AAl?$AAg?$AA?3?$AAS?$AAH?$AAI?$AAn?$AAi?$AAt?$AAD?$AAi?$AAa?$AAl?$AAo?$AAg?$AA?5?$AAF?$AAa?$AAi?$AAl?$AAe?$AAd?$AA?$AA@ 0003bee8     sipdlg.obj
 0002:0000df28       ??_C@_1EG@HLKDDICM@?$AAI?$AAn?$AAi?$AAt?$AAS?$AAi?$AAp?$AAD?$AAl?$AAg?$AA?3?$AA?3?$AAS?$AAH?$AAC?$AAr?$AAe?$AAa?$AAt?$AAe?$AAM?$AAe?$AAn?$AAu?$AAB?$AAa?$AAr?$AA?5?$AAF?$AAa?$AAl?$AAi@ 0003bf28     sipdlg.obj
 0002:0000df70       ??_C@_1BK@ODHMJKFJ@?$AA?4?$AA?2?$AAs?$AAi?$AAp?$AAd?$AAl?$AAg?$AA?4?$AAc?$AAp?$AAp?$AA?$AA@ 0003bf70     sipdlg.obj
 0002:0000df90       ??_C@_1EE@MKMNCNJL@?$AAI?$AAn?$AAi?$AAt?$AAS?$AAi?$AAp?$AAD?$AAl?$AAg?$AA?3?$AAS?$AAH?$AAC?$AAr?$AAe?$AAa?$AAt?$AAe?$AAM?$AAe?$AAn?$AAu?$AAB?$AAa?$AAr?$AA?5?$AAF?$AAa?$AAi?$AAl?$AAe@ 0003bf90     sipdlg.obj
 0002:0000dfd4       ??_C@_1CE@ICCPHCFM@?$AAI?$AAn?$AAi?$AAt?$AAS?$AAi?$AAp?$AAD?$AAl?$AAg?$AA?5?$AAF?$AAa?$AAi?$AAl?$AAe?$AAd?$AA?$AA@ 0003bfd4     sipdlg.obj
 0002:0000dff8       ??_C@_1FE@FKKCBPCG@?$AAC?$AAr?$AAe?$AAa?$AAt?$AAe?$AAS?$AAi?$AAp?$AAD?$AAl?$AAg?$AA?3?$AA?3?$AAF?$AAa?$AAl?$AAi?$AAe?$AAd?$AA?5?$AAt?$AAo?$AA?5?$AAC?$AAr?$AAe?$AAa?$AAt?$AAe?$AA?5?$AAD@ 0003bff8     sipdlg.obj
 0002:0000e050       ??_C@_1FE@NEGIJPOM@?$AAC?$AAr?$AAe?$AAa?$AAt?$AAe?$AAS?$AAi?$AAp?$AAD?$AAl?$AAg?$AA?3?$AA?3?$AAF?$AAa?$AAl?$AAi?$AAe?$AAd?$AA?5?$AAt?$AAo?$AA?5?$AAR?$AAe?$AAg?$AAi?$AAs?$AAt?$AAe?$AAr@ 0003c050     sipdlg.obj
 0002:0000e0a4       ??_C@_1CG@KONBGHOB@?$AAS?$AAP?$AAC?$AAV?$AAa?$AAl?$AAi?$AAd?$AAa?$AAt?$AAi?$AAo?$AAn?$AAC?$AAl?$AAa?$AAs?$AAs?$AA?$AA@ 0003c0a4     spcvalidation.obj
 0002:0000e0d0       ??_C@_1EO@BIEHIOOH@?$AAI?$AAn?$AAi?$AAt?$AAS?$AAP?$AAC?$AAV?$AAa?$AAl?$AAi?$AAd?$AAa?$AAt?$AAi?$AAo?$AAn?$AA?3?$AA?3?$AAS?$AAH?$AAI?$AAn?$AAi?$AAt?$AAD?$AAi?$AAa?$AAl?$AAo?$AAg?$AA?5@ 0003c0d0     spcvalidation.obj
 0002:0000e120       ??_C@_1EM@KDBCOEDO@?$AAI?$AAn?$AAi?$AAt?$AAS?$AAP?$AAC?$AAV?$AAa?$AAl?$AAi?$AAd?$AAa?$AAt?$AAi?$AAo?$AAn?$AA?3?$AAS?$AAH?$AAI?$AAn?$AAi?$AAt?$AAD?$AAi?$AAa?$AAl?$AAo?$AAg?$AA?5?$AAF@ 0003c120     spcvalidation.obj
 0002:0000e170       ??_C@_1FE@JENLJCMA@?$AAI?$AAn?$AAi?$AAt?$AAS?$AAP?$AAC?$AAV?$AAa?$AAl?$AAi?$AAd?$AAa?$AAt?$AAi?$AAo?$AAn?$AA?3?$AA?3?$AAS?$AAH?$AAC?$AAr?$AAe?$AAa?$AAt?$AAe?$AAM?$AAe?$AAn?$AAu?$AAB@ 0003c170     spcvalidation.obj
 0002:0000e1c4       ??_C@_1CI@NLJOCIBB@?$AA?4?$AA?2?$AAs?$AAp?$AAc?$AAv?$AAa?$AAl?$AAi?$AAd?$AAa?$AAt?$AAi?$AAo?$AAn?$AA?4?$AAc?$AAp?$AAp?$AA?$AA@ 0003c1c4     spcvalidation.obj
 0002:0000e1f0       ??_C@_1FC@BHIDCIPB@?$AAI?$AAn?$AAi?$AAt?$AAS?$AAP?$AAC?$AAV?$AAa?$AAl?$AAi?$AAd?$AAa?$AAt?$AAi?$AAo?$AAn?$AA?3?$AAS?$AAH?$AAC?$AAr?$AAe?$AAa?$AAt?$AAe?$AAM?$AAe?$AAn?$AAu?$AAB?$AAa@ 0003c1f0     spcvalidation.obj
 0002:0000e244       ??_C@_1DC@IDEKMJPP@?$AAI?$AAn?$AAi?$AAt?$AAS?$AAP?$AAC?$AAV?$AAa?$AAl?$AAi?$AAd?$AAa?$AAt?$AAi?$AAo?$AAn?$AA?5?$AAF?$AAa?$AAi?$AAl?$AAe?$AAd?$AA?$AA@ 0003c244     spcvalidation.obj
 0002:0000e278       ??_C@_17HMHMCIMC@?$AAE?$AAr?$AAr?$AA?$AA@ 0003c278     spcvalidation.obj
 0002:0000e280       ??_C@_1DE@CIOLLDC@?$AAp?$AAl?$AAe?$AAa?$AAs?$AAe?$AA?5?$AAE?$AAn?$AAt?$AAe?$AAr?$AA?5?$AAo?$AAn?$AAl?$AAy?$AA?5?$AAD?$AAi?$AAg?$AAi?$AAt?$AAs?$AA?$CB?$AA?$AA@ 0003c280     spcvalidation.obj
 0002:0000e2b8       ??_C@_1GC@LKMPGNOM@?$AAC?$AAr?$AAe?$AAa?$AAt?$AAe?$AAS?$AAP?$AAC?$AAV?$AAa?$AAl?$AAi?$AAd?$AAa?$AAt?$AAi?$AAo?$AAn?$AA?3?$AA?3?$AAF?$AAa?$AAl?$AAi?$AAe?$AAd?$AA?5?$AAt?$AAo?$AA?5?$AAC@ 0003c2b8     spcvalidation.obj
 0002:0000e320       ??_C@_1GC@DEAFONCG@?$AAC?$AAr?$AAe?$AAa?$AAt?$AAe?$AAS?$AAP?$AAC?$AAV?$AAa?$AAl?$AAi?$AAd?$AAa?$AAt?$AAi?$AAo?$AAn?$AA?3?$AA?3?$AAF?$AAa?$AAl?$AAi?$AAe?$AAd?$AA?5?$AAt?$AAo?$AA?5?$AAR@ 0003c320     spcvalidation.obj
 0002:0000e384       ??_C@_1BO@HAJPLHBB@?$AAS?$AAy?$AAs?$AAt?$AAe?$AAm?$AAD?$AAl?$AAg?$AAC?$AAl?$AAa?$AAs?$AAs?$AA?$AA@ 0003c384     systemdlg.obj
 0002:0000e3f8       ??_C@_1EG@JNDLIJPE@?$AAI?$AAn?$AAi?$AAt?$AAS?$AAy?$AAs?$AAt?$AAe?$AAm?$AAD?$AAl?$AAg?$AA?3?$AA?3?$AAS?$AAH?$AAI?$AAn?$AAi?$AAt?$AAD?$AAi?$AAa?$AAl?$AAo?$AAg?$AA?5?$AAF?$AAa?$AAl?$AAi@ 0003c3f8     systemdlg.obj
 0002:0000e440       ??_C@_1EE@PIOPMHKI@?$AAI?$AAn?$AAi?$AAt?$AAS?$AAy?$AAs?$AAt?$AAe?$AAm?$AAD?$AAl?$AAg?$AA?3?$AAS?$AAH?$AAI?$AAn?$AAi?$AAt?$AAD?$AAi?$AAa?$AAl?$AAo?$AAg?$AA?5?$AAF?$AAa?$AAi?$AAl?$AAe@ 0003c440     systemdlg.obj
 0002:0000e488       ??_C@_1EM@GFKOPIKK@?$AAI?$AAn?$AAi?$AAt?$AAS?$AAy?$AAs?$AAt?$AAe?$AAm?$AAD?$AAl?$AAg?$AA?3?$AA?3?$AAS?$AAH?$AAC?$AAr?$AAe?$AAa?$AAt?$AAe?$AAM?$AAe?$AAn?$AAu?$AAB?$AAa?$AAr?$AA?5?$AAF@ 0003c488     systemdlg.obj
 0002:0000e4d4       ??_C@_1CA@OGIFMHJE@?$AA?4?$AA?2?$AAs?$AAy?$AAs?$AAt?$AAe?$AAm?$AAd?$AAl?$AAg?$AA?4?$AAc?$AAp?$AAp?$AA?$AA@ 0003c4d4     systemdlg.obj
 0002:0000e4f8       ??_C@_1EK@EODIIHFA@?$AAI?$AAn?$AAi?$AAt?$AAS?$AAy?$AAs?$AAt?$AAe?$AAm?$AAD?$AAl?$AAg?$AA?3?$AAS?$AAH?$AAC?$AAr?$AAe?$AAa?$AAt?$AAe?$AAM?$AAe?$AAn?$AAu?$AAB?$AAa?$AAr?$AA?5?$AAF?$AAa@ 0003c4f8     systemdlg.obj
 0002:0000e544       ??_C@_1CK@DNGIGOL@?$AAI?$AAn?$AAi?$AAt?$AAS?$AAy?$AAs?$AAt?$AAe?$AAm?$AAD?$AAl?$AAg?$AA?5?$AAF?$AAa?$AAi?$AAl?$AAe?$AAd?$AA?$AA@ 0003c544     systemdlg.obj
 0002:0000e570       ??_C@_1KI@BOKFGPM@?$AAE?$AAN?$AA_?$AAC?$AAH?$AAA?$AAN?$AAG?$AAE?$AA?5?$AAH?$AAI?$AAW?$AAO?$AAR?$AAD?$AA?5?$AAw?$AAp?$AA?5?$AA?$DN?$AA?5?$AA0?$AAx?$AA?$CF?$AAx?$AA?0?$AA?5?$AAl?$AAp?$AAH?$AAa@ 0003c570     systemdlg.obj
 0002:0000e618       ??_C@_1FK@FHENGDHI@?$AAC?$AAr?$AAe?$AAa?$AAt?$AAe?$AAS?$AAy?$AAs?$AAt?$AAe?$AAm?$AAD?$AAl?$AAg?$AA?3?$AA?3?$AAF?$AAa?$AAl?$AAi?$AAe?$AAd?$AA?5?$AAt?$AAo?$AA?5?$AAC?$AAr?$AAe?$AAa?$AAt@ 0003c618     systemdlg.obj
 0002:0000e678       ??_C@_1FK@NJIHODLC@?$AAC?$AAr?$AAe?$AAa?$AAt?$AAe?$AAS?$AAy?$AAs?$AAt?$AAe?$AAm?$AAD?$AAl?$AAg?$AA?3?$AA?3?$AAF?$AAa?$AAl?$AAi?$AAe?$AAd?$AA?5?$AAt?$AAo?$AA?5?$AAR?$AAe?$AAg?$AAi?$AAs@ 0003c678     systemdlg.obj
 0002:0000e6d4       ??_C@_13LDEHOAPL@?$AA7?$AA?$AA@ 0003c6d4     usernamedlg.obj
 0002:0000e6d8       ??_C@_13LPLIHJO@?$AA6?$AA?$AA@ 0003c6d8     usernamedlg.obj
 0002:0000e6dc       ??_C@_13BJEOCIHA@?$AA5?$AA?$AA@ 0003c6dc     usernamedlg.obj
 0002:0000e6e0       ??_C@_13KBPCEPBF@?$AA4?$AA?$AA@ 0003c6e0     usernamedlg.obj
 0002:0000e6e4       ??_C@_13DMCFHHKM@?$AA3?$AA?$AA@ 0003c6e4     usernamedlg.obj
 0002:0000e6e8       ??_C@_13IEJJBAMJ@?$AA2?$AA?$AA@ 0003c6e8     usernamedlg.obj
 0002:0000e6ec       ??_C@_13JGCMLPCH@?$AA1?$AA?$AA@ 0003c6ec     usernamedlg.obj
 0002:0000e6f0       ??_C@_1CC@DJLLFMOM@?$AAU?$AAs?$AAe?$AAr?$AAn?$AAa?$AAm?$AAe?$AAD?$AAl?$AAg?$AAC?$AAl?$AAa?$AAs?$AAs?$AA?$AA@ 0003c6f0     usernamedlg.obj
 0002:0000e758       ??_C@_19KLMLHLJG@?$AAN?$AAo?$AAn?$AAe?$AA?$AA@ 0003c758     usernamedlg.obj
 0002:0000e764       ??_C@_1CE@FBDJFEEE@?$AA?4?$AA?2?$AAu?$AAs?$AAe?$AAr?$AAn?$AAa?$AAm?$AAe?$AAd?$AAl?$AAg?$AA?4?$AAc?$AAp?$AAp?$AA?$AA@ 0003c764     usernamedlg.obj
 0002:0000e788       ??_C@_1CK@KCOFACBK@?$AAF?$AAa?$AAi?$AAl?$AAe?$AAd?$AA?5?$AAG?$AAe?$AAt?$AAD?$AAs?$AAM?$AAi?$AAp?$AAL?$AAi?$AAs?$AAt?$AA?5?$AA?$AA@ 0003c788     usernamedlg.obj
 0002:0000e7b4       ??_C@_15BICKNCBF@?$AAN?$AAo?$AA?$AA@ 0003c7b4     usernamedlg.obj
 0002:0000e7bc       ??_C@_17PBAHFJOA@?$AAY?$AAe?$AAs?$AA?$AA@ 0003c7bc     usernamedlg.obj
 0002:0000e7c8       ??_C@_1EI@PKNKCCCE@?$AAS?$AAe?$AAt?$AAH?$AAd?$AAr?$AAN?$AAa?$AAi?$AAP?$AAa?$AAs?$AAs?$AAw?$AAo?$AAr?$AAd?$AA?5?$AAf?$AAa?$AAi?$AAl?$AAe?$AAd?$AA?5?$AAg?$AA_?$AAE?$AAr?$AAr?$AA?5?$AA?$DN@ 0003c7c8     usernamedlg.obj
 0002:0000e810       ??_C@_1EK@MCPKKELD@?$AAI?$AAn?$AAi?$AAt?$AAU?$AAs?$AAe?$AAr?$AAn?$AAa?$AAm?$AAe?$AAD?$AAl?$AAg?$AA?3?$AA?3?$AAS?$AAH?$AAI?$AAn?$AAi?$AAt?$AAD?$AAi?$AAa?$AAl?$AAo?$AAg?$AA?5?$AAF?$AAa@ 0003c810     usernamedlg.obj
 0002:0000e860       ??_C@_1EI@DMOKEGFB@?$AAI?$AAn?$AAi?$AAt?$AAU?$AAs?$AAe?$AAr?$AAn?$AAa?$AAm?$AAe?$AAD?$AAl?$AAg?$AA?3?$AAS?$AAH?$AAI?$AAn?$AAi?$AAt?$AAD?$AAi?$AAa?$AAl?$AAo?$AAg?$AA?5?$AAF?$AAa?$AAi@ 0003c860     usernamedlg.obj
 0002:0000e8a8       ??_C@_1FA@OHLDMJCF@?$AAI?$AAn?$AAi?$AAt?$AAU?$AAs?$AAe?$AAr?$AAn?$AAa?$AAm?$AAe?$AAD?$AAl?$AAg?$AA?3?$AA?3?$AAS?$AAH?$AAC?$AAr?$AAe?$AAa?$AAt?$AAe?$AAM?$AAe?$AAn?$AAu?$AAB?$AAa?$AAr@ 0003c8a8     usernamedlg.obj
 0002:0000e8f8       ??_C@_1EO@FBFLJIAN@?$AAI?$AAn?$AAi?$AAt?$AAU?$AAs?$AAe?$AAr?$AAn?$AAa?$AAm?$AAe?$AAD?$AAl?$AAg?$AA?3?$AAS?$AAH?$AAC?$AAr?$AAe?$AAa?$AAt?$AAe?$AAM?$AAe?$AAn?$AAu?$AAB?$AAa?$AAr?$AA?5@ 0003c8f8     usernamedlg.obj
 0002:0000e948       ??_C@_1CO@FLAPCCIP@?$AAI?$AAn?$AAi?$AAt?$AAU?$AAs?$AAe?$AAr?$AAn?$AAa?$AAm?$AAe?$AAD?$AAl?$AAg?$AA?5?$AAF?$AAa?$AAi?$AAl?$AAe?$AAd?$AA?$AA@ 0003c948     usernamedlg.obj
 0002:0000e978       ??_C@_1FO@NCPDMJAB@?$AAC?$AAr?$AAe?$AAa?$AAt?$AAe?$AAU?$AAs?$AAe?$AAr?$AAn?$AAa?$AAm?$AAe?$AAD?$AAl?$AAg?$AA?3?$AA?3?$AAF?$AAa?$AAl?$AAi?$AAe?$AAd?$AA?5?$AAt?$AAo?$AA?5?$AAC?$AAr?$AAe@ 0003c978     usernamedlg.obj
 0002:0000e9d8       ??_C@_1FO@FMDJEJML@?$AAC?$AAr?$AAe?$AAa?$AAt?$AAe?$AAU?$AAs?$AAe?$AAr?$AAn?$AAa?$AAm?$AAe?$AAD?$AAl?$AAg?$AA?3?$AA?3?$AAF?$AAa?$AAl?$AAi?$AAe?$AAd?$AA?5?$AAt?$AAo?$AA?5?$AAR?$AAe?$AAg@ 0003c9d8     usernamedlg.obj
 0002:0000ea38       ??_C@_1CI@NHCDLNLN@?$AAV?$AAe?$AAr?$AAs?$AAi?$AAo?$AAn?$AAI?$AAn?$AAf?$AAo?$AAD?$AAl?$AAg?$AAC?$AAl?$AAa?$AAs?$AAs?$AA?$AA@ 0003ca38     versioninfo.obj
 0002:0000ea60       ??_C@_1DE@EMJBEPGN@?$AA?2?$AAS?$AAt?$AAr?$AAi?$AAn?$AAg?$AAF?$AAi?$AAl?$AAe?$AAI?$AAn?$AAf?$AAo?$AA?2?$AA0?$AA4?$AA0?$AA9?$AA0?$AA4?$AAB?$AA0?$AA?2?$AA?$AA@ 0003ca60     versioninfo.obj
 0002:0000eacc       ??_C@_1CK@DENEAOOB@?$AAM?$AAE?$AAI?$AAD?$AA?5?$AAi?$AAs?$AA?5?$AAn?$AAo?$AAt?$AA?5?$AAp?$AAr?$AAe?$AAs?$AAe?$AAn?$AAt?$AA?4?$AA?$AA@ 0003cacc     versioninfo.obj
 0002:0000eaf8       ??_C@_17HDJIHIPC@?$AAN?$AA?1?$AAA?$AA?$AA@ 0003caf8     versioninfo.obj
 0002:0000eb00       ??_C@_1HM@DBKPLNBD@?$AAD?$AAo?$AA?5?$AAn?$AAo?$AAt?$AA?5?$AAl?$AAo?$AAa?$AAd?$AA?5?$AAa?$AAn?$AAy?$AAt?$AAh?$AAi?$AAn?$AAg?$AA?4?$AA?4?$AA?4?$AA?4?$AAt?$AAh?$AAi?$AAs?$AA?5?$AAv?$AAe?$AAr@ 0003cb00     versioninfo.obj
 0002:0000eb80       ??_C@_1HK@CBBKEHKD@?$AAD?$AAo?$AA?5?$AAn?$AAo?$AAt?$AA?5?$AAl?$AAo?$AAa?$AAd?$AA?5?$AAa?$AAn?$AAy?$AAt?$AAh?$AAi?$AAn?$AAg?$AA?4?$AA?4?$AA?4?$AA?4?$AAt?$AAh?$AAi?$AAs?$AA?5?$AAv?$AAe?$AAr@ 0003cb80     versioninfo.obj
 0002:0000ec00       ??_C@_1GA@PCBAEJHL@?$AA?4?$AA?4?$AA?2?$AA?4?$AA?4?$AA?2?$AA?4?$AA?4?$AA?2?$AAU?$AAt?$AAi?$AAl?$AAi?$AAt?$AAi?$AAe?$AAs?$AA?2?$AAs?$AAw?$AA_?$AAe?$AAm?$AAe?$AAx?$AAt?$AA?2?$AAs?$AAr?$AAc?$AA?2@ 0003cc00     versioninfo.obj
 0002:0000ec60       ??_C@_1LA@NDBKELK@?$AAD?$AAo?$AA?5?$AAn?$AAo?$AAt?$AA?5?$AAl?$AAo?$AAa?$AAd?$AA?5?$AAa?$AAn?$AAy?$AAt?$AAh?$AAi?$AAn?$AAg?$AA?4?$AA?4?$AA?4?$AA?4?$AAt?$AAh?$AAi?$AAs?$AA?5?$AAv?$AAe?$AAr@ 0003cc60     versioninfo.obj
 0002:0000ed10       ??_C@_1FA@DGJIKFJG@?$AAI?$AAn?$AAi?$AAt?$AAV?$AAe?$AAr?$AAs?$AAi?$AAo?$AAn?$AAI?$AAn?$AAf?$AAo?$AAD?$AAl?$AAg?$AA?3?$AA?3?$AAS?$AAH?$AAI?$AAn?$AAi?$AAt?$AAD?$AAi?$AAa?$AAl?$AAo?$AAg@ 0003cd10     versioninfo.obj
 0002:0000ed60       ??_C@_1EO@OOLDGNGO@?$AAI?$AAn?$AAi?$AAt?$AAV?$AAe?$AAr?$AAs?$AAi?$AAo?$AAn?$AAI?$AAn?$AAf?$AAo?$AAD?$AAl?$AAg?$AA?3?$AAS?$AAH?$AAI?$AAn?$AAi?$AAt?$AAD?$AAi?$AAa?$AAl?$AAo?$AAg?$AA?5@ 0003cd60     versioninfo.obj
 0002:0000edb0       ??_C@_1FG@KOFAJAJE@?$AAI?$AAn?$AAi?$AAt?$AAV?$AAe?$AAr?$AAs?$AAi?$AAo?$AAn?$AAI?$AAn?$AAf?$AAo?$AAD?$AAl?$AAg?$AA?3?$AA?3?$AAS?$AAH?$AAC?$AAr?$AAe?$AAa?$AAt?$AAe?$AAM?$AAe?$AAn?$AAu@ 0003cdb0     versioninfo.obj
 0002:0000ee08       ??_C@_1FE@CKGOJCBG@?$AAI?$AAn?$AAi?$AAt?$AAV?$AAe?$AAr?$AAs?$AAi?$AAo?$AAn?$AAI?$AAn?$AAf?$AAo?$AAD?$AAl?$AAg?$AA?3?$AAS?$AAH?$AAC?$AAr?$AAe?$AAa?$AAt?$AAe?$AAM?$AAe?$AAn?$AAu?$AAB@ 0003ce08     versioninfo.obj
 0002:0000ee5c       ??_C@_1DE@ONINLNPH@?$AAI?$AAn?$AAi?$AAt?$AAV?$AAe?$AAr?$AAs?$AAi?$AAo?$AAn?$AAI?$AAn?$AAf?$AAo?$AAD?$AAl?$AAg?$AA?5?$AAF?$AAa?$AAi?$AAl?$AAe?$AAd?$AA?$AA@ 0003ce5c     versioninfo.obj
 0002:0000ee90       ??_C@_1GE@KGICFLLF@?$AAC?$AAr?$AAe?$AAa?$AAt?$AAe?$AAV?$AAe?$AAr?$AAs?$AAi?$AAo?$AAn?$AAI?$AAn?$AAf?$AAo?$AAD?$AAl?$AAg?$AA?3?$AA?3?$AAF?$AAa?$AAl?$AAi?$AAe?$AAd?$AA?5?$AAt?$AAo?$AA?5@ 0003ce90     versioninfo.obj
 0002:0000eef8       ??_C@_1GE@CIEINLHP@?$AAC?$AAr?$AAe?$AAa?$AAt?$AAe?$AAV?$AAe?$AAr?$AAs?$AAi?$AAo?$AAn?$AAI?$AAn?$AAf?$AAo?$AAD?$AAl?$AAg?$AA?3?$AA?3?$AAF?$AAa?$AAl?$AAi?$AAe?$AAd?$AA?5?$AAt?$AAo?$AA?5@ 0003cef8     versioninfo.obj
 0002:0000ef5c       ??_C@_1CA@DDGFEPHN@?$AAV?$AAo?$AAc?$AAo?$AAd?$AAe?$AAr?$AAD?$AAl?$AAg?$AAC?$AAl?$AAa?$AAs?$AAs?$AA?$AA@ 0003cf5c     vocoderdlg.obj
 0002:0000efd0       ??_C@_1EI@DHFKFMNC@?$AAI?$AAn?$AAi?$AAt?$AAV?$AAo?$AAc?$AAo?$AAd?$AAe?$AAr?$AAD?$AAl?$AAg?$AA?3?$AA?3?$AAS?$AAH?$AAI?$AAn?$AAi?$AAt?$AAD?$AAi?$AAa?$AAl?$AAo?$AAg?$AA?5?$AAF?$AAa?$AAl@ 0003cfd0     vocoderdlg.obj
 0002:0000f018       ??_C@_1EG@KMHFNPI@?$AAI?$AAn?$AAi?$AAt?$AAV?$AAo?$AAc?$AAo?$AAd?$AAe?$AAr?$AAD?$AAl?$AAg?$AA?3?$AAS?$AAH?$AAI?$AAn?$AAi?$AAt?$AAD?$AAi?$AAa?$AAl?$AAo?$AAg?$AA?5?$AAF?$AAa?$AAi?$AAl@ 0003d018     vocoderdlg.obj
 0002:0000f060       ??_C@_1EO@KCDLKGHI@?$AAI?$AAn?$AAi?$AAt?$AAV?$AAo?$AAc?$AAo?$AAd?$AAe?$AAr?$AAD?$AAl?$AAg?$AA?3?$AA?3?$AAS?$AAH?$AAC?$AAr?$AAe?$AAa?$AAt?$AAe?$AAM?$AAe?$AAn?$AAu?$AAB?$AAa?$AAr?$AA?5@ 0003d060     vocoderdlg.obj
 0002:0000f0b0       ??_C@_1CC@FFIFJOIF@?$AA?4?$AA?2?$AAv?$AAo?$AAc?$AAo?$AAd?$AAe?$AAr?$AAd?$AAl?$AAg?$AA?4?$AAc?$AAp?$AAp?$AA?$AA@ 0003d0b0     vocoderdlg.obj
 0002:0000f0d8       ??_C@_1EM@KMGJAHJ@?$AAI?$AAn?$AAi?$AAt?$AAV?$AAo?$AAc?$AAo?$AAd?$AAe?$AAr?$AAD?$AAl?$AAg?$AA?3?$AAS?$AAH?$AAC?$AAr?$AAe?$AAa?$AAt?$AAe?$AAM?$AAe?$AAn?$AAu?$AAB?$AAa?$AAr?$AA?5?$AAF@ 0003d0d8     vocoderdlg.obj
 0002:0000f124       ??_C@_1CM@IELCGABB@?$AAI?$AAn?$AAi?$AAt?$AAV?$AAo?$AAc?$AAo?$AAd?$AAe?$AAr?$AAD?$AAl?$AAg?$AA?5?$AAF?$AAa?$AAi?$AAl?$AAe?$AAd?$AA?$AA@ 0003d124     vocoderdlg.obj
 0002:0000f150       ??_C@_1FM@IPDAIFMA@?$AAC?$AAr?$AAe?$AAa?$AAt?$AAe?$AAV?$AAo?$AAc?$AAo?$AAd?$AAe?$AAr?$AAD?$AAl?$AAg?$AA?3?$AA?3?$AAF?$AAa?$AAl?$AAi?$AAe?$AAd?$AA?5?$AAt?$AAo?$AA?5?$AAC?$AAr?$AAe?$AAa@ 0003d150     vocoderdlg.obj
 0002:0000f1b0       ??_C@_1FM@BPKAFAK@?$AAC?$AAr?$AAe?$AAa?$AAt?$AAe?$AAV?$AAo?$AAc?$AAo?$AAd?$AAe?$AAr?$AAD?$AAl?$AAg?$AA?3?$AA?3?$AAF?$AAa?$AAl?$AAi?$AAe?$AAd?$AA?5?$AAt?$AAo?$AA?5?$AAR?$AAe?$AAg?$AAi@ 0003d1b0     vocoderdlg.obj
 0002:0000f20c       ??_C@_08JCCMCCIL@HH?3mm?3ss?$AA@ 0003d20c     LIBCMT:strftime.obj
 0002:0000f218       ??_C@_0BE@CKGJFCPC@dddd?0?5MMMM?5dd?0?5yyyy?$AA@ 0003d218     LIBCMT:strftime.obj
 0002:0000f22c       ??_C@_08BPBNCDIB@MM?1dd?1yy?$AA@ 0003d22c     LIBCMT:strftime.obj
 0002:0000f238       ??_C@_02CJNFDJBF@PM?$AA@   0003d238     LIBCMT:strftime.obj
 0002:0000f23c       ??_C@_02DEDBPAFC@AM?$AA@   0003d23c     LIBCMT:strftime.obj
 0002:0000f240       ??_C@_08EDHMEBNP@December?$AA@ 0003d240     LIBCMT:strftime.obj
 0002:0000f24c       ??_C@_08HCHEGEOA@November?$AA@ 0003d24c     LIBCMT:strftime.obj
 0002:0000f258       ??_C@_07JJNFCEND@October?$AA@ 0003d258     LIBCMT:strftime.obj
 0002:0000f260       ??_C@_09BHHEALKD@September?$AA@ 0003d260     LIBCMT:strftime.obj
 0002:0000f26c       ??_C@_06LBBHFDDG@August?$AA@ 0003d26c     LIBCMT:strftime.obj
 0002:0000f274       ??_C@_04MIEPOIFP@July?$AA@ 0003d274     LIBCMT:strftime.obj
 0002:0000f27c       ??_C@_04CNLMGBGM@June?$AA@ 0003d27c     LIBCMT:strftime.obj
 0002:0000f284       ??_C@_05DMJDNLEJ@April?$AA@ 0003d284     LIBCMT:strftime.obj
 0002:0000f28c       ??_C@_05HPCKOFNC@March?$AA@ 0003d28c     LIBCMT:strftime.obj
 0002:0000f294       ??_C@_08GNJGEPFN@February?$AA@ 0003d294     LIBCMT:strftime.obj
 0002:0000f2a0       ??_C@_07CGJPFGJA@January?$AA@ 0003d2a0     LIBCMT:strftime.obj
 0002:0000f2a8       ??_C@_03MKABNOCG@Dec?$AA@  0003d2a8     LIBCMT:strftime.obj
 0002:0000f2ac       ??_C@_03JPJOFNIA@Nov?$AA@  0003d2ac     LIBCMT:strftime.obj
 0002:0000f2b0       ??_C@_03BMAOKBAD@Oct?$AA@  0003d2b0     LIBCMT:strftime.obj
 0002:0000f2b4       ??_C@_03GGCAPAJC@Sep?$AA@  0003d2b4     LIBCMT:strftime.obj
 0002:0000f2b8       ??_C@_03IFJFEIGA@Aug?$AA@  0003d2b8     LIBCMT:strftime.obj
 0002:0000f2bc       ??_C@_03LBGABGKK@Jul?$AA@  0003d2bc     LIBCMT:strftime.obj
 0002:0000f2c0       ??_C@_03IDFGHECI@Jun?$AA@  0003d2c0     LIBCMT:strftime.obj
 0002:0000f2c4       ??_C@_03CNMDKL@May?$AA@    0003d2c4     LIBCMT:strftime.obj
 0002:0000f2c8       ??_C@_03LEOLGMJP@Apr?$AA@  0003d2c8     LIBCMT:strftime.obj
 0002:0000f2cc       ??_C@_03ODNJBKGA@Mar?$AA@  0003d2cc     LIBCMT:strftime.obj
 0002:0000f2d0       ??_C@_03HJBDCHOM@Feb?$AA@  0003d2d0     LIBCMT:strftime.obj
 0002:0000f2d4       ??_C@_03JIHJHPIE@Jan?$AA@  0003d2d4     LIBCMT:strftime.obj
 0002:0000f2d8       ??_C@_08INBOOONO@Saturday?$AA@ 0003d2d8     LIBCMT:strftime.obj
 0002:0000f2e4       ??_C@_06JECMNKMI@Friday?$AA@ 0003d2e4     LIBCMT:strftime.obj
 0002:0000f2ec       ??_C@_08HACCIKIA@Thursday?$AA@ 0003d2ec     LIBCMT:strftime.obj
 0002:0000f2f8       ??_C@_09DLIGFAKA@Wednesday?$AA@ 0003d2f8     LIBCMT:strftime.obj
 0002:0000f304       ??_C@_07BAAGCFCM@Tuesday?$AA@ 0003d304     LIBCMT:strftime.obj
 0002:0000f30c       ??_C@_06JLEDEDGH@Monday?$AA@ 0003d30c     LIBCMT:strftime.obj
 0002:0000f314       ??_C@_06OOPIFAJ@Sunday?$AA@ 0003d314     LIBCMT:strftime.obj
 0002:0000f31c       ??_C@_03FEFJNEK@Sat?$AA@   0003d31c     LIBCMT:strftime.obj
 0002:0000f320       ??_C@_03IDIOELNC@Fri?$AA@  0003d320     LIBCMT:strftime.obj
 0002:0000f324       ??_C@_03IOFIKPDN@Thu?$AA@  0003d324     LIBCMT:strftime.obj
 0002:0000f328       ??_C@_03MHOMLAJA@Wed?$AA@  0003d328     LIBCMT:strftime.obj
 0002:0000f32c       ??_C@_03NAGEINEP@Tue?$AA@  0003d32c     LIBCMT:strftime.obj
 0002:0000f330       ??_C@_03PDAGKDH@Mon?$AA@   0003d330     LIBCMT:strftime.obj
 0002:0000f334       ??_C@_03KOEHGMDN@Sun?$AA@  0003d334     LIBCMT:strftime.obj
 0002:0000f338       ??_C@_03EBAPMIKO@a?1p?$AA@ 0003d338     LIBCMT:strftime.obj
 0002:0000f33c       ??_C@_05JAMEPDIN@am?1pm?$AA@ 0003d33c     LIBCMT:strftime.obj
 0002:0000f344       __dnames                   0003d344     LIBCMT:timeset.obj
 0002:0000f35c       __mnames                   0003d35c     LIBCMT:timeset.obj
 0002:0000f388       __newctype                 0003d388     LIBCMT:ctype.obj
 0002:0000f688       _wctype                    0003d688     LIBCMT:ctype.obj
 0002:0000fabc       __IMPORT_DESCRIPTOR_COREDLL 0003dabc     coredll:COREDLL.dll
 0002:0000fad0       __IMPORT_DESCRIPTOR_AYGSHELL 0003dad0     aygshell:AYGSHELL.dll
 0002:0000fae4       __IMPORT_DESCRIPTOR_sw_utilityG 0003dae4     sw_utilityG:sw_utilityG.dll
 0002:0000faf8       __IMPORT_DESCRIPTOR_GobiApi 0003daf8     GobiApi:GobiApi.dll
 0002:0000fb0c       __NULL_IMPORT_DESCRIPTOR   0003db0c     coredll:COREDLL.dll
 0003:00000000       __imp_SHInitDialog         0003f000     aygshell:AYGSHELL.dll
 0003:00000004       __imp_SHCreateMenuBar      0003f004     aygshell:AYGSHELL.dll
 0003:00000008       \177AYGSHELL_NULL_THUNK_DATA 0003f008     aygshell:AYGSHELL.dll
 0003:0000000c       __imp_LoadStringW          0003f00c     coredll:COREDLL.dll
 0003:00000010       __imp_GetWindowTextW       0003f010     coredll:COREDLL.dll
 0003:00000014       __imp_wcsncpy              0003f014     coredll:COREDLL.dll
 0003:00000018       __imp_wcscpy               0003f018     coredll:COREDLL.dll
 0003:0000001c       __imp_Sleep                0003f01c     coredll:COREDLL.dll
 0003:00000020       __imp_swprintf             0003f020     coredll:COREDLL.dll
 0003:00000024       __imp_SetWindowTextW       0003f024     coredll:COREDLL.dll
 0003:00000028       __imp_GetDlgItem           0003f028     coredll:COREDLL.dll
 0003:0000002c       __imp_SetDlgItemInt        0003f02c     coredll:COREDLL.dll
 0003:00000030       __imp_SetDlgItemTextW      0003f030     coredll:COREDLL.dll
 0003:00000034       __imp_memset               0003f034     coredll:COREDLL.dll
 0003:00000038       __imp_EndDialog            0003f038     coredll:COREDLL.dll
 0003:0000003c       __imp_MessageBoxW          0003f03c     coredll:COREDLL.dll
 0003:00000040       __imp_SetFocus             0003f040     coredll:COREDLL.dll
 0003:00000044       __imp_DialogBoxIndirectParamW 0003f044     coredll:COREDLL.dll
 0003:00000048       __imp_LoadResource         0003f048     coredll:COREDLL.dll
 0003:0000004c       __imp_FindResourceW        0003f04c     coredll:COREDLL.dll
 0003:00000050       __imp_GetLastError         0003f050     coredll:COREDLL.dll
 0003:00000054       __imp_RegisterClassW       0003f054     coredll:COREDLL.dll
 0003:00000058       __imp_GetStockObject       0003f058     coredll:COREDLL.dll
 0003:0000005c       __imp_RegisterWindowMessageW 0003f05c     coredll:COREDLL.dll
 0003:00000060       __imp_EnableMenuItem       0003f060     coredll:COREDLL.dll
 0003:00000064       __imp_wcslen               0003f064     coredll:COREDLL.dll
 0003:00000068       __imp_EnableWindow         0003f068     coredll:COREDLL.dll
 0003:0000006c       __imp_ShowWindow           0003f06c     coredll:COREDLL.dll
 0003:00000070       __imp__wtol                0003f070     coredll:COREDLL.dll
 0003:00000074       __imp_PostMessageW         0003f074     coredll:COREDLL.dll
 0003:00000078       __imp_PostQuitMessage      0003f078     coredll:COREDLL.dll
 0003:0000007c       __imp___utos               0003f07c     coredll:COREDLL.dll
 0003:00000080       __imp___gts                0003f080     coredll:COREDLL.dll
 0003:00000084       __imp___ges                0003f084     coredll:COREDLL.dll
 0003:00000088       __imp___les                0003f088     coredll:COREDLL.dll
 0003:0000008c       __imp___muls               0003f08c     coredll:COREDLL.dll
 0003:00000090       __imp___eqs                0003f090     coredll:COREDLL.dll
 0003:00000094       __imp___itos               0003f094     coredll:COREDLL.dll
 0003:00000098       __imp___stou               0003f098     coredll:COREDLL.dll
 0003:0000009c       __imp___rt_udiv            0003f09c     coredll:COREDLL.dll
 0003:000000a0       __imp___stod               0003f0a0     coredll:COREDLL.dll
 0003:000000a4       __imp___dtos               0003f0a4     coredll:COREDLL.dll
 0003:000000a8       __imp___utod               0003f0a8     coredll:COREDLL.dll
 0003:000000ac       __imp___muld               0003f0ac     coredll:COREDLL.dll
 0003:000000b0       __imp___dtou               0003f0b0     coredll:COREDLL.dll
 0003:000000b4       __imp_TerminateThread      0003f0b4     coredll:COREDLL.dll
 0003:000000b8       __imp_WaitForSingleObject  0003f0b8     coredll:COREDLL.dll
 0003:000000bc       __imp_CreateThread         0003f0bc     coredll:COREDLL.dll
 0003:000000c0       __imp_KillTimer            0003f0c0     coredll:COREDLL.dll
 0003:000000c4       __imp_SetTimer             0003f0c4     coredll:COREDLL.dll
 0003:000000c8       __imp_MultiByteToWideChar  0003f0c8     coredll:COREDLL.dll
 0003:000000cc       __imp_SetWindowPos         0003f0cc     coredll:COREDLL.dll
 0003:000000d0       __imp__wcsicmp             0003f0d0     coredll:COREDLL.dll
 0003:000000d4       __imp_LeaveCriticalSection 0003f0d4     coredll:COREDLL.dll
 0003:000000d8       __imp_EnterCriticalSection 0003f0d8     coredll:COREDLL.dll
 0003:000000dc       __imp_DeleteCriticalSection 0003f0dc     coredll:COREDLL.dll
 0003:000000e0       __imp_InitializeCriticalSection 0003f0e0     coredll:COREDLL.dll
 0003:000000e4       __imp___itod               0003f0e4     coredll:COREDLL.dll
 0003:000000e8       __imp___ltd                0003f0e8     coredll:COREDLL.dll
 0003:000000ec       __imp___negd               0003f0ec     coredll:COREDLL.dll
 0003:000000f0       __imp___subd               0003f0f0     coredll:COREDLL.dll
 0003:000000f4       __imp___dtoi               0003f0f4     coredll:COREDLL.dll
 0003:000000f8       __imp_free                 0003f0f8     coredll:COREDLL.dll
 0003:000000fc       __imp_wcstombs             0003f0fc     coredll:COREDLL.dll
 0003:00000100       __imp_malloc               0003f100     coredll:COREDLL.dll
 0003:00000104       __imp_strlen               0003f104     coredll:COREDLL.dll
 0003:00000108       __imp_sscanf               0003f108     coredll:COREDLL.dll
 0003:0000010c       __imp_wcscmp               0003f10c     coredll:COREDLL.dll
 0003:00000110       __imp_memcpy               0003f110     coredll:COREDLL.dll
 0003:00000114       __imp_HideCaret            0003f114     coredll:COREDLL.dll
 0003:00000118       __imp_GetWindowLongW       0003f118     coredll:COREDLL.dll
 0003:0000011c       __imp_??2@YAPAXI@Z         0003f11c     coredll:COREDLL.dll
 0003:00000120       __imp_SetWindowLongW       0003f120     coredll:COREDLL.dll
 0003:00000124       __imp_GetParent            0003f124     coredll:COREDLL.dll
 0003:00000128       __imp_CreateWindowExW      0003f128     coredll:COREDLL.dll
 0003:0000012c       __imp_DestroyWindow        0003f12c     coredll:COREDLL.dll
 0003:00000130       __imp_IsWindow             0003f130     coredll:COREDLL.dll
 0003:00000134       __imp_wcscat               0003f134     coredll:COREDLL.dll
 0003:00000138       __imp_MessageBeep          0003f138     coredll:COREDLL.dll
 0003:0000013c       __imp_iswctype             0003f13c     coredll:COREDLL.dll
 0003:00000140       __imp_OutputDebugStringW   0003f140     coredll:COREDLL.dll
 0003:00000144       __imp_DefWindowProcW       0003f144     coredll:COREDLL.dll
 0003:00000148       __imp_UpdateWindow         0003f148     coredll:COREDLL.dll
 0003:0000014c       __imp_GetWindowTextLengthW 0003f14c     coredll:COREDLL.dll
 0003:00000150       __imp___divd               0003f150     coredll:COREDLL.dll
 0003:00000154       __imp___addd               0003f154     coredll:COREDLL.dll
 0003:00000158       __imp_LoadBitmapW          0003f158     coredll:COREDLL.dll
 0003:0000015c       __imp__wcsupr              0003f15c     coredll:COREDLL.dll
 0003:00000160       __imp_CloseHandle          0003f160     coredll:COREDLL.dll
 0003:00000164       __imp_SetForegroundWindow  0003f164     coredll:COREDLL.dll
 0003:00000168       __imp_FindWindowW          0003f168     coredll:COREDLL.dll
 0003:0000016c       __imp_GetMessageW          0003f16c     coredll:COREDLL.dll
 0003:00000170       __imp_DispatchMessageW     0003f170     coredll:COREDLL.dll
 0003:00000174       __imp_TranslateMessage     0003f174     coredll:COREDLL.dll
 0003:00000178       __imp_CreateMutexW         0003f178     coredll:COREDLL.dll
 0003:0000017c       __imp_LoadLibraryW         0003f17c     coredll:COREDLL.dll
 0003:00000180       __imp__isctype             0003f180     coredll:COREDLL.dll
 0003:00000184       __imp_SendDlgItemMessageW  0003f184     coredll:COREDLL.dll
 0003:00000188       __imp__wtoll               0003f188     coredll:COREDLL.dll
 0003:0000018c       __imp_wsprintfW            0003f18c     coredll:COREDLL.dll
 0003:00000190       __imp_SetActiveWindow      0003f190     coredll:COREDLL.dll
 0003:00000194       __imp_??3@YAXPAX@Z         0003f194     coredll:COREDLL.dll
 0003:00000198       __imp_GetClientRect        0003f198     coredll:COREDLL.dll
 0003:0000019c       __imp_SendMessageW         0003f19c     coredll:COREDLL.dll
 0003:000001a0       __imp_SetLastError         0003f1a0     coredll:COREDLL.dll
 0003:000001a4       __imp_GetTimeZoneInformation 0003f1a4     coredll:COREDLL.dll
 0003:000001a8       __imp_WideCharToMultiByte  0003f1a8     coredll:COREDLL.dll
 0003:000001ac       __imp_RaiseException       0003f1ac     coredll:COREDLL.dll
 0003:000001b0       __imp_GetDateFormatW       0003f1b0     coredll:COREDLL.dll
 0003:000001b4       __imp_GetTimeFormatW       0003f1b4     coredll:COREDLL.dll
 0003:000001b8       __imp__stricmp             0003f1b8     coredll:COREDLL.dll
 0003:000001bc       __imp___rt_srem64by64      0003f1bc     coredll:COREDLL.dll
 0003:000001c0       __imp___rt_sdiv64by64      0003f1c0     coredll:COREDLL.dll
 0003:000001c4       __imp_mbstowcs             0003f1c4     coredll:COREDLL.dll
 0003:000001c8       __imp___security_gen_cookie 0003f1c8     coredll:COREDLL.dll
 0003:000001cc       __imp_LocalFree            0003f1cc     coredll:COREDLL.dll
 0003:000001d0       __imp___report_gsfailure   0003f1d0     coredll:COREDLL.dll
 0003:000001d4       __imp___C_specific_handler 0003f1d4     coredll:COREDLL.dll
 0003:000001d8       __imp__XcptFilter          0003f1d8     coredll:COREDLL.dll
 0003:000001dc       __imp_TerminateProcess     0003f1dc     coredll:COREDLL.dll
 0003:000001e0       \177COREDLL_NULL_THUNK_DATA 0003f1e0     coredll:COREDLL.dll
 0003:000001e4       __imp_SetConfig            0003f1e4     GobiApi:GobiApi.dll
 0003:000001e8       __imp_GetConfig            0003f1e8     GobiApi:GobiApi.dll
 0003:000001ec       __imp_QCWWANConnect        0003f1ec     GobiApi:GobiApi.dll
 0003:000001f0       __imp_GetTxRxInfo          0003f1f0     GobiApi:GobiApi.dll
 0003:000001f4       __imp_GetRFInfo            0003f1f4     GobiApi:GobiApi.dll
 0003:000001f8       __imp_GetHdrColorCode      0003f1f8     GobiApi:GobiApi.dll
 0003:000001fc       __imp_SwiGetHrpdStats      0003f1fc     GobiApi:GobiApi.dll
 0003:00000200       __imp_GetANAAAAuthenticationStatus 0003f200     GobiApi:GobiApi.dll
 0003:00000204       __imp_SwiGetSignalStrengthInfo 0003f204     GobiApi:GobiApi.dll
 0003:00000208       __imp_GetErrRate           0003f208     GobiApi:GobiApi.dll
 0003:0000020c       __imp_SwiGetCdmaDominantPn 0003f20c     GobiApi:GobiApi.dll
 0003:00000210       __imp_GetModelID           0003f210     GobiApi:GobiApi.dll
 0003:00000214       __imp_GetFirmwareRevisions 0003f214     GobiApi:GobiApi.dll
 0003:00000218       __imp_GetHardwareRevision  0003f218     GobiApi:GobiApi.dll
 0003:0000021c       __imp_GetPRLVersion        0003f21c     GobiApi:GobiApi.dll
 0003:00000220       __imp_GetSysInfo           0003f220     GobiApi:GobiApi.dll
 0003:00000224       __imp_SetDdtmPreference    0003f224     GobiApi:GobiApi.dll
 0003:00000228       \177GobiApi_NULL_THUNK_DATA 0003f228     GobiApi:GobiApi.dll
 0003:0000022c       __imp_GetProvisionInfo     0003f22c     sw_utilityG:sw_utilityG.dll
 0003:00000230       __imp_GetCallstate         0003f230     sw_utilityG:sw_utilityG.dll
 0003:00000234       __imp_GetProvisionState    0003f234     sw_utilityG:sw_utilityG.dll
 0003:00000238       __imp_GetDMMode            0003f238     sw_utilityG:sw_utilityG.dll
 0003:0000023c       __imp_GetPTMode            0003f23c     sw_utilityG:sw_utilityG.dll
 0003:00000240       __imp_StartPTMode          0003f240     sw_utilityG:sw_utilityG.dll
 0003:00000244       __imp_StartDMMode          0003f244     sw_utilityG:sw_utilityG.dll
 0003:00000248       __imp_StopPTMode           0003f248     sw_utilityG:sw_utilityG.dll
 0003:0000024c       __imp_StopDMMode           0003f24c     sw_utilityG:sw_utilityG.dll
 0003:00000250       __imp_GetRilStatus         0003f250     sw_utilityG:sw_utilityG.dll
 0003:00000254       __imp_ValidateSpc          0003f254     sw_utilityG:sw_utilityG.dll
 0003:00000258       __imp_StartDebugMode       0003f258     sw_utilityG:sw_utilityG.dll
 0003:0000025c       __imp_StopDebugMode        0003f25c     sw_utilityG:sw_utilityG.dll
 0003:00000260       __imp_EnableTechHdrNotifications 0003f260     sw_utilityG:sw_utilityG.dll
 0003:00000264       __imp_GetRilDebugInfo      0003f264     sw_utilityG:sw_utilityG.dll
 0003:00000268       __imp_?GetResolution@@YAHXZ 0003f268     sw_utilityG:sw_utilityG.dll
 0003:0000026c       __imp_?InitLog@@YAXPAUHINSTANCE__@@@Z 0003f26c     sw_utilityG:sw_utilityG.dll
 0003:00000270       __imp_GetMDNLengthSupported 0003f270     sw_utilityG:sw_utilityG.dll
 0003:00000274       __imp_InitiateHostBoot     0003f274     sw_utilityG:sw_utilityG.dll
 0003:00000278       __imp_RtnReset             0003f278     sw_utilityG:sw_utilityG.dll
 0003:0000027c       __imp_GetSIPNaiPassword    0003f27c     sw_utilityG:sw_utilityG.dll
 0003:00000280       __imp_SetSIPNaiPassword    0003f280     sw_utilityG:sw_utilityG.dll
 0003:00000284       __imp_ModGetRoamingMode    0003f284     sw_utilityG:sw_utilityG.dll
 0003:00000288       __imp_ModGetSysPrefMode    0003f288     sw_utilityG:sw_utilityG.dll
 0003:0000028c       __imp_ModGetHDRHybrPrefMode 0003f28c     sw_utilityG:sw_utilityG.dll
 0003:00000290       __imp_ModSetSysPrefMode    0003f290     sw_utilityG:sw_utilityG.dll
 0003:00000294       __imp_ModSetRoamingMode    0003f294     sw_utilityG:sw_utilityG.dll
 0003:00000298       __imp_ModSetHDRHybrPrefMode 0003f298     sw_utilityG:sw_utilityG.dll
 0003:0000029c       __imp_GetDsMipList         0003f29c     sw_utilityG:sw_utilityG.dll
 0003:000002a0       __imp_?DWORD2IP@@YAPBGK@Z  0003f2a0     sw_utilityG:sw_utilityG.dll
 0003:000002a4       __imp_GetDsMipProfile      0003f2a4     sw_utilityG:sw_utilityG.dll
 0003:000002a8       __imp_SetHdrNaiPassword    0003f2a8     sw_utilityG:sw_utilityG.dll
 0003:000002ac       __imp_SetDsMipProfile      0003f2ac     sw_utilityG:sw_utilityG.dll
 0003:000002b0       __imp_GetVersionInfo       0003f2b0     sw_utilityG:sw_utilityG.dll
 0003:000002b4       __imp_SetProvisionInfo     0003f2b4     sw_utilityG:sw_utilityG.dll
 0003:000002b8       __imp_DialEx               0003f2b8     sw_utilityG:sw_utilityG.dll
 0003:000002bc       __imp_HangUp               0003f2bc     sw_utilityG:sw_utilityG.dll
 0003:000002c0       __imp_?GetProductFeatures@@YAHAAK@Z 0003f2c0     sw_utilityG:sw_utilityG.dll
 0003:000002c4       __imp_SelectGSMBand        0003f2c4     sw_utilityG:sw_utilityG.dll
 0003:000002c8       __imp_GetCurrentGSMBandAndList 0003f2c8     sw_utilityG:sw_utilityG.dll
 0003:000002cc       __imp_GetItemnizedUMTSInfo 0003f2cc     sw_utilityG:sw_utilityG.dll
 0003:000002d0       __imp_?RelayoutDialog@@YAHPAUHINSTANCE__@@PAUHWND__@@PBG@Z 0003f2d0     sw_utilityG:sw_utilityG.dll
 0003:000002d4       __imp_GetGSMInfo           0003f2d4     sw_utilityG:sw_utilityG.dll
 0003:000002d8       __imp_SetPDSMPAParam       0003f2d8     sw_utilityG:sw_utilityG.dll
 0003:000002dc       __imp_ReadPDSMPAParam      0003f2dc     sw_utilityG:sw_utilityG.dll
 0003:000002e0       __imp_GetRilPAParam        0003f2e0     sw_utilityG:sw_utilityG.dll
 0003:000002e4       __imp_?IP2DWORD@@YAKPBG@Z  0003f2e4     sw_utilityG:sw_utilityG.dll
 0003:000002e8       __imp_StopPDSMDldNotifstatus 0003f2e8     sw_utilityG:sw_utilityG.dll
 0003:000002ec       __imp_StopPDSMLocNotifstatus 0003f2ec     sw_utilityG:sw_utilityG.dll
 0003:000002f0       __imp_StartPDSMDldNotifstatus 0003f2f0     sw_utilityG:sw_utilityG.dll
 0003:000002f4       __imp_StartPDSMLocNotifstatus 0003f2f4     sw_utilityG:sw_utilityG.dll
 0003:000002f8       __imp_?GetCarrierIndex@@YAKXZ 0003f2f8     sw_utilityG:sw_utilityG.dll
 0003:000002fc       __imp_EndLBTrackSession    0003f2fc     sw_utilityG:sw_utilityG.dll
 0003:00000300       __imp_ReadPDSMPAData       0003f300     sw_utilityG:sw_utilityG.dll
 0003:00000304       __imp_GetRilPDData         0003f304     sw_utilityG:sw_utilityG.dll
 0003:00000308       __imp_?InWideMode@@YAHXZ   0003f308     sw_utilityG:sw_utilityG.dll
 0003:0000030c       __imp_GetByteCounter       0003f30c     sw_utilityG:sw_utilityG.dll
 0003:00000310       __imp_SaveAkey             0003f310     sw_utilityG:sw_utilityG.dll
 0003:00000314       __imp_?SetLimitText@@YAJPAUHWND__@@H@Z 0003f314     sw_utilityG:sw_utilityG.dll
 0003:00000318       __imp_GetAdvancedMenuInfo  0003f318     sw_utilityG:sw_utilityG.dll
 0003:0000031c       __imp_SetEquipmentState    0003f31c     sw_utilityG:sw_utilityG.dll
 0003:00000320       __imp_ReadNv               0003f320     sw_utilityG:sw_utilityG.dll
 0003:00000324       __imp_?SetWaitCursor@@YAXXZ 0003f324     sw_utilityG:sw_utilityG.dll
 0003:00000328       __imp_?SetNormalCursor@@YAXXZ 0003f328     sw_utilityG:sw_utilityG.dll
 0003:0000032c       __imp_WriteNv              0003f32c     sw_utilityG:sw_utilityG.dll
 0003:00000330       __imp_?LogC@@YAXPBGZZ      0003f330     sw_utilityG:sw_utilityG.dll
 0003:00000334       __imp_?LogStoreFileLine@@YAXPAGH@Z 0003f334     sw_utilityG:sw_utilityG.dll
 0003:00000338       __imp_StartLBTrackSession  0003f338     sw_utilityG:sw_utilityG.dll
 0003:0000033c       \177sw_utilityG_NULL_THUNK_DATA 0003f33c     sw_utilityG:sw_utilityG.dll
 0003:00000340       __xc_a                     0003f340     corelibc:crt0init.obj
 0003:00000978       __xc_z                     0003f978     corelibc:crt0init.obj
 0003:0000097c       __xi_a                     0003f97c     corelibc:crt0init.obj
 0003:00000980       __xi_z                     0003f980     corelibc:crt0init.obj
 0003:00000984       __xp_a                     0003f984     corelibc:crt0init.obj
 0003:00000988       __xp_z                     0003f988     corelibc:crt0init.obj
 0003:0000098c       __xt_a                     0003f98c     corelibc:crt0init.obj
 0003:00000990       __xt_z                     0003f990     corelibc:crt0init.obj
 0003:00000998       ?g_szAdvanceClass@@3PAGA   0003f998     advanceddlg.obj
 0003:0000099c       ?g_szAuthKeyClass@@3PAGA   0003f99c     authkey.obj
 0003:000009a0       ?g_szBrowserDlgClass@@3PAGA 0003f9a0     browserdlg.obj
 0003:000009a4       ?g_szBWMeterClass@@3PAGA   0003f9a4     bwmeterdlg.obj
 0003:000009a8       ?g_fTxDiv@@3MA             0003f9a8     bwmeterdlg.obj
 0003:000009ac       ?g_fRxDiv@@3MA             0003f9ac     bwmeterdlg.obj
 0003:000009b0       ?szBWMList@@3PAPBGA        0003f9b0     bwmeterdlg.obj
 0003:000009c4       ?g_szConfigClass@@3PAGA    0003f9c4     configdlg.obj
 0003:000009c8       ?g_szEVDODlgClass@@3PAGA   0003f9c8     evdo.obj
 0003:000009cc       ?g_szFingerClass@@3PAGA    0003f9cc     finger.obj
 0003:000009d0       ?g_szGPSDataClass@@3PAGA   0003f9d0     gpsdatadlg.obj
 0003:000009d4       ?g_dwMaxDelay@@3KA         0003f9d4     gpsdatadlg.obj
 0003:000009d8       ?g_dwEditFixCount@@3KA     0003f9d8     gpsdatadlg.obj
 0003:000009dc       ?g_dwFixType@@3KA          0003f9dc     gpsdatadlg.obj
 0003:000009e0       ?g_bStart@@3HA             0003f9e0     gpsdatadlg.obj
 0003:000009e4       ?g_szGPSSettingsClass@@3PAGA 0003f9e4     gpssettingsdlg.obj
 0003:000009e8       ?g_szGSM2GClass@@3PAGA     0003f9e8     gsm2G.obj
 0003:000009ec       ?g_szGSM3GClass@@3PAGA     0003f9ec     gsm3G.obj
 0003:000009f0       ?g_szGSM3GItemnizeClass@@3PAGA 0003f9f0     gsm3G.obj
 0003:000009f4       ?g_szGSMBandClass@@3PAGA   0003f9f4     gsmband.obj
 0003:000009f8       ?g_szIOTAClass@@3PAGA      0003f9f8     iota.obj
 0003:000009fc       ?g_szLoopBackDlgClass@@3PAGA 0003f9fc     loopbackdlg.obj
 0003:00000a00       ?g_szMslClass@@3PAGA       0003fa00     msldlg.obj
 0003:00000a04       ?g_szNetworkClass@@3PAGA   0003fa04     network.obj
 0003:00000a08       ?g_szOtkslClass@@3PAGA     0003fa08     otksldlg.obj
 0003:00000a0c       ?g_szPassThruClass@@3PAGA  0003fa0c     passthrudlg.obj
 0003:00000a10       ?g_bPasstruStart@@3HA      0003fa10     passthrudlg.obj
 0003:00000a14       ?g_szAppWndClass@@3PBGB    0003fa14     phoneutility.obj
 0003:00000a18       ?g_szRTNClass@@3PAGA       0003fa18     rtndlg.obj
 0003:00000a1c       ?g_szSimpleIPClass@@3PAGA  0003fa1c     simpleipdlg.obj
 0003:00000a20       ?g_dwPreference@@3KA       0003fa20     simpleipdlg.obj
 0003:00000a24       ?szSimpleIPList@@3PAPBGA   0003fa24     simpleipdlg.obj
 0003:00000a30       ?g_szSipDlgClass@@3PAGA    0003fa30     sipdlg.obj
 0003:00000a34       ?g_szSPCValidationClass@@3PAGA 0003fa34     spcvalidation.obj
 0003:00000a38       ?g_szSystemDlgClass@@3PAGA 0003fa38     systemdlg.obj
 0003:00000a3c       ?g_szUsernameClass@@3PAGA  0003fa3c     usernamedlg.obj
 0003:00000a44       ?g_szVersionInfoDlgClass@@3PAGA 0003fa44     versioninfo.obj
 0003:00000a48       ?g_szVocoderDlgClass@@3PAGA 0003fa48     vocoderdlg.obj
 0003:00000a4c       ?g_wHomePageVoiceSO@@3GA   0003fa4c     vocoderdlg.obj
 0003:00000a50       ?g_wHomeOrigVoiceSO@@3GA   0003fa50     vocoderdlg.obj
 0003:00000a54       ?g_wRoamOrigVoiceSO@@3GA   0003fa54     vocoderdlg.obj
 0003:00000a58       __security_cookie_complement 0003fa58     corelibc:seccook.obj
 0003:00000a5c       __security_cookie          0003fa5c     corelibc:seccook.obj
 0003:00000a60       __lc_time_c                0003fa60     LIBCMT:strftime.obj
 0003:00000b18       __lc_time_curr             0003fb18     LIBCMT:strftime.obj
 0003:00000b38       _timezone                  0003fb38     LIBCMT:timeset.obj
 0003:00000b3c       _daylight                  0003fb3c     LIBCMT:timeset.obj
 0003:00000b40       _dstbias                   0003fb40     LIBCMT:timeset.obj
 0003:00000bc8       _tzname                    0003fbc8     LIBCMT:timeset.obj
 0003:00000bd0       __clocalestr               0003fbd0     LIBCMT:nlsdata2.obj
 0003:00000bd8       __initiallocinfo           0003fbd8     LIBCMT:nlsdata2.obj
 0003:00000ca8       __ptlocinfo                0003fca8     LIBCMT:nlsdata2.obj
 0003:00000cac       __lc_clike                 0003fcac     LIBCMT:nlsdata2.obj
 0003:00000cb0       _lpdays                    0003fcb0     LIBCMT:days.obj
 0003:00000ce4       _days                      0003fce4     LIBCMT:days.obj
 0003:00000e38       _pctype                    0003fe38     LIBCMT:ctype.obj
 0003:00000e3c       _pwctype                   0003fe3c     LIBCMT:ctype.obj
 0003:00000e40       __lconv_static_decimal     0003fe40     LIBCMT:lconv.obj
 0003:00000e44       __lconv_c                  0003fe44     LIBCMT:lconv.obj
 0003:00000e74       _aexit_rtn                 0003fe74     LIBCMT:crt0dat.obj
 0003:00000e78       ?g_szLockCode@@3PAGA       0003fe78     advanceddlg.obj
 0003:00001078       ?g_hWndLBOrg@@3PAUHWND__@@A 00040078     advanceddlg.obj
 0003:0000107c       ?g_hWndLBSID@@3PAUHWND__@@A 0004007c     advanceddlg.obj
 0003:00001080       ?g_hWndLBNID@@3PAUHWND__@@A 00040080     advanceddlg.obj
 0003:00001084       ?g_hWndLBHSys@@3PAUHWND__@@A 00040084     advanceddlg.obj
 0003:00001088       ?g_hWndCAIRev@@3PAUHWND__@@A 00040088     advanceddlg.obj
 0003:0000108c       ?g_hWndSCM@@3PAUHWND__@@A  0004008c     advanceddlg.obj
 0003:00001090       ?g_hWndCameraUrl@@3PAUHWND__@@A 00040090     advanceddlg.obj
 0003:00001094       ?g_hWndLockCode@@3PAUHWND__@@A 00040094     advanceddlg.obj
 0003:00001098       ?g_hWndNIDUPDOWN@@3PAUHWND__@@A 00040098     advanceddlg.obj
 0003:0000109c       ?g_hWndSIDUPDOWN@@3PAUHWND__@@A 0004009c     advanceddlg.obj
 0003:000010a0       ?g_hWndHSYSUPDOWN@@3PAUHWND__@@A 000400a0     advanceddlg.obj
 0003:000010a4       ?g_hWndORGUPDOWN@@3PAUHWND__@@A 000400a4     advanceddlg.obj
 0003:000010a8       ?g_hListDDTM@@3PAUHWND__@@A 000400a8     advanceddlg.obj
 0003:000010ac       ?g_dwAdvCAIRev@@3KA        000400ac     advanceddlg.obj
 0003:000010b0       ?g_dwHomeOrg@@3KA          000400b0     advanceddlg.obj
 0003:000010b4       ?g_dwFNID@@3HA             000400b4     advanceddlg.obj
 0003:000010b8       ?g_dwFSID@@3HA             000400b8     advanceddlg.obj
 0003:000010bc       ?g_dwHSYSReg@@3HA          000400bc     advanceddlg.obj
 0003:000010c0       ?g_dwSCM@@3KA              000400c0     advanceddlg.obj
 0003:000010c8       ?g_dwSaveResult@@3KA       000400c8     authkey.obj
 0003:000010cc       ?g_bMNCode@@3HA            000400cc     authkey.obj
 0003:000010d0       ?g_bAkey@@3HA              000400d0     authkey.obj
 0003:000010d4       ?g_hAkeyMenu@@3PAUHWND__@@A 000400d4     authkey.obj
 0003:000010e4       ?g_stRilByteCounterInfo@@3Urilbytecounter_tag@@A 000400e4     bwmeterdlg.obj
 0003:000010f8       ?g_stCallType@@3KA         000400f8     bwmeterdlg.obj
 0003:000010fc       ?g_hWndLBMaxRX@@3PAUHWND__@@A 000400fc     bwmeterdlg.obj
 0003:00001100       ?g_hWndLBMaxTX@@3PAUHWND__@@A 00040100     bwmeterdlg.obj
 0003:00001104       ?g_hThread@@3PAXA          00040104     bwmeterdlg.obj
 0003:00001108       ?g_dwRxNow@@3KA            00040108     bwmeterdlg.obj
 0003:0000110c       ?g_dwTxNow@@3KA            0004010c     bwmeterdlg.obj
 0003:00001110       ?g_dwCurrentHighRxCur@@3KA 00040110     bwmeterdlg.obj
 0003:00001114       ?g_dwCurrentHighTxCur@@3KA 00040114     bwmeterdlg.obj
 0003:00001118       ?g_dwRxCount@@3KA          00040118     bwmeterdlg.obj
 0003:0000111c       ?g_dwTxCount@@3KA          0004011c     bwmeterdlg.obj
 0003:00001120       ?g_dwHighTxAvg@@3KA        00040120     bwmeterdlg.obj
 0003:00001124       ?g_dwHighRxAvg@@3KA        00040124     bwmeterdlg.obj
 0003:00001128       ?g_hWndStatMaxTX@@3PAUHWND__@@A 00040128     bwmeterdlg.obj
 0003:0000112c       ?g_hWndStatMaxRX@@3PAUHWND__@@A 0004012c     bwmeterdlg.obj
 0003:00001130       ?g_hProgressTxAvg@@3PAUHWND__@@A 00040130     bwmeterdlg.obj
 0003:00001134       ?g_hProgressRxAvg@@3PAUHWND__@@A 00040134     bwmeterdlg.obj
 0003:00001138       ?g_hProgressTx@@3PAUHWND__@@A 00040138     bwmeterdlg.obj
 0003:0000113c       ?g_hProgressRx@@3PAUHWND__@@A 0004013c     bwmeterdlg.obj
 0003:00001140       ?g_hStaticTxVal@@3PAUHWND__@@A 00040140     bwmeterdlg.obj
 0003:00001144       ?g_hStaticRxVal@@3PAUHWND__@@A 00040144     bwmeterdlg.obj
 0003:00001148       ?g_hStaticTxAvg@@3PAUHWND__@@A 00040148     bwmeterdlg.obj
 0003:0000114c       ?g_hStaticRxAvg@@3PAUHWND__@@A 0004014c     bwmeterdlg.obj
 0003:00001150       ?g_hStaticHighTxCur@@3PAUHWND__@@A 00040150     bwmeterdlg.obj
 0003:00001154       ?g_hStaticHighTxAvg@@3PAUHWND__@@A 00040154     bwmeterdlg.obj
 0003:00001158       ?g_hStaticHighRxCur@@3PAUHWND__@@A 00040158     bwmeterdlg.obj
 0003:0000115c       ?g_hStaticHighRxAvg@@3PAUHWND__@@A 0004015c     bwmeterdlg.obj
 0003:00001160       ?g_hStaticTxBytes@@3PAUHWND__@@A 00040160     bwmeterdlg.obj
 0003:00001164       ?g_hStaticRxBytes@@3PAUHWND__@@A 00040164     bwmeterdlg.obj
 0003:00001168       ?g_fRxAvg@@3MA             00040168     bwmeterdlg.obj
 0003:0000116c       ?g_fTxAvg@@3MA             0004016c     bwmeterdlg.obj
 0003:00001170       ?g_bExitThread@@3_NA       00040170     bwmeterdlg.obj
 0003:00001174       ?g_dwRxBytes@@3KA          00040174     bwmeterdlg.obj
 0003:00001178       ?g_dwTxBytes@@3KA          00040178     bwmeterdlg.obj
 0003:00001270       ?g_PhUpdateEvdo@@3UCRITICAL_SECTION@@A 00040270     evdo.obj
 0003:00001284       ?g_hWndEvdoList@@3PAUHWND__@@A 00040284     evdo.obj
 0003:0000128c       ?g_hFingerList@@3PAUHWND__@@A 0004028c     finger.obj
 0003:00001290       ?g_hActivestList@@3PAUHWND__@@A 00040290     finger.obj
 0003:000012a0       ?g_szEditEndReason@@3PAGA  000402a0     gpsdatadlg.obj
 0003:00001750       ?g_szEditSessionStatus@@3PAGA 00040750     gpsdatadlg.obj
 0003:00001c00       ?g_szEditLongitude@@3PAGA  00040c00     gpsdatadlg.obj
 0003:000020b0       ?g_szEditLatitude@@3PAGA   000410b0     gpsdatadlg.obj
 0003:00002560       ?g_szEditLocTime@@3PAGA    00041560     gpsdatadlg.obj
 0003:00002a10       ?g_PDSMPDEndSession@@3UtagRILPDSMPDEndSession@@A 00041a10     gpsdatadlg.obj
 0003:00002a18       ?g_PDSMPDTrack@@3UtagRILPDSMPATrack@@A 00041a18     gpsdatadlg.obj
 0003:00002a30       ?g_PDSMPDData@@3UtagRILGETPAData@@A 00041a30     gpsdatadlg.obj
 0003:00002a6c       ?g_hEditStatus@@3PAUHWND__@@A 00041a6c     gpsdatadlg.obj
 0003:00002a70       ?g_hEditEndReason@@3PAUHWND__@@A 00041a70     gpsdatadlg.obj
 0003:00002a74       ?g_hEditTime@@3PAUHWND__@@A 00041a74     gpsdatadlg.obj
 0003:00002a78       ?g_hEditLatitude@@3PAUHWND__@@A 00041a78     gpsdatadlg.obj
 0003:00002a7c       ?g_hEditLongitude@@3PAUHWND__@@A 00041a7c     gpsdatadlg.obj
 0003:00002a80       ?g_hFixType@@3PAUHWND__@@A 00041a80     gpsdatadlg.obj
 0003:00002a84       ?g_hFixTypeUpDn@@3PAUHWND__@@A 00041a84     gpsdatadlg.obj
 0003:00002a88       ?g_hEditMaxDelay@@3PAUHWND__@@A 00041a88     gpsdatadlg.obj
 0003:00002a8c       ?g_hEDTMaxErrs@@3PAUHWND__@@A 00041a8c     gpsdatadlg.obj
 0003:00002a90       ?g_hEDTFixRate@@3PAUHWND__@@A 00041a90     gpsdatadlg.obj
 0003:00002a94       ?g_hEDTFixCt@@3PAUHWND__@@A 00041a94     gpsdatadlg.obj
 0003:00002a98       ?g_dwMaxError@@3KA         00041a98     gpsdatadlg.obj
 0003:00002a9c       ?g_dwEditFixRate@@3KA      00041a9c     gpsdatadlg.obj
 0003:00002ab4       ?g_stGetPDSMPAParam@@3UtagRILSETGETPAParam@@A 00041ab4     gpssettingsdlg.obj
 0003:00002ad8       ?g_hLBGPSLock@@3PAUHWND__@@A 00041ad8     gpssettingsdlg.obj
 0003:00002adc       ?g_hLBTMech@@3PAUHWND__@@A 00041adc     gpssettingsdlg.obj
 0003:00002ae0       ?g_hLBPrivacy@@3PAUHWND__@@A 00041ae0     gpssettingsdlg.obj
 0003:00002ae4       ?g_hLBNTACCSLVL@@3PAUHWND__@@A 00041ae4     gpssettingsdlg.obj
 0003:00002ae8       ?g_hLBGPSLockUPDN@@3PAUHWND__@@A 00041ae8     gpssettingsdlg.obj
 0003:00002aec       ?g_hLBTMechUPDN@@3PAUHWND__@@A 00041aec     gpssettingsdlg.obj
 0003:00002af0       ?g_hLBPrivacyUPDN@@3PAUHWND__@@A 00041af0     gpssettingsdlg.obj
 0003:00002af4       ?g_hLBNTACCSLVLUPDN@@3PAUHWND__@@A 00041af4     gpssettingsdlg.obj
 0003:00002af8       ?g_hEDTIP@@3PAUHWND__@@A   00041af8     gpssettingsdlg.obj
 0003:00002afc       ?g_hEDTPort@@3PAUHWND__@@A 00041afc     gpssettingsdlg.obj
 0003:00002b00       ?g_hFixRate@@3PAUHWND__@@A 00041b00     gpssettingsdlg.obj
 0003:00002b04       ?g_hAutoTrack@@3PAUHWND__@@A 00041b04     gpssettingsdlg.obj
 0003:00002b08       ?g_hFixMode@@3PAUHWND__@@A 00041b08     gpssettingsdlg.obj
 0003:00002b0c       ?g_u2GTimer@@3IA           00041b0c     gsm2G.obj
 0003:00002c00       ?g_u3GTimer@@3IA           00041c00     gsm3G.obj
 0003:00002c04       ?g_lIndex@@3JA             00041c04     gsm3G.obj
 0003:00002dec       ?m_hMenuConnect@@3PAUHWND__@@A 00041dec     loopbackdlg.obj
 0003:00002df0       ?m_hMenuDisConnect@@3PAUHWND__@@A 00041df0     loopbackdlg.obj
 0003:00002df4       ?g_hstatMsg@@3PAUHWND__@@A 00041df4     loopbackdlg.obj
 0003:00002df8       ?g_dwServiceOption@@3KA    00041df8     loopbackdlg.obj
 0003:00002e00       ?g_hActiveWindow@@3PAUHWND__@@A 00041e00     mainfrm.obj
 0003:00002e18       ?g_bNidOK@@3HA             00041e18     msldlg.obj
 0003:00002e1c       ?g_bMCCOK@@3HA             00041e1c     msldlg.obj
 0003:00002e20       ?g_bMNCOK@@3HA             00041e20     msldlg.obj
 0003:00002e24       ?g_bSidOK@@3HA             00041e24     msldlg.obj
 0003:00002e28       ?g_bMsidOK@@3HA            00041e28     msldlg.obj
 0003:00002e2c       ?g_bMDNOK@@3HA             00041e2c     msldlg.obj
 0003:00002e30       ?g_pMslInfo@@3UtagRILMSLINFO@@A 00041e30     msldlg.obj
 0003:00002eac       ?g_nPhoneNumLen@@3KA       00041eac     msldlg.obj
 0003:00002eb0       ?g_hMSLSaveMenu@@3PAUHWND__@@A 00041eb0     msldlg.obj
 0003:00002ebc       ?g_hWndNetworkList@@3PAUHWND__@@A 00041ebc     network.obj
 0003:00002ec8       ?g_bMsid@@3HA              00041ec8     otksldlg.obj
 0003:00002ecc       ?g_bMDN@@3HA               00041ecc     otksldlg.obj
 0003:00002ed0       ?g_pmslInfo@@3UtagRILMSLINFO@@A 00041ed0     otksldlg.obj
 0003:00002f4c       ?g_nphoneNumLen@@3KA       00041f4c     otksldlg.obj
 0003:00002f50       ?g_hOTKSLSaveMenu@@3PAUHWND__@@A 00041f50     otksldlg.obj
 0003:00002f60       ?g_stRilTechHdrInfo@@3USW_RILTECHHDRINFO@@A 00041f60     phoneutility.obj
 0003:00002ff8       ?g_stRilDbgInfo@@3UtagRILMODEMDEBUGINFO@@A 00041ff8     phoneutility.obj
 0003:000030d4       ?g_NoAAMResponseId@@3IA    000420d4     phoneutility.obj
 0003:000030d8       ?g_Err@@3UtagErrorInfo@@A  000420d8     phoneutility.obj
 0003:000032e0       ?g_bGrp@@3HA               000422e0     phoneutility.obj
 0003:000032e4       ?g_bSPCValidated@@3HA      000422e4     phoneutility.obj
 0003:000032e8       ?g_dwSPC@@3KA              000422e8     phoneutility.obj
 0003:000032ec       ?g_dwActiveTab@@3KA        000422ec     phoneutility.obj
 0003:000032f0       ?g_stRilStatus@@3USW_RILStatus@@A 000422f0     phoneutility.obj
 0003:00003330       ?g_strMSL@@3PAGA           00042330     phoneutility.obj
 0003:000037e0       ?g_szCmdLine@@3PAGA        000427e0     phoneutility.obj
 0003:00003c90       ?g_szMessage@@3PAGA        00042c90     phoneutility.obj
 0003:00004140       ?g_pszTitle@@3PAGA         00043140     phoneutility.obj
 0003:000045f0       ?g_pszAppName@@3PAGA       000435f0     phoneutility.obj
 0003:00004aa0       ?g_hWndMain@@3PAUHWND__@@A 00043aa0     phoneutility.obj
 0003:00004aa4       ?g_dwSpMode@@3KA           00043aa4     phoneutility.obj
 0003:00004aa8       ?g_nCarrier@@3KA           00043aa8     phoneutility.obj
 0003:00004aac       ?g_hResInst@@3PAUHINSTANCE__@@A 00043aac     phoneutility.obj
 0003:00004ab0       ?g_hInst@@3PAUHINSTANCE__@@A 00043ab0     phoneutility.obj
 0003:00004ab4       ?g_hWndListView@@3PAUHWND__@@A 00043ab4     phoneutility.obj
 0003:00004ab8       ?g_bDbgMode@@3HA           00043ab8     phoneutility.obj
 0003:00004abc       ?g_dwRtnOrClear@@3KA       00043abc     phoneutility.obj
 0003:00004ac8       ?g_szPass@@3PAGA           00043ac8     simpleipdlg.obj
 0003:00004f78       ?g_szUname@@3PAGA          00043f78     simpleipdlg.obj
 0003:00005430       ?g_hSpcMenu@@3PAUHWND__@@A 00044430     spcvalidation.obj
 0003:0000552c       ?g_dwCAIRev@@3KA           0004452c     systemdlg.obj
 0003:00005530       ?g_dwRoamMode@@3KA         00044530     systemdlg.obj
 0003:00005538       ?g_szHdrPass@@3PAGA        00044538     usernamedlg.obj
 0003:000059e8       ?g_szHdrUname@@3PAGA       000449e8     usernamedlg.obj
 0003:00005e98       ?g_stPDPList@@3UtagRILPDPLIST@@A 00044e98     usernamedlg.obj
 0003:00005eb8       ?g_stPDPPayload@@3UtagRILPDPPAYLOAD@@A 00044eb8     usernamedlg.obj
 0003:00005fb8       ?g_stcurrentPDP@@3UtagRILGETORSETPDP@@A 00044fb8     usernamedlg.obj
 0003:000060b8       ?g_nNumOfProfiles@@3HA     000450b8     usernamedlg.obj
 0003:000060bc       ?g_bChk@@3HA               000450bc     usernamedlg.obj
 0003:000060c0       ?g_hWndSPIMNAA@@3PAUHWND__@@A 000450c0     usernamedlg.obj
 0003:000060c4       ?g_hWndSPIMNHA@@3PAUHWND__@@A 000450c4     usernamedlg.obj
 0003:000060c8       ?g_hWndMNASSecret@@3PAUHWND__@@A 000450c8     usernamedlg.obj
 0003:000060cc       ?g_hWndMNHASSecret@@3PAUHWND__@@A 000450cc     usernamedlg.obj
 0003:000060d0       ?g_hWndUNai@@3PAUHWND__@@A 000450d0     usernamedlg.obj
 0003:000060d4       ?g_hWndRTunnel@@3PAUHWND__@@A 000450d4     usernamedlg.obj
 0003:000060d8       ?g_hWndSHomeAgent@@3PAUHWND__@@A 000450d8     usernamedlg.obj
 0003:000060dc       ?g_hWndPHomeAgent@@3PAUHWND__@@A 000450dc     usernamedlg.obj
 0003:000060e0       ?g_hWndHomeAgent@@3PAUHWND__@@A 000450e0     usernamedlg.obj
 0003:000060e4       ?g_hWndChkHex@@3PAUHWND__@@A 000450e4     usernamedlg.obj
 0003:000060e8       ?g_hWndPDPList@@3PAUHWND__@@A 000450e8     usernamedlg.obj
 0003:000060ec       ?g_hWndActivePDP@@3PAUHWND__@@A 000450ec     usernamedlg.obj
 0003:000060f0       ?g_hWndHdrAAASSecret@@3PAUHWND__@@A 000450f0     usernamedlg.obj
 0003:000060f4       ?g_hWndHdrNai@@3PAUHWND__@@A 000450f4     usernamedlg.obj
 0003:00006100       ?g_VersionInfo@@3UtagRILVERNOINFO@@A 00045100     versioninfo.obj
 0003:00006e00       ?m_hMenuVocoder@@3PAUHWND__@@A 00045e00     vocoderdlg.obj
 0003:00006e04       ?g_namID@@3EA              00045e04     vocoderdlg.obj
 0003:00006e08       ?g_bEvrcEnabled@@3HA       00045e08     vocoderdlg.obj
 0003:00006ed0       __lc_handle                00045ed0     LIBCMT:nlsdata2.obj
 0003:00006ee8       __lc_codepage              00045ee8     LIBCMT:nlsdata2.obj
 0003:00006eec       __lc_collate_cp            00045eec     LIBCMT:nlsdata2.obj
 0003:0000700c       __lconv_static_null        0004600c     LIBCMT:lconv.obj
 0003:00007014       __onexitend                00046014     <common>
 0003:00007018       __onexitbegin              00046018     <common>
 0003:0000701c       _exitflag                  0004601c     <common>

 entry point at        0001:0001683c

 Static symbols

 0001:00016974       doexit                     00027974 f   corelibc:crt0dat.obj
 0001:00016b70       _wcsftime_l_stat           00027b70 f   LIBCMT:wcsftime.obj
 0001:00017258       _store_str                 00028258 f   LIBCMT:strftime.obj
 0001:000172a4       _store_num                 000282a4 f   LIBCMT:strftime.obj
 0001:000173bc       _expandtime                000283bc f   LIBCMT:strftime.obj
 0001:00017e24       _store_winword             00028e24 f   LIBCMT:strftime.obj
 0001:000189a8       _tzset_nolock              000299a8 f   LIBCMT:tzset.obj
 0001:00018c70       cvtdate                    00029c70 f   LIBCMT:tzset.obj
 0001:00018f98       _isindst_nolock            00029f98 f   LIBCMT:tzset.obj
 0001:00019b3c       __crtInitCritSecNoSpinCount 0002ab3c f   LIBCMT:initcrit.obj
 0001:00019d08       ??__ERIL_STATUS_CHANGED@@YAXXZ 0002ad08 f   advanceddlg.obj
 0001:00019d28       ??__EPHONEUTILS_END_MESSAGE@@YAXXZ 0002ad28 f   authkey.obj
 0001:00019d48       ??__ERIL_STATUS_CHANGED@@YAXXZ 0002ad48 f   authkey.obj
 0001:00019d68       ??__ERIL_STATUS_CHANGED@@YAXXZ 0002ad68 f   browserdlg.obj
 0001:00019d88       ??__ERIL_STATUS_CHANGED@@YAXXZ 0002ad88 f   bwmeterdlg.obj
 0001:00019da8       ??__EPOWER_ON@@YAXXZ       0002ada8 f   configdlg.obj
 0001:00019dc8       ??__EPOWER_OFF@@YAXXZ      0002adc8 f   configdlg.obj
 0001:00019de8       ??__EIOTA_BEGIN_MESSAGE@@YAXXZ 0002ade8 f   configdlg.obj
 0001:00019e08       ??__EIOTA_END_MESSAGE@@YAXXZ 0002ae08 f   configdlg.obj
 0001:00019e28       ??__EIOTA_BEGIN_ACK@@YAXXZ 0002ae28 f   configdlg.obj
 0001:00019e48       ??__EIOTA_BEGIN_NACK@@YAXXZ 0002ae48 f   configdlg.obj
 0001:00019e68       ??__EIOTA_END_ACK@@YAXXZ   0002ae68 f   configdlg.obj
 0001:00019e88       ??__EIOTA_EXIT_MESSAGE@@YAXXZ 0002ae88 f   configdlg.obj
 0001:00019ea8       ??__EIOTA_ALIVE_MESSAGE@@YAXXZ 0002aea8 f   configdlg.obj
 0001:00019ec8       ??__EIOTA_PING_MESSAGE@@YAXXZ 0002aec8 f   configdlg.obj
 0001:00019ee8       ??__EIOTA_PING_ACK@@YAXXZ  0002aee8 f   configdlg.obj
 0001:00019f08       ??__EIOTA_CRITICAL_ERROR@@YAXXZ 0002af08 f   configdlg.obj
 0001:00019f28       ??__EIOTA_NON_CRITICAL_ERROR@@YAXXZ 0002af28 f   configdlg.obj
 0001:00019f48       ??__EIOTA_KILL_ME@@YAXXZ   0002af48 f   configdlg.obj
 0001:00019f68       ??__EIOTA_UPDATE_STATUS@@YAXXZ 0002af68 f   configdlg.obj
 0001:00019f88       ??__EIOTA_DATAPORT_INUSE@@YAXXZ 0002af88 f   configdlg.obj
 0001:00019fa8       ??__EIOTA_DONE@@YAXXZ      0002afa8 f   configdlg.obj
 0001:00019fc8       ??__EIOTA_DIAL@@YAXXZ      0002afc8 f   configdlg.obj
 0001:00019fe8       ??__EIOTA_1012_MIP_ERR@@YAXXZ 0002afe8 f   configdlg.obj
 0001:0001a008       ??__EPHONEUTILS_BEGIN_MESSAGE@@YAXXZ 0002b008 f   configdlg.obj
 0001:0001a028       ??__EPHONEUTILS_END_MESSAGE@@YAXXZ 0002b028 f   configdlg.obj
 0001:0001a048       ??__EPHONEUTILS_BEGIN_ACK@@YAXXZ 0002b048 f   configdlg.obj
 0001:0001a068       ??__EPHONEUTILS_BEGIN_NACK@@YAXXZ 0002b068 f   configdlg.obj
 0001:0001a088       ??__EPHONEUTILS_END_ACK@@YAXXZ 0002b088 f   configdlg.obj
 0001:0001a0a8       ??__EPHONEUTILS_EXIT_MESSAGE@@YAXXZ 0002b0a8 f   configdlg.obj
 0001:0001a0c8       ??__EPHONEUTILS_ALIVE_MESSAGE@@YAXXZ 0002b0c8 f   configdlg.obj
 0001:0001a0e8       ??__EPHONEUTILS_PING_MESSAGE@@YAXXZ 0002b0e8 f   configdlg.obj
 0001:0001a108       ??__EPHONEUTILS_PING_ACK@@YAXXZ 0002b108 f   configdlg.obj
 0001:0001a128       ??__EAW_BEGIN_MESSAGE@@YAXXZ 0002b128 f   configdlg.obj
 0001:0001a148       ??__EAW_END_MESSAGE@@YAXXZ 0002b148 f   configdlg.obj
 0001:0001a168       ??__EAW_BEGIN_ACK@@YAXXZ   0002b168 f   configdlg.obj
 0001:0001a188       ??__EAW_BEGIN_NACK@@YAXXZ  0002b188 f   configdlg.obj
 0001:0001a1a8       ??__EAW_END_ACK@@YAXXZ     0002b1a8 f   configdlg.obj
 0001:0001a1c8       ??__EAW_EXIT_MESSAGE@@YAXXZ 0002b1c8 f   configdlg.obj
 0001:0001a1e8       ??__EAW_ALIVE_MESSAGE@@YAXXZ 0002b1e8 f   configdlg.obj
 0001:0001a208       ??__EAW_PING_MESSAGE@@YAXXZ 0002b208 f   configdlg.obj
 0001:0001a228       ??__EAW_PING_ACK@@YAXXZ    0002b228 f   configdlg.obj
 0001:0001a248       ??__EUPDATER_BEGIN@@YAXXZ  0002b248 f   configdlg.obj
 0001:0001a268       ??__EUPDATER_END@@YAXXZ    0002b268 f   configdlg.obj
 0001:0001a288       ??__EUPDATER_BEGIN_ACK@@YAXXZ 0002b288 f   configdlg.obj
 0001:0001a2a8       ??__EUPDATER_BEGIN_NACK@@YAXXZ 0002b2a8 f   configdlg.obj
 0001:0001a2c8       ??__EUPDATER_END_ACK@@YAXXZ 0002b2c8 f   configdlg.obj
 0001:0001a2e8       ??__EUPDATER_END_NACK@@YAXXZ 0002b2e8 f   configdlg.obj
 0001:0001a308       ??__ERIL_STATUS_CHANGED@@YAXXZ 0002b308 f   configdlg.obj
 0001:0001a328       ??__ERIL_DBG_NOTIFY@@YAXXZ 0002b328 f   configdlg.obj
 0001:0001a348       ??__ERIL_TECHHDR_NOTIFY@@YAXXZ 0002b348 f   configdlg.obj
 0001:0001a368       ??__ERIL_IOTA_STATUS_CHANGED@@YAXXZ 0002b368 f   configdlg.obj
 0001:0001a388       ??__ERIL_IOTA_WAP_URI@@YAXXZ 0002b388 f   configdlg.obj
 0001:0001a3a8       ??__ERIL_PDSM_PD_DATA@@YAXXZ 0002b3a8 f   configdlg.obj
 0001:0001a3c8       ??__ERIL_PDSM_PD_DONE@@YAXXZ 0002b3c8 f   configdlg.obj
 0001:0001a3e8       ??__ERIL_PDSM_PD_END@@YAXXZ 0002b3e8 f   configdlg.obj
 0001:0001a408       ??__ERIL_PDSM_PD_BEGIN@@YAXXZ 0002b408 f   configdlg.obj
 0001:0001a428       ??__ERIL_PDSM_PD_UPDATE_FAILURE@@YAXXZ 0002b428 f   configdlg.obj
 0001:0001a448       ??__ERIL_PDSM_PD_DLD_DATA@@YAXXZ 0002b448 f   configdlg.obj
 0001:0001a468       ??__ERIL_PDSM_PD_DLD_DONE@@YAXXZ 0002b468 f   configdlg.obj
 0001:0001a488       ??__ERIL_PDSM_PD_DLD_END@@YAXXZ 0002b488 f   configdlg.obj
 0001:0001a4a8       ??__ERIL_PDSM_PD_DLD_BEGIN@@YAXXZ 0002b4a8 f   configdlg.obj
 0001:0001a4c8       ??__ERIL_PDSM_PA_PARAM@@YAXXZ 0002b4c8 f   configdlg.obj
 0001:0001a4e8       ??__ERIL_CALL_BYTE_CTR@@YAXXZ 0002b4e8 f   configdlg.obj
 0001:0001a508       ??__ERIL_CREATE_MAIN_LIST@@YAXXZ 0002b508 f   configdlg.obj
 0001:0001a528       ??__ERIL_STATUS_CHANGED@@YAXXZ 0002b528 f   evdo.obj
 0001:0001a548       ??__ERIL_STATUS_CHANGED@@YAXXZ 0002b548 f   finger.obj
 0001:0001a568       ??__ERIL_DBG_NOTIFY@@YAXXZ 0002b568 f   finger.obj
 0001:0001a588       ??__ERIL_PDSM_PD_DATA@@YAXXZ 0002b588 f   gpsdatadlg.obj
 0001:0001a5a8       ??__ERIL_PDSM_PD_DONE@@YAXXZ 0002b5a8 f   gpsdatadlg.obj
 0001:0001a5c8       ??__ERIL_PDSM_PD_END@@YAXXZ 0002b5c8 f   gpsdatadlg.obj
 0001:0001a5e8       ??__ERIL_PDSM_PD_BEGIN@@YAXXZ 0002b5e8 f   gpsdatadlg.obj
 0001:0001a608       ??__ERIL_PDSM_PD_UPDATE_FAILURE@@YAXXZ 0002b608 f   gpsdatadlg.obj
 0001:0001a628       ??__EPOWER_ON@@YAXXZ       0002b628 f   gsm2G.obj
 0001:0001a648       ??__EPOWER_OFF@@YAXXZ      0002b648 f   gsm2G.obj
 0001:0001a668       ??__EIOTA_BEGIN_MESSAGE@@YAXXZ 0002b668 f   gsm2G.obj
 0001:0001a688       ??__EIOTA_END_MESSAGE@@YAXXZ 0002b688 f   gsm2G.obj
 0001:0001a6a8       ??__EIOTA_BEGIN_ACK@@YAXXZ 0002b6a8 f   gsm2G.obj
 0001:0001a6c8       ??__EIOTA_BEGIN_NACK@@YAXXZ 0002b6c8 f   gsm2G.obj
 0001:0001a6e8       ??__EIOTA_END_ACK@@YAXXZ   0002b6e8 f   gsm2G.obj
 0001:0001a708       ??__EIOTA_EXIT_MESSAGE@@YAXXZ 0002b708 f   gsm2G.obj
 0001:0001a728       ??__EIOTA_ALIVE_MESSAGE@@YAXXZ 0002b728 f   gsm2G.obj
 0001:0001a748       ??__EIOTA_PING_MESSAGE@@YAXXZ 0002b748 f   gsm2G.obj
 0001:0001a768       ??__EIOTA_PING_ACK@@YAXXZ  0002b768 f   gsm2G.obj
 0001:0001a788       ??__EIOTA_CRITICAL_ERROR@@YAXXZ 0002b788 f   gsm2G.obj
 0001:0001a7a8       ??__EIOTA_NON_CRITICAL_ERROR@@YAXXZ 0002b7a8 f   gsm2G.obj
 0001:0001a7c8       ??__EIOTA_KILL_ME@@YAXXZ   0002b7c8 f   gsm2G.obj
 0001:0001a7e8       ??__EIOTA_UPDATE_STATUS@@YAXXZ 0002b7e8 f   gsm2G.obj
 0001:0001a808       ??__EIOTA_DATAPORT_INUSE@@YAXXZ 0002b808 f   gsm2G.obj
 0001:0001a828       ??__EIOTA_DONE@@YAXXZ      0002b828 f   gsm2G.obj
 0001:0001a848       ??__EIOTA_DIAL@@YAXXZ      0002b848 f   gsm2G.obj
 0001:0001a868       ??__EIOTA_1012_MIP_ERR@@YAXXZ 0002b868 f   gsm2G.obj
 0001:0001a888       ??__EPHONEUTILS_BEGIN_MESSAGE@@YAXXZ 0002b888 f   gsm2G.obj
 0001:0001a8a8       ??__EPHONEUTILS_END_MESSAGE@@YAXXZ 0002b8a8 f   gsm2G.obj
 0001:0001a8c8       ??__EPHONEUTILS_BEGIN_ACK@@YAXXZ 0002b8c8 f   gsm2G.obj
 0001:0001a8e8       ??__EPHONEUTILS_BEGIN_NACK@@YAXXZ 0002b8e8 f   gsm2G.obj
 0001:0001a908       ??__EPHONEUTILS_END_ACK@@YAXXZ 0002b908 f   gsm2G.obj
 0001:0001a928       ??__EPHONEUTILS_EXIT_MESSAGE@@YAXXZ 0002b928 f   gsm2G.obj
 0001:0001a948       ??__EPHONEUTILS_ALIVE_MESSAGE@@YAXXZ 0002b948 f   gsm2G.obj
 0001:0001a968       ??__EPHONEUTILS_PING_MESSAGE@@YAXXZ 0002b968 f   gsm2G.obj
 0001:0001a988       ??__EPHONEUTILS_PING_ACK@@YAXXZ 0002b988 f   gsm2G.obj
 0001:0001a9a8       ??__EAW_BEGIN_MESSAGE@@YAXXZ 0002b9a8 f   gsm2G.obj
 0001:0001a9c8       ??__EAW_END_MESSAGE@@YAXXZ 0002b9c8 f   gsm2G.obj
 0001:0001a9e8       ??__EAW_BEGIN_ACK@@YAXXZ   0002b9e8 f   gsm2G.obj
 0001:0001aa08       ??__EAW_BEGIN_NACK@@YAXXZ  0002ba08 f   gsm2G.obj
 0001:0001aa28       ??__EAW_END_ACK@@YAXXZ     0002ba28 f   gsm2G.obj
 0001:0001aa48       ??__EAW_EXIT_MESSAGE@@YAXXZ 0002ba48 f   gsm2G.obj
 0001:0001aa68       ??__EAW_ALIVE_MESSAGE@@YAXXZ 0002ba68 f   gsm2G.obj
 0001:0001aa88       ??__EAW_PING_MESSAGE@@YAXXZ 0002ba88 f   gsm2G.obj
 0001:0001aaa8       ??__EAW_PING_ACK@@YAXXZ    0002baa8 f   gsm2G.obj
 0001:0001aac8       ??__EUPDATER_BEGIN@@YAXXZ  0002bac8 f   gsm2G.obj
 0001:0001aae8       ??__EUPDATER_END@@YAXXZ    0002bae8 f   gsm2G.obj
 0001:0001ab08       ??__EUPDATER_BEGIN_ACK@@YAXXZ 0002bb08 f   gsm2G.obj
 0001:0001ab28       ??__EUPDATER_BEGIN_NACK@@YAXXZ 0002bb28 f   gsm2G.obj
 0001:0001ab48       ??__EUPDATER_END_ACK@@YAXXZ 0002bb48 f   gsm2G.obj
 0001:0001ab68       ??__EUPDATER_END_NACK@@YAXXZ 0002bb68 f   gsm2G.obj
 0001:0001ab88       ??__ERIL_STATUS_CHANGED@@YAXXZ 0002bb88 f   gsm2G.obj
 0001:0001aba8       ??__ERIL_DBG_NOTIFY@@YAXXZ 0002bba8 f   gsm2G.obj
 0001:0001abc8       ??__ERIL_TECHHDR_NOTIFY@@YAXXZ 0002bbc8 f   gsm2G.obj
 0001:0001abe8       ??__ERIL_IOTA_STATUS_CHANGED@@YAXXZ 0002bbe8 f   gsm2G.obj
 0001:0001ac08       ??__ERIL_IOTA_WAP_URI@@YAXXZ 0002bc08 f   gsm2G.obj
 0001:0001ac28       ??__ERIL_PDSM_PD_DATA@@YAXXZ 0002bc28 f   gsm2G.obj
 0001:0001ac48       ??__ERIL_PDSM_PD_DONE@@YAXXZ 0002bc48 f   gsm2G.obj
 0001:0001ac68       ??__ERIL_PDSM_PD_END@@YAXXZ 0002bc68 f   gsm2G.obj
 0001:0001ac88       ??__ERIL_PDSM_PD_BEGIN@@YAXXZ 0002bc88 f   gsm2G.obj
 0001:0001aca8       ??__ERIL_PDSM_PD_UPDATE_FAILURE@@YAXXZ 0002bca8 f   gsm2G.obj
 0001:0001acc8       ??__ERIL_PDSM_PD_DLD_DATA@@YAXXZ 0002bcc8 f   gsm2G.obj
 0001:0001ace8       ??__ERIL_PDSM_PD_DLD_DONE@@YAXXZ 0002bce8 f   gsm2G.obj
 0001:0001ad08       ??__ERIL_PDSM_PD_DLD_END@@YAXXZ 0002bd08 f   gsm2G.obj
 0001:0001ad28       ??__ERIL_PDSM_PD_DLD_BEGIN@@YAXXZ 0002bd28 f   gsm2G.obj
 0001:0001ad48       ??__ERIL_PDSM_PA_PARAM@@YAXXZ 0002bd48 f   gsm2G.obj
 0001:0001ad68       ??__ERIL_CALL_BYTE_CTR@@YAXXZ 0002bd68 f   gsm2G.obj
 0001:0001ad88       ??__ERIL_CREATE_MAIN_LIST@@YAXXZ 0002bd88 f   gsm2G.obj
 0001:0001ada8       ??__EPOWER_ON@@YAXXZ       0002bda8 f   gsm3G.obj
 0001:0001adc8       ??__EPOWER_OFF@@YAXXZ      0002bdc8 f   gsm3G.obj
 0001:0001ade8       ??__EIOTA_BEGIN_MESSAGE@@YAXXZ 0002bde8 f   gsm3G.obj
 0001:0001ae08       ??__EIOTA_END_MESSAGE@@YAXXZ 0002be08 f   gsm3G.obj
 0001:0001ae28       ??__EIOTA_BEGIN_ACK@@YAXXZ 0002be28 f   gsm3G.obj
 0001:0001ae48       ??__EIOTA_BEGIN_NACK@@YAXXZ 0002be48 f   gsm3G.obj
 0001:0001ae68       ??__EIOTA_END_ACK@@YAXXZ   0002be68 f   gsm3G.obj
 0001:0001ae88       ??__EIOTA_EXIT_MESSAGE@@YAXXZ 0002be88 f   gsm3G.obj
 0001:0001aea8       ??__EIOTA_ALIVE_MESSAGE@@YAXXZ 0002bea8 f   gsm3G.obj
 0001:0001aec8       ??__EIOTA_PING_MESSAGE@@YAXXZ 0002bec8 f   gsm3G.obj
 0001:0001aee8       ??__EIOTA_PING_ACK@@YAXXZ  0002bee8 f   gsm3G.obj
 0001:0001af08       ??__EIOTA_CRITICAL_ERROR@@YAXXZ 0002bf08 f   gsm3G.obj
 0001:0001af28       ??__EIOTA_NON_CRITICAL_ERROR@@YAXXZ 0002bf28 f   gsm3G.obj
 0001:0001af48       ??__EIOTA_KILL_ME@@YAXXZ   0002bf48 f   gsm3G.obj
 0001:0001af68       ??__EIOTA_UPDATE_STATUS@@YAXXZ 0002bf68 f   gsm3G.obj
 0001:0001af88       ??__EIOTA_DATAPORT_INUSE@@YAXXZ 0002bf88 f   gsm3G.obj
 0001:0001afa8       ??__EIOTA_DONE@@YAXXZ      0002bfa8 f   gsm3G.obj
 0001:0001afc8       ??__EIOTA_DIAL@@YAXXZ      0002bfc8 f   gsm3G.obj
 0001:0001afe8       ??__EIOTA_1012_MIP_ERR@@YAXXZ 0002bfe8 f   gsm3G.obj
 0001:0001b008       ??__EPHONEUTILS_BEGIN_MESSAGE@@YAXXZ 0002c008 f   gsm3G.obj
 0001:0001b028       ??__EPHONEUTILS_END_MESSAGE@@YAXXZ 0002c028 f   gsm3G.obj
 0001:0001b048       ??__EPHONEUTILS_BEGIN_ACK@@YAXXZ 0002c048 f   gsm3G.obj
 0001:0001b068       ??__EPHONEUTILS_BEGIN_NACK@@YAXXZ 0002c068 f   gsm3G.obj
 0001:0001b088       ??__EPHONEUTILS_END_ACK@@YAXXZ 0002c088 f   gsm3G.obj
 0001:0001b0a8       ??__EPHONEUTILS_EXIT_MESSAGE@@YAXXZ 0002c0a8 f   gsm3G.obj
 0001:0001b0c8       ??__EPHONEUTILS_ALIVE_MESSAGE@@YAXXZ 0002c0c8 f   gsm3G.obj
 0001:0001b0e8       ??__EPHONEUTILS_PING_MESSAGE@@YAXXZ 0002c0e8 f   gsm3G.obj
 0001:0001b108       ??__EPHONEUTILS_PING_ACK@@YAXXZ 0002c108 f   gsm3G.obj
 0001:0001b128       ??__EAW_BEGIN_MESSAGE@@YAXXZ 0002c128 f   gsm3G.obj
 0001:0001b148       ??__EAW_END_MESSAGE@@YAXXZ 0002c148 f   gsm3G.obj
 0001:0001b168       ??__EAW_BEGIN_ACK@@YAXXZ   0002c168 f   gsm3G.obj
 0001:0001b188       ??__EAW_BEGIN_NACK@@YAXXZ  0002c188 f   gsm3G.obj
 0001:0001b1a8       ??__EAW_END_ACK@@YAXXZ     0002c1a8 f   gsm3G.obj
 0001:0001b1c8       ??__EAW_EXIT_MESSAGE@@YAXXZ 0002c1c8 f   gsm3G.obj
 0001:0001b1e8       ??__EAW_ALIVE_MESSAGE@@YAXXZ 0002c1e8 f   gsm3G.obj
 0001:0001b208       ??__EAW_PING_MESSAGE@@YAXXZ 0002c208 f   gsm3G.obj
 0001:0001b228       ??__EAW_PING_ACK@@YAXXZ    0002c228 f   gsm3G.obj
 0001:0001b248       ??__EUPDATER_BEGIN@@YAXXZ  0002c248 f   gsm3G.obj
 0001:0001b268       ??__EUPDATER_END@@YAXXZ    0002c268 f   gsm3G.obj
 0001:0001b288       ??__EUPDATER_BEGIN_ACK@@YAXXZ 0002c288 f   gsm3G.obj
 0001:0001b2a8       ??__EUPDATER_BEGIN_NACK@@YAXXZ 0002c2a8 f   gsm3G.obj
 0001:0001b2c8       ??__EUPDATER_END_ACK@@YAXXZ 0002c2c8 f   gsm3G.obj
 0001:0001b2e8       ??__EUPDATER_END_NACK@@YAXXZ 0002c2e8 f   gsm3G.obj
 0001:0001b308       ??__ERIL_STATUS_CHANGED@@YAXXZ 0002c308 f   gsm3G.obj
 0001:0001b328       ??__ERIL_DBG_NOTIFY@@YAXXZ 0002c328 f   gsm3G.obj
 0001:0001b348       ??__ERIL_TECHHDR_NOTIFY@@YAXXZ 0002c348 f   gsm3G.obj
 0001:0001b368       ??__ERIL_IOTA_STATUS_CHANGED@@YAXXZ 0002c368 f   gsm3G.obj
 0001:0001b388       ??__ERIL_IOTA_WAP_URI@@YAXXZ 0002c388 f   gsm3G.obj
 0001:0001b3a8       ??__ERIL_PDSM_PD_DATA@@YAXXZ 0002c3a8 f   gsm3G.obj
 0001:0001b3c8       ??__ERIL_PDSM_PD_DONE@@YAXXZ 0002c3c8 f   gsm3G.obj
 0001:0001b3e8       ??__ERIL_PDSM_PD_END@@YAXXZ 0002c3e8 f   gsm3G.obj
 0001:0001b408       ??__ERIL_PDSM_PD_BEGIN@@YAXXZ 0002c408 f   gsm3G.obj
 0001:0001b428       ??__ERIL_PDSM_PD_UPDATE_FAILURE@@YAXXZ 0002c428 f   gsm3G.obj
 0001:0001b448       ??__ERIL_PDSM_PD_DLD_DATA@@YAXXZ 0002c448 f   gsm3G.obj
 0001:0001b468       ??__ERIL_PDSM_PD_DLD_DONE@@YAXXZ 0002c468 f   gsm3G.obj
 0001:0001b488       ??__ERIL_PDSM_PD_DLD_END@@YAXXZ 0002c488 f   gsm3G.obj
 0001:0001b4a8       ??__ERIL_PDSM_PD_DLD_BEGIN@@YAXXZ 0002c4a8 f   gsm3G.obj
 0001:0001b4c8       ??__ERIL_PDSM_PA_PARAM@@YAXXZ 0002c4c8 f   gsm3G.obj
 0001:0001b4e8       ??__ERIL_CALL_BYTE_CTR@@YAXXZ 0002c4e8 f   gsm3G.obj
 0001:0001b508       ??__ERIL_CREATE_MAIN_LIST@@YAXXZ 0002c508 f   gsm3G.obj
 0001:0001b528       ??__EPOWER_ON@@YAXXZ       0002c528 f   gsmband.obj
 0001:0001b548       ??__EPOWER_OFF@@YAXXZ      0002c548 f   gsmband.obj
 0001:0001b568       ??__EIOTA_BEGIN_MESSAGE@@YAXXZ 0002c568 f   gsmband.obj
 0001:0001b588       ??__EIOTA_END_MESSAGE@@YAXXZ 0002c588 f   gsmband.obj
 0001:0001b5a8       ??__EIOTA_BEGIN_ACK@@YAXXZ 0002c5a8 f   gsmband.obj
 0001:0001b5c8       ??__EIOTA_BEGIN_NACK@@YAXXZ 0002c5c8 f   gsmband.obj
 0001:0001b5e8       ??__EIOTA_END_ACK@@YAXXZ   0002c5e8 f   gsmband.obj
 0001:0001b608       ??__EIOTA_EXIT_MESSAGE@@YAXXZ 0002c608 f   gsmband.obj
 0001:0001b628       ??__EIOTA_ALIVE_MESSAGE@@YAXXZ 0002c628 f   gsmband.obj
 0001:0001b648       ??__EIOTA_PING_MESSAGE@@YAXXZ 0002c648 f   gsmband.obj
 0001:0001b668       ??__EIOTA_PING_ACK@@YAXXZ  0002c668 f   gsmband.obj
 0001:0001b688       ??__EIOTA_CRITICAL_ERROR@@YAXXZ 0002c688 f   gsmband.obj
 0001:0001b6a8       ??__EIOTA_NON_CRITICAL_ERROR@@YAXXZ 0002c6a8 f   gsmband.obj
 0001:0001b6c8       ??__EIOTA_KILL_ME@@YAXXZ   0002c6c8 f   gsmband.obj
 0001:0001b6e8       ??__EIOTA_UPDATE_STATUS@@YAXXZ 0002c6e8 f   gsmband.obj
 0001:0001b708       ??__EIOTA_DATAPORT_INUSE@@YAXXZ 0002c708 f   gsmband.obj
 0001:0001b728       ??__EIOTA_DONE@@YAXXZ      0002c728 f   gsmband.obj
 0001:0001b748       ??__EIOTA_DIAL@@YAXXZ      0002c748 f   gsmband.obj
 0001:0001b768       ??__EIOTA_1012_MIP_ERR@@YAXXZ 0002c768 f   gsmband.obj
 0001:0001b788       ??__EPHONEUTILS_BEGIN_MESSAGE@@YAXXZ 0002c788 f   gsmband.obj
 0001:0001b7a8       ??__EPHONEUTILS_END_MESSAGE@@YAXXZ 0002c7a8 f   gsmband.obj
 0001:0001b7c8       ??__EPHONEUTILS_BEGIN_ACK@@YAXXZ 0002c7c8 f   gsmband.obj
 0001:0001b7e8       ??__EPHONEUTILS_BEGIN_NACK@@YAXXZ 0002c7e8 f   gsmband.obj
 0001:0001b808       ??__EPHONEUTILS_END_ACK@@YAXXZ 0002c808 f   gsmband.obj
 0001:0001b828       ??__EPHONEUTILS_EXIT_MESSAGE@@YAXXZ 0002c828 f   gsmband.obj
 0001:0001b848       ??__EPHONEUTILS_ALIVE_MESSAGE@@YAXXZ 0002c848 f   gsmband.obj
 0001:0001b868       ??__EPHONEUTILS_PING_MESSAGE@@YAXXZ 0002c868 f   gsmband.obj
 0001:0001b888       ??__EPHONEUTILS_PING_ACK@@YAXXZ 0002c888 f   gsmband.obj
 0001:0001b8a8       ??__EAW_BEGIN_MESSAGE@@YAXXZ 0002c8a8 f   gsmband.obj
 0001:0001b8c8       ??__EAW_END_MESSAGE@@YAXXZ 0002c8c8 f   gsmband.obj
 0001:0001b8e8       ??__EAW_BEGIN_ACK@@YAXXZ   0002c8e8 f   gsmband.obj
 0001:0001b908       ??__EAW_BEGIN_NACK@@YAXXZ  0002c908 f   gsmband.obj
 0001:0001b928       ??__EAW_END_ACK@@YAXXZ     0002c928 f   gsmband.obj
 0001:0001b948       ??__EAW_EXIT_MESSAGE@@YAXXZ 0002c948 f   gsmband.obj
 0001:0001b968       ??__EAW_ALIVE_MESSAGE@@YAXXZ 0002c968 f   gsmband.obj
 0001:0001b988       ??__EAW_PING_MESSAGE@@YAXXZ 0002c988 f   gsmband.obj
 0001:0001b9a8       ??__EAW_PING_ACK@@YAXXZ    0002c9a8 f   gsmband.obj
 0001:0001b9c8       ??__EUPDATER_BEGIN@@YAXXZ  0002c9c8 f   gsmband.obj
 0001:0001b9e8       ??__EUPDATER_END@@YAXXZ    0002c9e8 f   gsmband.obj
 0001:0001ba08       ??__EUPDATER_BEGIN_ACK@@YAXXZ 0002ca08 f   gsmband.obj
 0001:0001ba28       ??__EUPDATER_BEGIN_NACK@@YAXXZ 0002ca28 f   gsmband.obj
 0001:0001ba48       ??__EUPDATER_END_ACK@@YAXXZ 0002ca48 f   gsmband.obj
 0001:0001ba68       ??__EUPDATER_END_NACK@@YAXXZ 0002ca68 f   gsmband.obj
 0001:0001ba88       ??__ERIL_STATUS_CHANGED@@YAXXZ 0002ca88 f   gsmband.obj
 0001:0001baa8       ??__ERIL_DBG_NOTIFY@@YAXXZ 0002caa8 f   gsmband.obj
 0001:0001bac8       ??__ERIL_TECHHDR_NOTIFY@@YAXXZ 0002cac8 f   gsmband.obj
 0001:0001bae8       ??__ERIL_IOTA_STATUS_CHANGED@@YAXXZ 0002cae8 f   gsmband.obj
 0001:0001bb08       ??__ERIL_IOTA_WAP_URI@@YAXXZ 0002cb08 f   gsmband.obj
 0001:0001bb28       ??__ERIL_PDSM_PD_DATA@@YAXXZ 0002cb28 f   gsmband.obj
 0001:0001bb48       ??__ERIL_PDSM_PD_DONE@@YAXXZ 0002cb48 f   gsmband.obj
 0001:0001bb68       ??__ERIL_PDSM_PD_END@@YAXXZ 0002cb68 f   gsmband.obj
 0001:0001bb88       ??__ERIL_PDSM_PD_BEGIN@@YAXXZ 0002cb88 f   gsmband.obj
 0001:0001bba8       ??__ERIL_PDSM_PD_UPDATE_FAILURE@@YAXXZ 0002cba8 f   gsmband.obj
 0001:0001bbc8       ??__ERIL_PDSM_PD_DLD_DATA@@YAXXZ 0002cbc8 f   gsmband.obj
 0001:0001bbe8       ??__ERIL_PDSM_PD_DLD_DONE@@YAXXZ 0002cbe8 f   gsmband.obj
 0001:0001bc08       ??__ERIL_PDSM_PD_DLD_END@@YAXXZ 0002cc08 f   gsmband.obj
 0001:0001bc28       ??__ERIL_PDSM_PD_DLD_BEGIN@@YAXXZ 0002cc28 f   gsmband.obj
 0001:0001bc48       ??__ERIL_PDSM_PA_PARAM@@YAXXZ 0002cc48 f   gsmband.obj
 0001:0001bc68       ??__ERIL_CALL_BYTE_CTR@@YAXXZ 0002cc68 f   gsmband.obj
 0001:0001bc88       ??__ERIL_CREATE_MAIN_LIST@@YAXXZ 0002cc88 f   gsmband.obj
 0001:0001bca8       ??__ERIL_STATUS_CHANGED@@YAXXZ 0002cca8 f   iota.obj
 0001:0001bcc8       ??__ERIL_STATUS_CHANGED@@YAXXZ 0002ccc8 f   loopbackdlg.obj
 0001:0001bce8       ??__EPHONEUTILS_BEGIN_MESSAGE@@YAXXZ 0002cce8 f   mainfrm.obj
 0001:0001bd08       ??__EPHONEUTILS_END_MESSAGE@@YAXXZ 0002cd08 f   mainfrm.obj
 0001:0001bd28       ??__EPHONEUTILS_BEGIN_ACK@@YAXXZ 0002cd28 f   mainfrm.obj
 0001:0001bd48       ??__EPHONEUTILS_BEGIN_NACK@@YAXXZ 0002cd48 f   mainfrm.obj
 0001:0001bd68       ??__EPHONEUTILS_EXIT_MESSAGE@@YAXXZ 0002cd68 f   mainfrm.obj
 0001:0001bd88       ??__EPHONEUTILS_END_MESSAGE@@YAXXZ 0002cd88 f   msldlg.obj
 0001:0001bda8       ??__ERIL_STATUS_CHANGED@@YAXXZ 0002cda8 f   msldlg.obj
 0001:0001bdc8       ??__ERIL_STATUS_CHANGED@@YAXXZ 0002cdc8 f   network.obj
 0001:0001bde8       ??__EPHONEUTILS_END_MESSAGE@@YAXXZ 0002cde8 f   otksldlg.obj
 0001:0001be08       ??__ERIL_STATUS_CHANGED@@YAXXZ 0002ce08 f   otksldlg.obj
 0001:0001be28       ??__EPHONEUTILS_END_MESSAGE@@YAXXZ 0002ce28 f   passthrudlg.obj
 0001:0001be48       ??__EPHONEUTILS_END_MESSAGE@@YAXXZ 0002ce48 f   rtndlg.obj
 0001:0001be68       ??__ERIL_STATUS_CHANGED@@YAXXZ 0002ce68 f   rtndlg.obj
 0001:0001be88       ??__ERIL_STATUS_CHANGED@@YAXXZ 0002ce88 f   simpleipdlg.obj
 0001:0001bea8       ??__ERIL_STATUS_CHANGED@@YAXXZ 0002cea8 f   sipdlg.obj
 0001:0001bec8       ??__EPHONEUTILS_END_MESSAGE@@YAXXZ 0002cec8 f   spcvalidation.obj
 0001:0001bee8       ??__ERIL_STATUS_CHANGED@@YAXXZ 0002cee8 f   spcvalidation.obj
 0001:0001bf08       ??__EPOWER_ON@@YAXXZ       0002cf08 f   stdafx.obj
 0001:0001bf28       ??__EPOWER_OFF@@YAXXZ      0002cf28 f   stdafx.obj
 0001:0001bf48       ??__EIOTA_BEGIN_MESSAGE@@YAXXZ 0002cf48 f   stdafx.obj
 0001:0001bf68       ??__EIOTA_END_MESSAGE@@YAXXZ 0002cf68 f   stdafx.obj
 0001:0001bf88       ??__EIOTA_BEGIN_ACK@@YAXXZ 0002cf88 f   stdafx.obj
 0001:0001bfa8       ??__EIOTA_BEGIN_NACK@@YAXXZ 0002cfa8 f   stdafx.obj
 0001:0001bfc8       ??__EIOTA_END_ACK@@YAXXZ   0002cfc8 f   stdafx.obj
 0001:0001bfe8       ??__EIOTA_EXIT_MESSAGE@@YAXXZ 0002cfe8 f   stdafx.obj
 0001:0001c008       ??__EIOTA_ALIVE_MESSAGE@@YAXXZ 0002d008 f   stdafx.obj
 0001:0001c028       ??__EIOTA_PING_MESSAGE@@YAXXZ 0002d028 f   stdafx.obj
 0001:0001c048       ??__EIOTA_PING_ACK@@YAXXZ  0002d048 f   stdafx.obj
 0001:0001c068       ??__EIOTA_CRITICAL_ERROR@@YAXXZ 0002d068 f   stdafx.obj
 0001:0001c088       ??__EIOTA_NON_CRITICAL_ERROR@@YAXXZ 0002d088 f   stdafx.obj
 0001:0001c0a8       ??__EIOTA_KILL_ME@@YAXXZ   0002d0a8 f   stdafx.obj
 0001:0001c0c8       ??__EIOTA_UPDATE_STATUS@@YAXXZ 0002d0c8 f   stdafx.obj
 0001:0001c0e8       ??__EIOTA_DATAPORT_INUSE@@YAXXZ 0002d0e8 f   stdafx.obj
 0001:0001c108       ??__EIOTA_DONE@@YAXXZ      0002d108 f   stdafx.obj
 0001:0001c128       ??__EIOTA_DIAL@@YAXXZ      0002d128 f   stdafx.obj
 0001:0001c148       ??__EIOTA_1012_MIP_ERR@@YAXXZ 0002d148 f   stdafx.obj
 0001:0001c168       ??__EPHONEUTILS_BEGIN_MESSAGE@@YAXXZ 0002d168 f   stdafx.obj
 0001:0001c188       ??__EPHONEUTILS_END_MESSAGE@@YAXXZ 0002d188 f   stdafx.obj
 0001:0001c1a8       ??__EPHONEUTILS_BEGIN_ACK@@YAXXZ 0002d1a8 f   stdafx.obj
 0001:0001c1c8       ??__EPHONEUTILS_BEGIN_NACK@@YAXXZ 0002d1c8 f   stdafx.obj
 0001:0001c1e8       ??__EPHONEUTILS_END_ACK@@YAXXZ 0002d1e8 f   stdafx.obj
 0001:0001c208       ??__EPHONEUTILS_EXIT_MESSAGE@@YAXXZ 0002d208 f   stdafx.obj
 0001:0001c228       ??__EPHONEUTILS_ALIVE_MESSAGE@@YAXXZ 0002d228 f   stdafx.obj
 0001:0001c248       ??__EPHONEUTILS_PING_MESSAGE@@YAXXZ 0002d248 f   stdafx.obj
 0001:0001c268       ??__EPHONEUTILS_PING_ACK@@YAXXZ 0002d268 f   stdafx.obj
 0001:0001c288       ??__EAW_BEGIN_MESSAGE@@YAXXZ 0002d288 f   stdafx.obj
 0001:0001c2a8       ??__EAW_END_MESSAGE@@YAXXZ 0002d2a8 f   stdafx.obj
 0001:0001c2c8       ??__EAW_BEGIN_ACK@@YAXXZ   0002d2c8 f   stdafx.obj
 0001:0001c2e8       ??__EAW_BEGIN_NACK@@YAXXZ  0002d2e8 f   stdafx.obj
 0001:0001c308       ??__EAW_END_ACK@@YAXXZ     0002d308 f   stdafx.obj
 0001:0001c328       ??__EAW_EXIT_MESSAGE@@YAXXZ 0002d328 f   stdafx.obj
 0001:0001c348       ??__EAW_ALIVE_MESSAGE@@YAXXZ 0002d348 f   stdafx.obj
 0001:0001c368       ??__EAW_PING_MESSAGE@@YAXXZ 0002d368 f   stdafx.obj
 0001:0001c388       ??__EAW_PING_ACK@@YAXXZ    0002d388 f   stdafx.obj
 0001:0001c3a8       ??__EUPDATER_BEGIN@@YAXXZ  0002d3a8 f   stdafx.obj
 0001:0001c3c8       ??__EUPDATER_END@@YAXXZ    0002d3c8 f   stdafx.obj
 0001:0001c3e8       ??__EUPDATER_BEGIN_ACK@@YAXXZ 0002d3e8 f   stdafx.obj
 0001:0001c408       ??__EUPDATER_BEGIN_NACK@@YAXXZ 0002d408 f   stdafx.obj
 0001:0001c428       ??__EUPDATER_END_ACK@@YAXXZ 0002d428 f   stdafx.obj
 0001:0001c448       ??__EUPDATER_END_NACK@@YAXXZ 0002d448 f   stdafx.obj
 0001:0001c468       ??__ERIL_STATUS_CHANGED@@YAXXZ 0002d468 f   stdafx.obj
 0001:0001c488       ??__ERIL_DBG_NOTIFY@@YAXXZ 0002d488 f   stdafx.obj
 0001:0001c4a8       ??__ERIL_TECHHDR_NOTIFY@@YAXXZ 0002d4a8 f   stdafx.obj
 0001:0001c4c8       ??__ERIL_IOTA_STATUS_CHANGED@@YAXXZ 0002d4c8 f   stdafx.obj
 0001:0001c4e8       ??__ERIL_IOTA_WAP_URI@@YAXXZ 0002d4e8 f   stdafx.obj
 0001:0001c508       ??__ERIL_PDSM_PD_DATA@@YAXXZ 0002d508 f   stdafx.obj
 0001:0001c528       ??__ERIL_PDSM_PD_DONE@@YAXXZ 0002d528 f   stdafx.obj
 0001:0001c548       ??__ERIL_PDSM_PD_END@@YAXXZ 0002d548 f   stdafx.obj
 0001:0001c568       ??__ERIL_PDSM_PD_BEGIN@@YAXXZ 0002d568 f   stdafx.obj
 0001:0001c588       ??__ERIL_PDSM_PD_UPDATE_FAILURE@@YAXXZ 0002d588 f   stdafx.obj
 0001:0001c5a8       ??__ERIL_PDSM_PD_DLD_DATA@@YAXXZ 0002d5a8 f   stdafx.obj
 0001:0001c5c8       ??__ERIL_PDSM_PD_DLD_DONE@@YAXXZ 0002d5c8 f   stdafx.obj
 0001:0001c5e8       ??__ERIL_PDSM_PD_DLD_END@@YAXXZ 0002d5e8 f   stdafx.obj
 0001:0001c608       ??__ERIL_PDSM_PD_DLD_BEGIN@@YAXXZ 0002d608 f   stdafx.obj
 0001:0001c628       ??__ERIL_PDSM_PA_PARAM@@YAXXZ 0002d628 f   stdafx.obj
 0001:0001c648       ??__ERIL_CALL_BYTE_CTR@@YAXXZ 0002d648 f   stdafx.obj
 0001:0001c668       ??__ERIL_CREATE_MAIN_LIST@@YAXXZ 0002d668 f   stdafx.obj
 0001:0001c688       ??__ERIL_STATUS_CHANGED@@YAXXZ 0002d688 f   systemdlg.obj
 0001:0001c6a8       ??__ERIL_STATUS_CHANGED@@YAXXZ 0002d6a8 f   usernamedlg.obj
 0001:0001c6c8       ??__EPOWER_ON@@YAXXZ       0002d6c8 f   versioninfo.obj
 0001:0001c6e8       ??__EPOWER_OFF@@YAXXZ      0002d6e8 f   versioninfo.obj
 0001:0001c708       ??__EIOTA_BEGIN_MESSAGE@@YAXXZ 0002d708 f   versioninfo.obj
 0001:0001c728       ??__EIOTA_END_MESSAGE@@YAXXZ 0002d728 f   versioninfo.obj
 0001:0001c748       ??__EIOTA_BEGIN_ACK@@YAXXZ 0002d748 f   versioninfo.obj
 0001:0001c768       ??__EIOTA_BEGIN_NACK@@YAXXZ 0002d768 f   versioninfo.obj
 0001:0001c788       ??__EIOTA_END_ACK@@YAXXZ   0002d788 f   versioninfo.obj
 0001:0001c7a8       ??__EIOTA_EXIT_MESSAGE@@YAXXZ 0002d7a8 f   versioninfo.obj
 0001:0001c7c8       ??__EIOTA_ALIVE_MESSAGE@@YAXXZ 0002d7c8 f   versioninfo.obj
 0001:0001c7e8       ??__EIOTA_PING_MESSAGE@@YAXXZ 0002d7e8 f   versioninfo.obj
 0001:0001c808       ??__EIOTA_PING_ACK@@YAXXZ  0002d808 f   versioninfo.obj
 0001:0001c828       ??__EIOTA_CRITICAL_ERROR@@YAXXZ 0002d828 f   versioninfo.obj
 0001:0001c848       ??__EIOTA_NON_CRITICAL_ERROR@@YAXXZ 0002d848 f   versioninfo.obj
 0001:0001c868       ??__EIOTA_KILL_ME@@YAXXZ   0002d868 f   versioninfo.obj
 0001:0001c888       ??__EIOTA_UPDATE_STATUS@@YAXXZ 0002d888 f   versioninfo.obj
 0001:0001c8a8       ??__EIOTA_DATAPORT_INUSE@@YAXXZ 0002d8a8 f   versioninfo.obj
 0001:0001c8c8       ??__EIOTA_DONE@@YAXXZ      0002d8c8 f   versioninfo.obj
 0001:0001c8e8       ??__EIOTA_DIAL@@YAXXZ      0002d8e8 f   versioninfo.obj
 0001:0001c908       ??__EIOTA_1012_MIP_ERR@@YAXXZ 0002d908 f   versioninfo.obj
 0001:0001c928       ??__EPHONEUTILS_BEGIN_MESSAGE@@YAXXZ 0002d928 f   versioninfo.obj
 0001:0001c948       ??__EPHONEUTILS_END_MESSAGE@@YAXXZ 0002d948 f   versioninfo.obj
 0001:0001c968       ??__EPHONEUTILS_BEGIN_ACK@@YAXXZ 0002d968 f   versioninfo.obj
 0001:0001c988       ??__EPHONEUTILS_BEGIN_NACK@@YAXXZ 0002d988 f   versioninfo.obj
 0001:0001c9a8       ??__EPHONEUTILS_END_ACK@@YAXXZ 0002d9a8 f   versioninfo.obj
 0001:0001c9c8       ??__EPHONEUTILS_EXIT_MESSAGE@@YAXXZ 0002d9c8 f   versioninfo.obj
 0001:0001c9e8       ??__EPHONEUTILS_ALIVE_MESSAGE@@YAXXZ 0002d9e8 f   versioninfo.obj
 0001:0001ca08       ??__EPHONEUTILS_PING_MESSAGE@@YAXXZ 0002da08 f   versioninfo.obj
 0001:0001ca28       ??__EPHONEUTILS_PING_ACK@@YAXXZ 0002da28 f   versioninfo.obj
 0001:0001ca48       ??__EAW_BEGIN_MESSAGE@@YAXXZ 0002da48 f   versioninfo.obj
 0001:0001ca68       ??__EAW_END_MESSAGE@@YAXXZ 0002da68 f   versioninfo.obj
 0001:0001ca88       ??__EAW_BEGIN_ACK@@YAXXZ   0002da88 f   versioninfo.obj
 0001:0001caa8       ??__EAW_BEGIN_NACK@@YAXXZ  0002daa8 f   versioninfo.obj
 0001:0001cac8       ??__EAW_END_ACK@@YAXXZ     0002dac8 f   versioninfo.obj
 0001:0001cae8       ??__EAW_EXIT_MESSAGE@@YAXXZ 0002dae8 f   versioninfo.obj
 0001:0001cb08       ??__EAW_ALIVE_MESSAGE@@YAXXZ 0002db08 f   versioninfo.obj
 0001:0001cb28       ??__EAW_PING_MESSAGE@@YAXXZ 0002db28 f   versioninfo.obj
 0001:0001cb48       ??__EAW_PING_ACK@@YAXXZ    0002db48 f   versioninfo.obj
 0001:0001cb68       ??__EUPDATER_BEGIN@@YAXXZ  0002db68 f   versioninfo.obj
 0001:0001cb88       ??__EUPDATER_END@@YAXXZ    0002db88 f   versioninfo.obj
 0001:0001cba8       ??__EUPDATER_BEGIN_ACK@@YAXXZ 0002dba8 f   versioninfo.obj
 0001:0001cbc8       ??__EUPDATER_BEGIN_NACK@@YAXXZ 0002dbc8 f   versioninfo.obj
 0001:0001cbe8       ??__EUPDATER_END_ACK@@YAXXZ 0002dbe8 f   versioninfo.obj
 0001:0001cc08       ??__EUPDATER_END_NACK@@YAXXZ 0002dc08 f   versioninfo.obj
 0001:0001cc28       ??__ERIL_STATUS_CHANGED@@YAXXZ 0002dc28 f   versioninfo.obj
 0001:0001cc48       ??__ERIL_DBG_NOTIFY@@YAXXZ 0002dc48 f   versioninfo.obj
 0001:0001cc68       ??__ERIL_TECHHDR_NOTIFY@@YAXXZ 0002dc68 f   versioninfo.obj
 0001:0001cc88       ??__ERIL_IOTA_STATUS_CHANGED@@YAXXZ 0002dc88 f   versioninfo.obj
 0001:0001cca8       ??__ERIL_IOTA_WAP_URI@@YAXXZ 0002dca8 f   versioninfo.obj
 0001:0001ccc8       ??__ERIL_PDSM_PD_DATA@@YAXXZ 0002dcc8 f   versioninfo.obj
 0001:0001cce8       ??__ERIL_PDSM_PD_DONE@@YAXXZ 0002dce8 f   versioninfo.obj
 0001:0001cd08       ??__ERIL_PDSM_PD_END@@YAXXZ 0002dd08 f   versioninfo.obj
 0001:0001cd28       ??__ERIL_PDSM_PD_BEGIN@@YAXXZ 0002dd28 f   versioninfo.obj
 0001:0001cd48       ??__ERIL_PDSM_PD_UPDATE_FAILURE@@YAXXZ 0002dd48 f   versioninfo.obj
 0001:0001cd68       ??__ERIL_PDSM_PD_DLD_DATA@@YAXXZ 0002dd68 f   versioninfo.obj
 0001:0001cd88       ??__ERIL_PDSM_PD_DLD_DONE@@YAXXZ 0002dd88 f   versioninfo.obj
 0001:0001cda8       ??__ERIL_PDSM_PD_DLD_END@@YAXXZ 0002dda8 f   versioninfo.obj
 0001:0001cdc8       ??__ERIL_PDSM_PD_DLD_BEGIN@@YAXXZ 0002ddc8 f   versioninfo.obj
 0001:0001cde8       ??__ERIL_PDSM_PA_PARAM@@YAXXZ 0002dde8 f   versioninfo.obj
 0001:0001ce08       ??__ERIL_CALL_BYTE_CTR@@YAXXZ 0002de08 f   versioninfo.obj
 0001:0001ce28       ??__ERIL_CREATE_MAIN_LIST@@YAXXZ 0002de28 f   versioninfo.obj
 0001:0001ce48       ??__EPHONEUTILS_END_MESSAGE@@YAXXZ 0002de48 f   vocoderdlg.obj
 0001:0001ce68       ??__ERIL_STATUS_CHANGED@@YAXXZ 0002de68 f   vocoderdlg.obj
